:020000040000FA
:06000000020A000201B03B
:03002B000209BF08
:030033000206388A
:030043000208822E
:03004B00020702A7
:03005300020103A4
:03005B0002071188
:0300630002071D74
:03006B0002061E6C
:1000830002014C0101FF0503010F030003000300FC
:1000930003000300030003000300030005000A003C
:1000A300140028004F009E0000001D101D101D109D
:1000B3001D10DF0ED90E1D10D81B000000003A1CC6
:1000C300000000000C0000000C0001BB05FF010054
:1000D30001010100630E000000D80EE80364006410
:1000E30000B8010202000800000502071E02051EF7
:1000F30003B80B020103320002F7FF0202020605F6
:10010300C0E074F21203C2E5A7F8E5A1F958541050
:10011300600812168F53A1EF802AE8A2E0C0D0E94D
:10012300A2E092F012099B158182F050179061981A
:10013300E0F89011EBE0C398A2D265D0335002E807
:10014300F053A1FE7F01020421C0E074F21203C246
:100153009061A4E0F8759B00E59158540860087518
:1001630091F71216D1802AE59158541060087591C1
:10017300EF1216D7801BE8A2E0C0D0E591A2E0926F
:10018300F012099B158182F05007E0C2E0F01217CC
:10019300F79061A3E0F8E5E9585404600E1217CD17
:1001A30075E9FB906193E0A2E640F28097C0E074AA
:1001B300F21203C29061A5E0F8E5BF58540460064B
:1001C30053BFFB12180F020147C3E498F8E499F9EF
:1001D30012020D8026C3E49AFAE49BFBE920E7E9C7
:1001E30012020DE498F8E499F922C3E498F8E4992B
:1001F300F912020DE498F8E499F9C3E49AFAE49B3E
:10020300FB22EB20E7CFE920E7E0B90010BB0008B1
:10021300E88AF084F8AAF022E4FBC8FA22EB702201
:100223007B10C833C8C933C9335007C39AC3DBF241
:1002330080069A50012ADBEAC833F4C8C933F4C9EB
:10024300FA2275F008E4C833C8C933C933C99AC957
:100253009B5004C92AC93BD5F0ECFBC833F4C8E46E
:10026300C9FA22080808EAC0E0EBC0E086F0E7A478
:10027300FA180986F0E7A42AFA180986F0E7A42AEF
:10028300FA180986F0E7A42AFA1986F0E7A4FBE531
:10029300F02AFA190886F0E7A42BFBE5F03AFA19DD
:1002A3000886F0E7A42BFBE5F03AFA18180986F064
:1002B300E7A4C5F02BFBE43AFA1908E7C5F0C6A496
:1002C30026F6E5F03BFBE43AFA1886F0E7A4F6E5F8
:1002D300F00826F6E43B08F6E43A08F6D0E0FBD053
:1002E300E0FA22E4CFC0E0E4CEC0E0E4CDC0E0E435
:1002F300CCC0E075F020C3E633F608E633F608E633
:1003030033F608E633F6181818EC33FCED33FDEE3C
:1003130033FEEF33FFC3EC9709ED9709EE9709EF2F
:1003230097191919400FFFEC97FC09ED97FD09EE9A
:1003330097FE191906D5F0BEECF709EDF709EEF7AC
:1003430009EFF7191919D0E0FCD0E0FDD0E0FED099
:10035300E0FF222510C582C0E0E51134FFC583C04C
:10036300E0E510C3958224F810AF088583118582D8
:10037300108008858311858210D2AFCEF0A3E520CB
:10038300F0A37808E608F0A3DEFAEFF0A3E58124F2
:10039300FAF8E608F0A3E608F0A3E608F0A30808D5
:1003A300E608F0A3E608F0A315811581D0E0FED09E
:1003B300E0F8158115811581E8C0E0EEC0E022C0A8
:1003C300D02510C582C0E0E51134FFC583C0E0E548
:1003D30010C3958224F310AF0885831185821080A2
:1003E30008858311858210D2AFC8F0A3E9F0A3EA90
:1003F300F0A3EBF0A37908E709F0A3D8FAECF0A394
:10040300EDF0A3EEF0A3EFF0A3D0E0F0A3D0E0F083
:10041300A3D0E0F0A3E520F0A3E5F0F0A32285113B
:1004230083851082E0C0E0A3E0F9A3E0FAA3E0FB38
:10043300A37808E0F608A3DFFAE0FCA3E0FDA3E05D
:10044300FEA3E0FFA3E0C0E0A3E0C0E0A3E0F5D09B
:10045300A3E0F520A3E0A3F5F010AF088583118591
:1004630082108008858311858210D2AFD082D08319
:10047300D0E0F8D0E032120A62B900030204BBE410
:10048300900400784179118002F0A3D8FCD9FA9046
:100493001440AA82AB83900086787E79018015E4AC
:1004A30093A3AC82AD838A828B83F0A3AA82AB83AE
:1004B3008C828D83D8E9D9E77582BF7583DB74029B
:1004C3001207C975828575831A74001207C9D08310
:1004D300D082ECC0E0EDC0E0E493A3FCE493A3FD81
:1004E300ED4C600D1205A9EC24FFFCED34FFFD80FB
:1004F300EFE493A3FCE493A3FDED4C600D1206AD72
:10050300EC24FFFCED34FFFD80EFD0E0FDD0E0FCF8
:10051300E493A3C0E0E493C0E022D083D082E9C097
:10052300E0E493A3C386F0C5F095F0F908E493A340
:1005330086F0C5F095F0700BE493A3C3994005E9E9
:10054300048002A3E475F002A42582F582E5F03568
:1005530083F583D0E0F9E493A3C0E0E493C0E02201
:10056300851183851082E0A3FEE0A3F5207808E0DF
:10057300A3F608DFFAE0A3FFE0A3C0E0E0A3C0E036
:10058300E0A3C0E0E0A3C0E0E0A3C0E010AF0885B3
:1005930082108583118008858210858311D2AFD0A4
:1005A30083D0820207CFC0E0C3E49396087401931B
:1005B3009618400FE49366700808740193661870E8
:1005C300007019A3A3C3E49396087401939618A328
:1005D300A3400DD0E0D0E0D0E002050DA3A3A3A378
:1005E300A3A3D0E022D083D082C5F0E493A3C5F0C7
:1005F300C395F0F5F0E493A3C395F04005E5F0044B
:100603008001E475F002A42582F582E5F03583F5D7
:1006130083E493A3C0E0E493C0E022C0E074F21249
:1006230003C2E589A2E1500312155D758900C2C5B5
:100633007F01020421C0E074F21203C2E58BA2E041
:10064300500312155D758B00C2E880E474048004C6
:1006530074028000CCC0E0EDC0E0E510C39CCCADDB
:100663001150011D10AF068C108D1180068C108D5A
:1006730011D2AF12074BD0E0FDD0E0FC2274028010
:1006830000CCC0E0EDC0E0E510C39CCCAD1150013F
:100693001D10AF068C108D1180068C108D11D2AFFA
:1006A300120729D0E0FDD0E0FC22C0E0C0F088F0C2
:1006B300E4936670080874019366187000A8F0A3A9
:1006C300A3700BD0F0D0E0D0E0D0E002050DA3A3DF
:1006D300D0F0D0E022D083D082CCC0E0E493A360FA
:1006E300061207AA1470FAE493A360061208991479
:1006F30070FAD0E0FCE493A3C0E0E493C0E022C02E
:10070300E074F21203C21215E17F01020421C0E07A
:1007130074F21203C21215E780EFC0E074F2120301
:10072300C21215ED80E3CAC0E0E493A3C582CCC531
:1007330082C583CDC583F0A3C582CCC582C583CDD5
:10074300C583DAE5D0E0CA22CAC0E0E0A3C582CC03
:10075300C582C583CDC583F0A3C582CCC582C583BD
:10076300CDC583DAE6D0E0CA22C008C3E096F50817
:1007730008A3E096420808A3E096420808A3E0967F
:1007830045087001D3D008227009080808226016B2
:10079300181818C6C333C608C633C608C633C608F6
:1007A300C633C6D5E0EA22C0E0E493A3D39C50103D
:1007B300E493A3C39C400AD0E0D0E0D0E00206F566
:1007C300A3A3A3D0E022C09FF59FE473D09F22D0C0
:1007D30083D082C09FE493C0E0740193C0E07402AD
:1007E30093F59F227404800A7403800674028002C6
:1007F3007401C0E0F404120802D0E0120A3D22257D
:1008030010F58210AF08F510400215118008F5109D
:1008130040021511D2AF85118322C0D0251010AF2D
:1008230008F510500205118008F51050020511D289
:10083300AFD0D022BB0102E722C082C08389828A63
:1008430083BB0003E08002E493D083D0822260164E
:10085300080808C6C313C618C613C618C613C61895
:10086300C613C6D5E0EA22C3E0C696F608A3E0C6DF
:1008730096F608A3E0C696F608A3E0C696F622C04D
:10088300E074F21203C2C2C0E5D1A2E4500312160F
:10089300117F01020421C0E0E493A36C7009D0E04E
:1008A300D0E0D0E00206F5A3A3D0E022251010AFDC
:1008B30008F510400215118008F51040021511D2F9
:1008C300AF22C3E09608A3E09608A3E09608A3E04E
:1008D30096A2D265D03322E066701008A3E066705A
:1008E3000A08A3E066700408A3E06622C3E096F05A
:1008F30008A3E096F008A3E096F008A3E096F022A0
:10090300E026F608A3E036F608A3E036F608A3E0EF
:1009130036F622E627F60809E637F60809E637F63B
:100923000809E637F622E056F608A3E056F608A3D0
:10093300E056F608A3E056F622E056F008A3E05688
:10094300F008A3E056F008A3E056F022E657F608B5
:1009530009E657F60809E657F60809E657F622E0CE
:1009630026F008A3E036F008A3E036F008A3E0364B
:10097300F022E647F60809E647F60809E647F608CF
:1009830009E647F622700422600D18C6C333C60871
:10099300C633C6D5E0F41822C0E0E8C0E0E5812400
:1009A300FCF8E6A2E7D0E0F8D0E022E4C396F6082C
:1009B300E496F608E496F608E496F622C0E074F2AC
:1009C3001203C2C2C71217137F01020421C6F4C661
:1009D30008C6F4C608C6F4C608C6F4C622C3E7961A
:1009E3000809E7960809E7960809E79622C3E096FF
:1009F30008A3E09608A3E09608A3E0962275D0002A
:100A030075814075100075110400020479600C08AB
:100A1300C6C313C618C613C6D5E0F422E6F008A36E
:100A2300E6F008A3E6F008A3E6F022E0F608A3E068
:100A3300F608A3E0F608A3E0F622CAC0E0E6F0A3B6
:100A430008DAFAD0E0FA22E0FAA3E0FBA3E0FCA381
:100A5300E0FD22EAF0A3EBF0A3ECF0A3EDF022E536
:100A6300C754F84401F5C77901222510F582E4350E
:100A730011F583221207D22CB3011207D269B401F4
:100A83001207D204B5011207D204B6011207D2220B
:100A9300B6011207D29B5B001207D2AD5B001207AF
:100AA300D2DB5B001207D23D5C001207D2C25C00AE
:100AB3001207D2605D001207D2E35D001207D2FE77
:100AC3005D001207D2255E001207D2605E00120796
:100AD300D2A05E001207D2F05E001207D2AA5F0016
:100AE3001207D22F60001207D2B660001207D29EFF
:100AF30061001207D2F761001207D26F620012077A
:100B0300D28162001207D28B62001207D26863009F
:100B13001207D2C763001207D2C964001207D24278
:100B230065001207D29665001207D20B6600120702
:100B3300D2B767001207D2CB67001207D22D680025
:100B43001207D2B268001207D2FF68001207D22739
:100B53006A001207D2126B001207D27F6B001207D2
:100B6300D2FB6B001207D25D6C001207D2956C00AA
:100B73001207D2706D001207D2706E001207D2CD29
:100B83006E001207D2166F001207D23E6F001207D3
:100B9300D2C76F001207D25D70001207D2C3700074
:100BA3001207D2D470001207D24D71001207D2DAA5
:100BB30071001207D21C72001207D2AC7200120726
:100BC300D2E172001207D22273001207D2BB740063
:100BD3001207D25A76001207D29676001207D2B7BE
:100BE30077001207D28679001207D2907900120794
:100BF300D29A79001207D2A479001207D2AE7900F3
:100C03001207D2B879001207D2C279001207D210A4
:100C13007A001207D2347A001207D2587A001207E8
:100C2300D2B17A001207D2F67A001207D2147B00EF
:100C33001207D28B7B001207D2D57B001207D20B8F
:100C43007C001207D2A07D001207D22C1E001207CF
:100C5300D2781E001207D24420001207D28220004D
:100C63001207D22421001207D25821001207D27D85
:100C730021001207D2DA22001207D2DA2300120768
:100C8300D2AC26001207D29D27001207D2472800B4
:100C93001207D26229001207D29B2C001207D22717
:100CA3002D001207D25C2D001207D2342E0012073A
:100CB300D20A2F001207D2AD2F001207D20830003C
:100CC3001207D23530001207D25730001207D29DD7
:100CD30032001207D24F33001207D2A63300120795
:100CE300D21334001207D2D434001207D2093500CC
:100CF3001207D25D35001207D29235001207D2E0F7
:100D030035001207D23736001207D2C23600120757
:100D1300D24B38001207D20839001207D2373A00F3
:100D23001207D2A63C001207D24E3D001207D27121
:100D33003F001207D20E40001207D255400012079F
:100D4300D21C42001207D23042001207D23D4200A9
:100D53001207D26742001207D27342001207D291E0
:100D630042001207D25B43001207D28543001207E9
:100D7300D29243001207D2EA43001207D270440012
:100D83001207D25745001207D24946001207D2F97B
:100D930046001207D29747001207D2AE4700120748
:100DA300D2E747001207D20548001207D24948008C
:100DB3001207D27048001207D26C49001207D2E71B
:100DC30049001207D20A4B001207D21C4C0012072B
:100DD300D20D4D001207D2744D001207D24E4E00B1
:100DE3001207D2824E001207D2F84E001207D21D0C
:100DF3004F001207D2434F001207D2794F00120758
:100E0300D27D51001207D26F52001207D234530021
:100E13001207D2B454001207D2FD54001207D2298C
:100E230055001207D2B055001207D2185600120708
:100E3300D26A56001207D2B156001207D2DD56000D
:100E43001207D21257001207D23957001207D2974E
:100E530057001207D27458001207D2DC5800120749
:100E6300D20559001207D27559001207D2EA590068
:100E73001207D23C5A001207D2615A001207D2A7B6
:100E83005A001207D2C45A001207D2615B0012073C
:100E9300D2ABFF011207D2F6FF011207D27DB701D1
:100EA3001207D2C8B7011207D223B8011207D274AE
:100EB300B8011207D28FB8011207D2C5B8011207C1
:100EC300D2E6B8011207D2F0B8011207D205BA016F
:100ED3001207D223BA011207D293BA011207D2A67C
:100EE300BA011207D2B4BA011207D255BB011207D5
:100EF300D229BC011207D244BD011207D2C0BD01E1
:100F03001207D2CABD011207D23DBE011207D25445
:100F1300BE011207D296BE011207D2D4BE01120738
:100F2300D203BF011207D23ABF011207D258BF0141
:100F33001207D27CBF011207D2BDBF011207D2A88C
:100F4300C0011207D2EEC0011207D219C101120764
:100F5300D286C1011207D2ADC1011207D2F2C1017B
:100F63001207D200C2011207D259C2011207D29648
:100F7300C2011207D2DDC2011207D20EC30112074A
:100F8300D231C3011207D23CC3011207D25AC301A3
:100F93001207D216C4011207D220C4011207D25F6E
:100FA300C4011207D275C4011207D27EC40112070D
:100FB300D2C2C4011207D2D6C4011207D2C1C501DD
:100FC3001207D2D4C5011207D2E9C5011207D29183
:100FD300C6011207D2DDC6011207D293C701120759
:100FE300D29EC7011207D2ECC8011207D218C90159
:100FF3001207D259C9011207D273C9011207D2AA23
:10100300C9011207D20DCC011207D295CC011207E8
:10101300D215CD011207D258CF011207D268CF01E2
:101023001207D26BCF011207D277CF011207D28BEF
:10103300CF011207D2AACF011207D2DDCF011207C7
:10104300D2A2D0011207D209D1011207D26DD10168
:101053001207D2F7D1011207D2A8D2011207D2CFB9
:10106300D2011207D25FD3011207D26BD301120749
:10107300D29AD3011207D2BCD3011207D2E3D30110
:101083001207D248D4011207D2FBD5011207D2FEB0
:10109300D5011207D268D6011207D25BD701120716
:1010A300D240D8011207D2CBD8011207D20EDA01EF
:1010B3001207D2D1DA011207D20ADB011207D23B9F
:1010C300DB011207D244DB011207D228DC0112072D
:1010D300D2B8DC011207D256DD011207D216DE01A7
:1010E3001207D28FDE011207D2BEDE011207D2FB36
:1010F300DE011207D2AD99021207D2BB9902120781
:10110300D2319A021207D2699A021207D2B19A0215
:101113001207D2B89C021207D29A9E021207D25922
:10112300A1021207D285A1021207D2A5A1021207BA
:10113300D208A2021207D246A2021207D272A20258
:101143001207D2ACA2021207D219F5021207D24932
:10115300F5021207D29EF5021207D2F7A202120776
:10116300D201A3021207D245A3021207D2ECA302B3
:101173001207D20FA4021207D2AFA4021207D2772A
:10118300A7021207D285A7021207D2D8A702120715
:10119300D2FEA7021207D256A8021207D2C6A8028D
:1011A3001207D219A9021207D282A9021207D2008A
:1011B300AA021207D260AA021207D29FAA0212073A
:1011C300D2B1AA021207D2C3AA021207D2E2AA021A
:1011D3001207D2C3A7011207D2BEAB021207D289EC
:1011E300FB021207D2ADF1021207D20CF202120770
:1011F300D235F2021207D22BF3021207D23CDF01DF
:101203001207D21BE0011207D257E0011207D200E6
:10121300E2011207D242E2011207D2EDE301120703
:10122300D231E4011207D2EDB0011207D286E501F3
:101233001207D217E6011207D26DE6011207D2ADEB
:10124300E6011207D253E8011207D2F8E9011207A7
:10125300D246EC011207D254EC011207D2BCEC01C6
:101263001207D2F8EF011207D20981031207D289BC
:10127300FF021207D29DE4021207D2B0E402120762
:10128300D23DE5021207D278E5021207D293E502B6
:101293001207D2B8E5021207D2ECE5021207D21DFB
:1012A300E6021207D23CE7021207D2F0EF0212075E
:1012B300D25DF0021207D279F0021207D2BBF0021C
:1012C3001207D2E4F0021207D27CF1021207D29580
:1012D300F1021207D20ABC021207D2A7BC021207FC
:1012E300D270BE021207D286BF021207D29AC00280
:1012F3001207D21FC1021207D237C1021207D2C28C
:10130300C2021207D2858E021207D2D08E021207B2
:10131300D2768F021207D2FC8F021207D24D9002AF
:101323001207D26190021207D24892021207D2C565
:1013330092021207D2EF92021207D27A9402120794
:10134300D29794021207D2D894021207D20D9502B3
:101353001207D26695021207D28195021207D2F6BE
:1013630095021207D28897021207D2B0970212078A
:10137300D2D997021207D23998021207D25698028D
:101383001207D25998021207D25C98021207D2C7E9
:1013930098021207D2F698021207D209990212078D
:1013A300D26F99021207D2AA99021207D2A0FE02A3
:1013B3001207D2ACFE021207D2E6FE021207D237A0
:1013C300B4021207D286B4021207D228B602120759
:1013D300D2D4B7021207D21CB8021207D253B902F1
:1013E3001207D2E0BA021207D202BB021207D2548A
:1013F300BB021207D2D6BB021207D239F001120781
:10140300D264F0011207D251F1011207D2A5F10102
:101413001207D201F2011207D24DF2011207D2C014
:10142300F2011207D244F3011207D2BAF3011207F1
:10143300D2FCF3011207D226F8011207D2C7F90131
:101443001207D2A7FB011207D2D3FB011207D2E680
:10145300FC011207D279FE011207D20080021207A3
:10146300D2B880021207D24181021207D20282024D
:101473001207D2E682021207D24383021207D25125
:1014830084021207D20285021207D2528502120782
:10149300D21187021207D2C187021207D22888020B
:1014A3001207D2728A021207D2CD8B021207D267B9
:1014B3008C021207D22F8D021207D2268103120744
:1014C300D22F81031207D227EC021207D291EC022A
:1014D3001207D24AED021207D2B0ED021207D276FA
:1014E300DC021207D2CFDC021207D25EDE02120741
:1014F300D217FE021207D261FE021207D264F30270
:101503001207D272F3021207D23481031207D27E7A
:10151300FD021207D28EFD021207D2ACFD021207A2
:10152300D20DFE021207D260F9021207D287F90226
:101533001207D20CFA021207D265FA021207D2DDA1
:101543009D031207D27EFA021207D2A0FA021207F3
:10155300D20AFB021207D215FB021207D252FB0278
:101563001207D241C8021207D24FC8021207D29003
:10157300C8021207D2AAC8021207D2FBC802120776
:10158300D2FCC9021207D221CA021207D23ECA02F2
:101593001207D25BCA021207D280CA021207D2B95B
:1015A300CA021207D2F7CA021207D26ECB0212077F
:1015B300D20ACC021207D2BFCC021207D2CDCC0280
:1015C3001207D247CD021207D203CE021207D28EE0
:1015D300D0021207D2A47E001207D2DD7E001207CA
:1015E300D2FA7E001207D2587F001207D2BD7F00C5
:1015F3001207D2F3D0021207D260D1021207D21A15
:10160300D2021207D28DD2021207D200D4021207DD
:10161300D264D4021207D2B0D4021207D2B9D402D0
:101623001207D2C8D4021207D2E0D4021207D2EDB5
:10163300C2021207D240C3021207D2B4C502120774
:10164300D2E6C5021207D208C6021207D221C60289
:101653001207D23AC6021207D26CC7021207D2028D
:10166300C8021207D221EE021207D253EE0212076A
:10167300D25FEE021207D292EE021207D2BBEE0243
:101683001207D2E9EE021207D266EF021207D295D1
:10169300EF021207D253E7021207D279E7021207C9
:1016A300D2B6E7021207D2C8E7021207D2E4E70272
:1016B3001207D252E8021207D25BE8021207D2BA2B
:1016C300E8021207D2DEE8021207D29DE9021207EE
:1016D300D2AAE9021207D2BBE9021207D21DFF0206
:1016E3001207D26AFF021207D269D8021207D291F7
:1016F300D9021207D29ED9021207D2BDD90212070C
:10170300D2D3D9021207D2E7D9021207D261DA0281
:101713001207D2DFDA021207D258DB021207D2A075
:10172300DB021207D2B0DB021207D212FF0112074B
:10173300D236FF011207D25EFF011207D286FF01E4
:101743001207D2E9E9021207D202EA021207D20E05
:10175300EA021207D222EA021207D240EA02120771
:10176300D24AEA021207D254EA021207D267EA0205
:101773001207D29BEA021207D2D4EA021207D20559
:10178300EB021207D253EB021207D2A0EB021207AD
:10179300D2BBEB021207D2C5EB021207D2D6EB0281
:1017A3001207D21CEC021207D20080031207D2E404
:1017B300AB021207D210AC021207D22CAC021207F2
:1017C300D23FAC021207D255AC021207D2C5AC020B
:1017D3001207D2F8AC021207D252B0021207D28813
:1017E300B1021207D2BBB1021207D220B202120712
:1017F300D20FB3021207D237B3021207D24CB3028D
:101803001207D25CB3021207D2A0B3021207D2F5B9
:10181300B3021207D20BB4021207D22DF802120739
:10182300D248F8021207D271F8021207D28BF802DB
:101833001207D2B0F8021207D2CFF8021207D2E78A
:10184300F8021207D215F9021207D22FF902120772
:10185300D24880031207D2E9D4021207D2F0D4028D
:101863001207D2FCD5021207D22CD6021207D2528B
:10187300D6021207D285D6021207D297D6021207D2
:10188300D2D1D6021207D237D7021207D270D702AB
:101893001207D2BCD7021207D2E9D7021207D20924
:1018A300D8021207D2A8F6021207D2C0F602120714
:1018B300D2A0F7021207D287FC021207D2DEFC0283
:1018C3001207D21BFD021207D25CFD021207D2E5FA
:1018D300E1021207D201E2021207D24CE20212071E
:1018E300D268E2021207D299E2021207D2C0E202E0
:1018F3001207D2A3E3021207D2ADE3021207D2BA50
:10190300E3021207D271E4021207D285E40212073E
:10191300D28EE4021207D2FFDE021207D2E0E10206
:101923001207D2BE80031207D28880031207D2D4D3
:10193300FF021207D2EB80031207D2F3A5011207AD
:10194300D242A4011207D2D3A3011207D277A30173
:101953001207D21AA3011207D2F0A2011207D2E88A
:10196300A0011207D2B4A0011207D272A00112077C
:10197300D247A0011207D2899F011207D23C9F01CF
:101983001207D2B29D011207D2AF9D011207D2B541
:101993009C011207D2819C011207D2BC9B01120742
:1019A300D2EF99011207D2A299011207D2739901BA
:1019B3001207D27099011207D264B0011207D21E26
:1019C300B0011207D26DAF011207D260AF01120747
:1019D300D23EAC011207D26399011207D2269901B4
:1019E3001207D21899011207D2DBA9011207D2C438
:1019F30097011207D24897011207D21597011207D0
:101A0300D2B996011207D2F9E4011207D274A801E0
:101A13001207D28C96011207D29393011207D29523
:101A230092011207D21C92011207D2E79101120709
:101A3300D2B091011207D2A491011207D2049101ED
:101A43001207D24090011207D2068E011207D22B41
:101A53008B011207D2EC8A011207D28B890112077C
:101A6300D23789011207D27E88011207D2E4870197
:101A73001207D28387011207D2BD87011207D284CE
:101A8300AB0200000080FBE4730001363601010065
:101A93000102010001030100010401060605020021
:101AA30000070100340801000F090401010D0100C2
:101AB300FF0E08000017020000190100FF1A0100C1
:101AC300011B0100051C0100081D0200001F01008D
:101AD3000120010001210200002301000F24020064
:101AE300002601000127010308280200FF2A010044
:101AF300072B0102402C0100002D0100012E0100E3
:101B0300012F0100FF30010B1C310800003A0100D6
:101B130008010171010101010111010101310101FB
:101B23000101018001100161013B00140063017395
:101B3300017201620143010001130106013D0135F8
:101B4300000401120100010001000100010401046D
:101B530001330133013C014401320136000001002D
:101B63000165010001350081010001050182018346
:101B730001000103027102300160021102700201CF
:101B830002020202028002100261023A0041006373
:101B9300027302720262024302000213023800005F
:101BA3000200020402120200020002000200020408
:101BB300020402370037003C0244020002390000ED
:101BC3000200026502000235028102000205028260
:101BD30002830200020300710030016000110070F3
:101BE3000031022003500480001000610000001443
:101BF30000630073007200620043000000130006DC
:101C030000000000000400120000000000000000BB
:101C13000004000400370037003C024400000000C9
:101C23000000000000650000003500810000000591
:101C3300000000830000000103710301030103019D
:101C43000301030103220302030103100300030042
:101C53000300030003000300030003420300032403
:101C630003060300030003040312032503230325D0
:101C730003230304030403000300030003440300DA
:101C830003000323030003650321003503810300DD
:101C930003050300030003000336000100060000F0
:101CA300000F00000000000000000000000000031F
:101CB300FFFF00000403FFFF0000FFFF0FF401001C
:101CC30005C4040320000100000B00000000000015
:101CD30000000301030003000400080010001F00BC
:101CE3003E007B00F600EC01D703AF075D0FB91E82
:101CF300713D00000100791402001314030019144C
:101D030004001F140500251406003114FFFF000012
:101D1300390F690F3F0F450F630F570F510F6F0FA8
:101D2300750F7B0F870F4B0F330F2D0FD5C5C5B520
:101D3300A5A5958585757565655555454535352540
:101D43002515050AB70C02810C05930C07870C0CAB
:101D53006F0C0D7B0CFF00009C36063A703DD9409A
:101D63004344AD47174B814EEA5100160F00000B59
:101D7300150B020002220F320000065677777777A1
:101D83007777777777777777777777000102030429
:101D930005060708090A0B0C0D0E0F1D102F103531
:101DA30010030F3B10FD0E090F9510B310B9109BD4
:101DB30010A710A11000034948424D18172505022A
:101DC30000011916181616152303003030171819B9
:101DD30021301B1D1F300C0E020B040B0A070800D9
:101DE3000F303016181920231A1C1E3000383C3EC1
:101DF300363B3B352B432C5D0F810FAD108D0F937D
:101E03000F89104110471053104D100005150D098F
:101E130010080400000000000000BE040A0E0004C5
:101E23000015000405080F040CC082C083E9900468
:101E3300BBF0E4900470F01218A59004CEE4F0A374
:101E4300F09004BCF0A3F0120E191218AB900440EA
:101E5300E4F0A3F09004DEE07002A3E060099004D4
:101E6300DE1243D5121A8A901E29E493FA790212DC
:101E7300190502404E74F2120356EAFEEBFF74801A
:101E83005FF9E47001E9706CEEA2E04003021F14F5
:101E9300900475E0640F700B7900120C57E960032E
:101EA30012203A74016EFAEFFB02201F0CEC75F05E
:101EB30003A4A9F02446F582E9341DF583E4936471
:101EC300FF602AE493FA8508828B83E06A70DDAAB7
:101ED30008EC75F003A42447F582E9341DF583E487
:101EE30093C0E0740193F583D082121A8AAA08ABD7
:101EF3000912118B9004BBE0F91211978A088B0920
:101F0300EA7001EB60047C0080A3EEFA74806F80BA
:101F13009754207003021FEB750A007C027D007A40
:101F23002012202F7C0079047A007B00120CED8AAA
:101F3300088B0980187401850882850983A3A3A3EC
:101F4300A3A3A3A3A3A3F0850C08850D09E508703B
:101F530002E509606E7C007904AA08AB09120CED56
:101F63008A0C8B0D750A01E508240412548524FF9D
:101F7300F0A3E034FF1232967002A3E070C9850823
:101F830082850983A3A3A3A3A3A3A3A3A3A3E06419
:101F93000170A2850882850983A3A3A3A3A3A3E059
:101FA300540470917406850882850983A3A3A3A3AF
:101FB300A3A3A3A3A3F07AB785088285098312217B
:101FC300198084120CBD7C0079017A007B00120C0D
:101FD300EDEA7001EB7009E50A70057A20124350AF
:101FE30074206EFAEF021EAB74025FF9E47001E92C
:101FF300600A120DE3EEFA7402021F1174045FF912
:10200300E47001E960121244FD1241CF79011227F5
:1020130093EEFA74046F80CD7A007B00800312087C
:102023001D7F06020563EAFCEBFD7A017B00900449
:10203300BBE0F912128D22901498124778120C69A2
:1020430022C082C08374EA1208AF8510828511838F
:10205300AA82AB83794B1218DB7408120A6D7402DF
:10206300F07409120A6DAA82AB8379501218DB74DB
:1020730013120A6D1249591218F9741602404B745F
:10208300F4120356EAFEEBFF7508018E828F83A3D9
:10209300A3A3A3A3A3E05440600D8E828F831238C1
:1020A30042FAA3E0FB8003120D4D74FE6A700374C1
:1020B300FF6B60308E828F831243D51243A2120DC1
:1020C300A7E98E828F836006122107E4800512211F
:1020D300077401122F03FAA3E0FB1218FFE9F509B5
:1020E300700580127509CDAA098E828F831221197A
:1020F300E96003750800A908EEFAEFFB120CC9A901
:1021030009022D57E0240DF8A3E012211122340017
:10211300F98882898322E0240C124788F9120C6320
:102123002274F6120356E9FEEAFF7A0F7B001211BE
:1021330085EA7001EB6019740C8A828B83F0EEA33D
:10214300A3F0EF8A828B83A3F012443D79008002CF
:1021530079100243ADC082C083900475E0640F70B0
:1021630016EA7001EB6010900470E064086005E00B
:102173006404700312202902404E74F4120356744F
:10218300FD1208AFEAFEEBFF8E828F83A3A3E0F973
:10219300120CF38A088B09EA7001EB70030222C464
:1021A3008E828F83A3E064F160288E828F83A3E005
:1021B30064CD601E8E828F83A3E0641A60148E82C6
:1021C3008F83A3E064E9600A8E828F83A3E064E1D6
:1021D300701E7900120CC9E960168508828509838F
:1021E300A3A3A3A3A3A3E04420F0A3E0F0022293BC
:1021F3008E828F83A3E0C0E07402120A6DD0E012D6
:102203003F4D124BF8122C2D125169851082851106
:1022130083AA82AB837005120BD98003120D8F8EB4
:10222300828F83A3E064F160678E828F83A3E0646F
:10223300CD605D8E828F83A3E0641A60538E828F9C
:1022430083A3E064E160498E828F83A3E064F0603E
:102253003F7402120A6DE064B76035850882850910
:10226300831222D0750A01780A1207F37403120A43
:102273006DE0F50A780A1207F3EE240C12267512A4
:102283003671A3A3A3A3A3123669122C6912081DE6
:10229300850882850983A3A3A3A3A3A3A3A3A3E080
:1022A300640270127406850882850983A3A3A3A31D
:1022B300A3A3A3A3A3F08E828F83A3A3E0F9120C9D
:1022C300CF120CBD90149C12203D022D52E0F8A3B6
:1022D300E0F9E8FAE9FB2274F4120356EAFEEBFF95
:1022E3007508008E828F83A3A3A3A3A3E060417527
:1022F30008088E828F83A3A3A3A3A3A3A3A3A312DC
:1023030038327001EB601075082C8E828F83A3A383
:10231300A3A3A3E0D2E0F08E828F83A3A3A3A3A3FE
:10232300E05403640160030223B34308110223B39F
:10233300EE24181251666030EE241A125166700FA3
:10234300124E387003A3E06970667508228061EE4F
:10235300241B1223CB241A124346EE2419F582EFD1
:102363001236BD120C4580481223B870037508015C
:10237300124E387003A3E0697006E508D2E1F50850
:10238300E5088E828F83A3A36011E07006E508D26F
:10239300E5801BE508D2E6F5088003E060121238F9
:1023A3003CF9120D95E964016006E508C2E0F50801
:1023B300A908022D578E828F83A3A3A3A3A3A3A34C
:1023C300A3A312463F640222F582EF122C7E12234E
:1023D300D522124C18EE2274F012035674DB120845
:1023E300AFEAFEEBFF8E828F83A3A3A3A3E060106B
:1023F30090149AE07002A3E0600690149A12203DB4
:102403007406120A6DAC82AD838E828F8312269F6F
:10241300124C0AEE241B124E747413120A6D1241ED
:10242300CF7406120A6DAA82AB83120C75E985106C
:1024330082851183F0740C120A6DE06022741D1200
:102443000A6DE0FD7407120A6DE0FC8E828F831221
:1024530047727901120A89E9600302266D8014909C
:102463000458E0600E851082851183E0A2E14003E9
:1024730002266D851082851183E0A2E6502E742317
:10248300120A6D1238426403700E7423120A6D121D
:1024930046F2A3E0640D60147406120A6DAA82ABBF
:1024A30083120DB9E96401700302266DEE242C1228
:1024B300267512295C7003A3E069701F7508007804
:1024C300081207F378081207F3EE242EF582EF12B1
:1024D30036BD122690122C6912081D7409120A6D5A
:1024E300E0FA90045EE06A600302266D740C120A3F
:1024F3006DE070030225B4122690124774120E4346
:102503007401120A6D1243A27401120A6DE0700283
:10251300A3E0700302266D7407120A6DE0F88E8241
:102523008F83A3A3E028F8A3E03400F9740D28F502
:1025330082E439F583E0FA7401120A6D122684E00D
:102543006A601D7401120A6D12267CEAF090876D91
:102553007808120A2E7401120A6D12268A120A1FB3
:1025630079047407120A6D124C002AFCA3E03400AC
:102573008C82F583A3AA82AB831211738A088B0919
:102583008C0A8D0B7401120A6D122684A3780C1227
:102593000A2E780C79081209E0500302266D908701
:1025A3007978081209037401120A6D12268A120A35
:1025B3001F900470E064046008E06409600302266D
:1025C3006D851082851183E0A2E55055EE242E120D
:1025D3005166C0E07403120A6DD0E0F0EE242F12AE
:1025E3005166C0E07404120A6DD0E0F0EE2430129C
:1025F3005166C0E07405120A6DD0E0F0EE24241297
:10260300267512064F7407120A6DAC82AD83740AE5
:10261300120A6DAA82AB83120BDF740412081D80A9
:1026230049A2E650457423120A6D12477E7018744E
:102633001D120A6DE0640270317406120A6DAA82DB
:10264300AB83120D8380237423120A6D1246F2E0CA
:1026530064077016741D120A6DE06404700C74062E
:10266300120A6DAA82AB83120D7D7425024AEAEE2B
:10267300240BF582EF122C7E22A31246F3A3A3A30D
:1026830022124629A3A322123A1E780822EE242AF4
:10269300122C7B1223D52412122C7B22A3A3A3A3D7
:1026A300E0F98E828F83A3A32274F712035674F783
:1026B3001208AFEAFEEBFF900470E06403600DE0E4
:1026C30064016008E06409600302278E8E828F83B1
:1026D300A3E0600302276A7C007D007A027B00127C
:1026E30018B1EE2402FAEF124446124E7A900461B6
:1026F3001241CF79531218E1790012279390047095
:10270300E06409600990046E124774120E3D74016F
:102713001243CC7404900470F07401120A6DAA82FF
:10272300AB83794A1218DB7401120A6DAC82AD8354
:102733007A667B041218C9900461124C147A037BE5
:10274300001218B1900464124C147A047B0012181E
:10275300B190045BE0A2E35004D2F08002C2F01215
:1027630043B212203A80218E828F83A3AE82AF833D
:10277300FC7D007A037B101218B18E828F83E0F9FF
:10278300122793E4900470F0120C9F7409023661CF
:1027930090046E124778120BEB22C082C083900420
:1027A30040E07002A3E07041900470E01206D8008C
:1027B3000301BF2705CE2706DD27EC27900448E059
:1027C3007002A3E0607B9004488070900444E07042
:1027D30002A3E0606C9004448061900446E07002C0
:1027E300A3E0605D9004468052900440E07002A331
:1027F300E06005122C44702379009004BC80090921
:10280300EA124AF2EB1226781235587001EB70EF98
:102813009004BC124774120BE580269004411226E3
:102823007DA3A3A3E064027005120DD78013900467
:10283300E4E07002A3E060099004E41243D5121AA5
:102843008A02404E74F412035674FB1208AF8A08CE
:102853008B091229457001EF700302294074028E1F
:10286300828F8312495A79501218DB8508828509B1
:1028730083A3E0600302292E90046EE064FF7004DA
:10288300A3E064FF603590046EE064FE7004A3E08F
:1028930064FF602785108285118312295C7003A36E
:1028A300E069601774EA850882850983A3122C8383
:1028B3007A6E7B0479501218E1807085108285113D
:1028C30083124EEB1241CF7A617B0479531218DBEA
:1028D3009004611241C67A647B04794B1218DB7A47
:1028E300637B0479E11218DB900475E0C3940F5005
:1028F30022900463E0C0E07402120A6DD0E0F07429
:1029030004120A6D7401F07402120A6DAA82AB8379
:102913001218F3750A00780A1207F3780A1207F3FC
:102923009014BBE0F9122C6012081D8508828509FA
:1029330083122956F0740390047012443474050210
:102943002D547A0F7B001211858A0A8B0BAE0AAFC6
:102953000BEE22A3124181A322124EEFE0682274F0
:10296300F212035674ED1208AFEAFEEBFF8E828F6C
:1029730083A312368C851082851183AC82AD838E3E
:10298300828F83A3A3A3A312269F12476D120CABBE
:10299300851082851183E0706A8E828F83A3A3A33F
:1029A300A3A3A3A3A3E0C3940B405885088285097E
:1029B30083A3A3A3A3A3A3A3A3E0640270459004EA
:1029C30070E064026042E06406603D900440E070A1
:1029D30002A3E06005122C44605E900470E064087A
:1029E3006005E06404701C7402120A6DE0F9740758
:1029F300120A6DAC82AD8385088285098312476B09
:102A0300120CB17413022021900440E07002A3E081
:102A13007026750A00780A1207F3780A1207F31270
:102A23002C24122678122C4DFCA3E0FD8508828508
:102A33000983122C6912081D9004BC123A319004C8
:102A4300BCE0F50AA3E0F50B80378E828F83E0F8B4
:102A5300A3122C4D687003A3E06970198E828F83D3
:102A6300A3A3E0FAE508240DF582E5091251696A8A
:102A73007003022AF88E0A8F0BEE124AF2EF123A13
:102A83002EEE7001EF70C37A187B001211F18A0CDD
:102A93008B0DAE0CAF0DEE7001EF7003022A0690A2
:102AA30004BCE07002A3E070059004BC800AE50A50
:102AB300124AF2E50B122678124D6E8E828F831224
:102AC300445FEE240C12267574FFF0E48E828F832C
:102AD300A3A3A3A3A31234B9A3A3A3122C72E4F058
:102AE300A3F0E508240B125485122C1A123296C453
:102AF300122C1AA3F07401120A6D12442EF0740200
:102B0300120A6D122C3CA3F0E508240DF582E509A9
:102B1300122678122957A3124529A3A31254A012EF
:102B230041CF7402120A6DE0640160117407120A46
:102B33006DAC82AD83EE240D122C3380117C087DA5
:102B43000079FFEE240DFAEF3400FB12116D7412BD
:102B5300120A6DE0C0E0EE2415122675D0E0F09065
:102B630014BBE0C0E0122C24124349D0E0C39A40C6
:102B730003022A06122C2D122678A3E05480F9E4CE
:102B83007001E97009900E5AE07003022A06740678
:102B9300120A6D122C3C700EE070627404120A6DFE
:102BA300E07006022A06E060147405120A6DE0C0A4
:102BB300E0EE240C124346D0E0C39A502B850882E2
:102BC3008509831254AE1241CD122C24125169C0CF
:102BD300E0122672D0E0F07405120A6DE0C0E0EE58
:102BE300240C122675D0E0F07406120A6DE0600D15
:102BF30074018E828F83A3A3A3A3A3A3F0740412EF
:102C03000A6DE07003022A0674018E828F83A3A3E8
:102C1300A3A3A3F0022A06540F8E828F83A3A3A338
:102C230022E5082410F582E50922E508240B80F546
:102C3300FAEF3400FB1218C922122C4022E00234AE
:102C430008900440122FA6640122E0F985088285CA
:102C53000983A3A3A3A3A3A3A3A3A3E02290046E26
:102C6300124C18900464124778120D5F740222A369
:102C7300F0EE2416122C7B22F582EF3400F583222A
:102C8300F07A617B047953122C8E221218E17A6454
:102C93007B04794B1218E12274F212035674F81272
:102CA30008AF8A0A8B0B8C0C8D0D890885108285E1
:102CB3001183AC82AD837583877582017408120713
:102CC3004BF509AC0AAD0B851082851183AA82AB43
:102CD3008312495470037509019004BC80158E82D8
:102CE3008F83E0650C7004A3E0650D6023EE24166A
:102CF300122675123A31EE7001EF601FE50960DEAE
:102D0300AC0AAD0BEE240DFAEF340012495360DD2B
:102D13008E828F83A3A3E0650870D2EEFAEFFB7473
:102D23000802202174F71203569004BCE0FAA3E0D2
:102D3300800CEA2416123A2B1211F7EEFAEFFBEA93
:102D43007001EB70ED9004BCE4F0A3F00236647400
:102D53000312081D7F0402056374F21203568A0CE2
:102D63008B0DECFEEDFF890B8A828B83124AF78A67
:102D7300828B83122E1FEEF8EFF9A30EAF838A82A4
:102D83008B83A3A3E0C454F0FA88828983E04A12B8
:102D93002E2A124181122E25E0333354FCFA8E82FF
:102DA3008F83E04A122E25A3E033333354F8FA8E8F
:102DB300828F83E04AF008EFF9A30EAF83850C827C
:102DC3008B83A3A3A3A3A3A3E0A2E0E492E0131342
:102DD3005480FA88828983E04AF0E50C2407F508D9
:102DE300EB123EE91207EB7C08123C6012081D123D
:102DF3004BD7E50C240FF508E50D3400F5097808E9
:102E03001207EB7C03123C6012081DE50BC3940F01
:102E13004007122EEC124177F0022024A3124181C5
:102E2300F022122E2AA322F0850C828B83A3A3A364
:102E33002274F2120356EAFEEBFF890B8C0C8D0D04
:102E43008E828F83E08C828D831234BEAE82AF83F9
:102E5300E0123FFE122F02C4123FFE122EF5E05481
:102E6300038C828D83122F00A2E2E492E08C828D88
:102E730083122EFF131313541F123FFE122EFEA2B2
:102E8300E7E492E08C828D83A3A3A3A3122EF58E95
:102E9300088F09750A0078081207EB7C087D00E5A6
:102EA3000C2407124BAD12081D124BD78E088F0945
:102EB30078081207EB7C037D00E50C240F124BAD61
:102EC30012081DE50BC3940F40148E828F83A3A3B6
:102ED300A3E0C0E0122EEC122678D0E08007122E79
:102EE300EC122678E4F0022024E50C2412F582E5A6
:102EF3000D22A3A31234BE0EAF8322A3A3A3A3A3C5
:102F0300F08E828F83E02274F412035674F9120850
:102F1300AFEAFEEBFF900440E07002A3E060101202
:102F23002F9F64027009EEFAEFFB120DD1806890B7
:102F3300046EE06E7003A3E06F705C740169600956
:102F43007A827B04124954704E7A007B029004BB50
:102F5300E0F9121299EA7001EB703C900471780861
:102F6300120A2E8510828511837808120A1F900495
:102F730077E0C0E07404120A6DD0E0F07405120A21
:102F83006D7401F07406120A6D740212495A120B21
:102F9300B5E96092120BBB7407022D5490044012E2
:102FA3002FA622123A22A3A3E02274F6120356EAB2
:102FB300FEEBFF8E828F83A3858208858309E0F968
:102FC300120C03850882850983E064EB600A8E8214
:102FD3008F83A3E064E17007E48E828F83A3F012F2
:102FE300203A75080178081207F38E828F83A3E0D5
:102FF300F50878081207F37900122C6012081D12E5
:103003000CBD0243AD74F61203569004CDE0701F5D
:103013007C0079017A007B00120CEDEA7001EB6011
:103023000E8A828B83E07002A3E06003120C5D02C0
:1030330043ADC082C0831234AA401079FF120CE75B
:10304300E9FA901E2BE493C39A5004790180027924
:103053000002404E74F11203568A0A8B0B890E75D7
:1030630009008A828B83A3A3A3A3A3A3A3A3E0F949
:10307300120CF38A0C8B0DAE0CAF0D750801EE70BC
:1030830001EF600302312D850A82850B83A3A3A37D
:10309300A3A3A3124C14850A82850B83A3A3A3A322
:1030A300A3A3A3A3E0F9850A82850B8312477412B5
:1030B3000CDB8A0C8B0DAE0CAF0DEE7001EF7003C1
:1030C30002326C8E828F83A3A3A3A3E4F0A3F0E563
:1030D3000A240BFAE50B124446E0C0E0122672D034
:1030E300E0F0120DADEE240C12439B750901EE24A2
:1030F30006F8EF125488547FF0A3E054FC12329682
:10310300540460030231B39014A0E0F50A750B0078
:103113007407780A1209888E828F83A3A3A3A3A3BB
:10312300A3E0450AF0A3E0450BF08E828F83A3A3AF
:10313300A3A3A3A3E05480F50AA3E05403F50B74FF
:1031430007780A120A10E50E607974028E828F8363
:10315300A3A3A3A3122EFE240D124784A2E2500BB5
:1031630090045CE0F81226A21241CDE50A70030236
:10317300323AEE2406F8EF3400F9E8FAE9FB8A82E2
:103183008B83E0547FFCA3E054FCFD74FF250AF518
:103193000A74FF3400F50B7407780A120988E50AEC
:1031A3004CF8E50B4DF98A828B831241CF02323AF8
:1031B3008E828F83A3A3A3A3A3A3E04480F0A3E001
:1031C30002312CE50A7005750800806B8E828F83AF
:1031D300A3A3A3A3A3A3E05420601712117F8A0A19
:1031E300747F550AF8745F288E828F83A3A3A3A3E9
:1031F30080278E828F83A3A3A3A3A3A3E05410608D
:103203000E12117F8A0A740F550AF8740180D88E42
:10321300828F83A3A3A3A37401F0A3E4F074048EA9
:10322300828F83A3A3A3A3A3A3A3A3A31234C570D1
:1032330001EB700312327674016509702F8E828F51
:1032430083A3A3A3A31249C9F9EEFAEFFB120CE17E
:10325300E96019EE240C1251667002A3E0600312B8
:103263003283EEFAEFFB1211F7750800A9087F0706
:103273000205637A207B009004BBE0F91211B522AA
:10328300EE240C122C7B12328D22E0FAA3E0FB1207
:1032930011F722F088828983E02274F412035675B1
:1032A3000800120CF38A0A8B0BAE0AAF0BEE700107
:1032B300EF70030233428E828F83A3A3A3A3A3A33E
:1032C300A3A3A3E064067077120D058E828F83A3F8
:1032D300A3A3A3A3A3A3E05408F9E47001E9605CEA
:1032E3008E828F831236807A007B00120CD5EA70AF
:1032F30001EB704812334512190B7C007D007A00F4
:103303007B0080228E828F8312367A7004A3E0645E
:10331300FF6029123345121635E9641A601E7C00DA
:103323007D00EEFAEFFB120CD58A088B09AE08AFCD
:1033330009EE7001EF70CD790012191175080102C1
:1033430023B390046E1249CF1247782274F7120305
:10335300568A828B83E5827002E58370099004CEDE
:1033630080068A828B83A3A31235587001EB602CED
:103373008A828B83A3A3A3A3A3A3A3E05408F9E4A2
:103383007001E960DDEC7001ED60158A828B8312B8
:1033930038426C7003A3E06D70C880047A007B0030
:1033A30002366474F21203568A088B09890AECFE0A
:1033B300EDFF7A0E7B001211F1EA7001EB603EE43F
:1033C3008A828B83A3A3A3A3A3A3A3A3123403E59A
:1033D3000A123F33A3A3124D6A8A828B83A3A3A34A
:1033E300A3E4F0123403123F31124BF8EA240CF534
:1033F30082EB12382C123F32A3A3F0A3F002202455
:1034030012526880058E828F83A3A3A3A3A3A32252
:1034130074F5120356EAFEEBFF890A8C088D09EE58
:103423007001EF60597401650A70147901120CE799
:10343300E9FA901E28E493C39A500F7911806374BC
:1034430004650A70331234AA40F18E828F83A3A3DA
:10345300A3A3A3A3A3A3A3E50A1234B9124BF68E25
:10346300828F83A3A3E4F0A3F09004CEE07002A3C1
:10347300E09004CE601B800A7402650A60CC79C1B7
:1034830080201249DC7002A3E088828983A3A370A1
:10349300F1EEF0A3EF1234C57001EB700312327634
:1034A30079007F030205637904120CE7E9FA901EA1
:1034B30027E493C39A221234BEA322F08E828F8311
:1034C300A322F07A207B009004BBE0F9121299EA60
:1034D30022C082C083E9FC79009004CE801D8A82D9
:1034E3008B83A3A3A3A3A3A3A3A3A3E06C600574EB
:1034F300FF6C7001098A828B83A3A3123558700174
:10350300EB70DB02404E74F71203568A828B83E51D
:10351300827002E58370099004CE80068A828B83D1
:10352300A3A31235587001EB60248A828B83A3A373
:10353300A3A3A3A3A3A3A3E06970E1EC60148A820D
:103543008B83E0240D124B01A2E240D080047A0069
:103553007B00023664124778EA22C082C08390045B
:10356300CE80068A828B83A3A31235587001EB6049
:10357300128A828B83A3A3A3A3A3A3A3A3E069704B
:10358300E280047A007B0002404E124E7EE82274F1
:10359300F11203568A0A8B0B8C0C8D0D750800757E
:1035A3000900EA7001EB602E9004CE80068E828FB4
:1035B30083A3A3123A31EE7001EF601AAC0CAD0D88
:1035C300EEFAEFFB850A82850B83121A8AE96401FE
:1035D30070DB8E088F09AA08AB0902327174F712E7
:1035E30003569004CE124E7A7C007D00800DE8FCD9
:1035F300E9FD88828983A3A3124E7AE87001E9600A
:1036030030EA687002EB6970E59004CE124774E803
:103613006A7002E96B88828983A3A37008124E7AC9
:103623009004CE8009124E7A8C828D83A3A312411B
:10363300CF02366474F7120356EAFEEBFFEE700115
:10364300EF6016120CFF1236967002A3E0600312AD
:103653003283EEFAEFFB1211F7023664741F12087D
:103663001D7F01020563124C188A828B8322E0F9C5
:103673008A828B8302340E12384664FF2212384644
:10368300FCA3E0FD228E828F83A3A3E0F508A3E0D1
:10369300F509228E828F83E0241C12478812328E12
:1036A3008E828F8312328DEE240C1236B122F58274
:1036B300EF3400F583E022F582EB1236B4F922747D
:1036C300F212035674FC1208AFEAFEEBFF7508FE14
:1036D3007509FF120CC3E960057911023821EE2444
:1036E3001512516660379014B5E0C43354E0C0E05E
:1036F300E0333354FCFAD0E04AC0E0EE241512263E
:1037030075D0E01234B91238327001EB600F7508CE
:10371300FF124515EE2415125166D2E0F08E828F0A
:10372300831246396006EE2412123829EE2413124E
:1037330051667003741EF012516364017016900F8A
:103743002AE0600D900458E0700A8E828F83E07047
:1037530003123826EE2414125166701590044DE0BE
:10376300C0E0EE2414122675D0E0F090044DE0047E
:10377300F08E828F83E064017016EE240B12383FC3
:103783006402700CEE240F1251664440F0A3E0F083
:10379300851082851183AC82AD83EEFAEFFB120DA7
:1037A3001D8A0A8B0B74FE6508700474FF64FF7036
:1037B30003123688EA7001EB60608E828F83E0C06B
:1037C300E07401120A6DD0E0F07402120A6D124D1A
:1037D3006E7401120A6D85820C85830D780C1207B5
:1037E300EFEE240F122675120653EE240E125166C5
:1037F300F50C780C1207F37405120A6DE0F9AC08A6
:10380300AD09120D17740512081DE9FE74106E70D0
:103813000BAA0AAB0B1211F780027E10EEF97404A7
:10382300022021EE2411F582EF122C7EE4F0221205
:10383300477879FF1219BFEA22EE241D122C7B125E
:103843003846221246E8E022C082C08374DE1208A2
:10385300AF8A828B83A3A3A3A3124E7A740E120A98
:103863006DE8F0A3E91238FD740C120A6D1238F6F4
:10387300240DF582EB125169C0E0741A120A6DD05F
:10388300E0F01249D5124E777420120A6D1238F601
:103893002415F582EB125169C0E07408120A6DD049
:1038A300E0F0EA241CF582EB124E777412120A6DD3
:1038B3001241CF74FF851082851183F07401120ABF
:1038C3006D74FFF07402120A6D74FFF090876D122D
:1038D300064F7404120A6DAC82AD837407120A6D2D
:1038E300AA82AB83120BDF740412081D79007422C1
:1038F30002404BE8F0A3E9F0EA22F08A828B83A32B
:10390300A3124E7E2274F012035674EE1208AF74A3
:1039130010120A6D1243A28C088D09890B742212AE
:103923000A6DE0F50C7423120A6D123A31742512F4
:103933000A6DE0F50EA3E0F50F750A107A1E7B0001
:103943001211F17402120A6D1243A27402120A6D6B
:10395300E07002A3E07003023A118510828511839F
:10396300AA82AB837950124258120A6D123A18A3F5
:103973001243A27402120A6DE0240B12210A74028C
:10398300F0120A6D123A187402F0120A6D1243D53E
:10399300124BF87402120A6DE0241B12210AE50B84
:1039A300F07402120A6DE0240C12210AE50CF07483
:1039B30010120A6D124261120A6DE0241C12210AD0
:1039C3001243A27408120A6D124D6E740A120A6D24
:1039D300E50CF0850E82850F83C082C083740D12BF
:1039E3000A6DAC82AD83D083D082740312074BF986
:1039F3007402120A6DAA82AB83120CC9E9640170C6
:103A030005750A0080087402120A6D123289A90A28
:103A13007412024AEA123A1E02340E123A22221297
:103A230046EC02340EEA240BF582EB122C7EE0FE08
:103A3300A3E0FF2274F0120356EAFEEBFF8C088D1D
:103A43000974088E828F83122C72E0600874108EC2
:103A5300828F83A3F0EE241712516660098E828F42
:103A630083A3E02408F0EE241512516660088E82C9
:103A73008F83A3E004F08E828F83A3A3A3A3A3A3C6
:103A8300E060198E828F83A3A3A3A3A3A3A3E0C3A0
:103A9300332402FA8E828F83A3E02AF012516360EB
:103AA30005750B0E8003750B008E828F83A3E0C018
:103AB300E0EE240D122675D0E0FAE02A250B8C8265
:103AC3008D83F012516360051241FC2AF085088250
:103AD300850983E0C394754003023C53E0FA7B00FD
:103AE3001211F18A0E8B0FEA7001EB7003023C593D
:103AF300EEFAEFFB120D23EA850E82850F83124344
:103B0300A3EE2402F8123C6C123C8BF0EE24040862
:103B130008123C6CA3A3123C8BA3A3F0EE24131254
:103B23003C77F0EE2414123C77A3F0750C08EE24D6
:103B3300161251666013EE2418124C11E50E240878
:103B4300FAE50F122C35750C10EE2417125166602E
:103B530019EE241A124C11850C08E50E2508FAE516
:103B63000F122C357408250CF50C8E828F83A3A3BA
:103B7300A3A3A3A3E060728E828F83A3A3A3A3A3B3
:103B8300A3A3E0C0E0850C08E50E2508F582E50F48
:103B9300122678D0E0123C81E0C0E0850C08E50EE7
:103BA3002508F582E50F122678D0E0123C81A31296
:103BB3004BB61207EB8E828F83A3A3A3A3A3A3A366
:103BC300E0C333FCE433FD850C08E50E2508FAE574
:103BD3000F124BB012081D8E828F83A3A3A3A3A33E
:103BE300A3A3E0C333250CF50CEE24151251666034
:103BF30010C0E0E50E250CF582E50F122678D0E023
:103C0300F0122672124BB61207EBEE240D12516618
:103C1300FC7D00850B088E828F83A3123F0CE50881
:103C230028FAE439123C6512081D1251636027EE2D
:103C3300240D125166FD8E828F83A3E0FCAA0EAB86
:103C43000F7900120A89E9600DAA0EAB0F1211F762
:103C5300750E00750F00AA0EAB0F024AED7D00EE44
:103C6300FAEFFB121161740322EF12548C850E825A
:103C7300850F8322122C7B123C92A3A3A322F0056F
:103C83000C8E828F83025847123C9D123C9222E095
:103C9300850E82850F83A3A3A322A3A3F088828921
:103CA30083A32274F6120356EA2415F582EB12510C
:103CB3006960047C0180027C008A828B83E0FE9031
:103CC300045E123D4774027808120988E5084EFE27
:103CD300AF09EA2412123D4174067808120988E5F7
:103CE300084EF8E5094FF9ECFDE8FCED49FDEA243F
:103CF30011123D4174097808120988E5094DFDEA5E
:103D03002416123D41740B7808120988E5094DFD0C
:103D1300EA2417123D41740C7808120988E5094D0D
:103D2300FD8A828B83A3A3A3A3A3A3123D47740A93
:103D33007808120988ECFAE5094DFB0243ADF582D8
:103D4300EB122C7EE0F5087509002274F01203567D
:103D530074FE1208AF8A0E8B0FECFEEDFFE98E8224
:103D63008F83123F3312418E850E82850F83A3A367
:103D7300123F071241B8123F55123F071241A712D3
:103D83003F55A3A3E0C0E0EE2411122675D0E01244
:103D93003F5CA3A3A3E0C0E0EE2412122675D0E09B
:103DA30012420E600AE50E2408F8E50F1241D58E83
:103DB300828F83A3A3A3A3A3A3A3A3E060218E82E3
:103DC3008F83A385820C85830D123F0CEE2415127D
:103DD30026751241CF850C82850D83E02408F08E71
:103DE300828F83A3A3A3A3A3E0600F123F188E8245
:103DF3008F83A3A3A3A3A3123F66EE2418125166D5
:103E0300607C123F18C0E0EE2419122675D0E01230
:103E13003F66F8E50E28F582E50F125169C0E0EE22
:103E2300241A122675D0E0123F66123EDFE433FBFC
:103E3300123F377002A3E060458E828F83A3E0F8C0
:103E4300E50E28F508E50F123EE91207EBEE2419FB
:103E5300125166C333FCE433FD7403120A6D124737
:103E630074123C6612081D123EDF850C82850D8399
:103E7300E02A124BBEEE241B1226751241CF8E820E
:103E83008F83A3E0FA8A08E50E2508F8E50F3400CE
:103E9300123EF3122F03C39AC0E0EE2417122675C5
:103EA300D0E0125960E06031EE2417F508EF3400DA
:103EB300F509850882F583E024F2F0EE241DF8EF7E
:103EC300125488240EFAA3E03400FB88828983EA23
:103ED300F0A3EB1241F7C39AF0024AE8EE24191259
:103EE30036B1C333FA223400F509750A0078082283
:103EF300F9EE241D123EFB22F582EF3400F583E830
:103F0300F0A3E922E0FA023C70E0F8E50E28F8E5B8
:103F13000F3400F9228E828F83A385820C85830D53
:103F2300E0F8E50E28F582E50F1236B422A3A3A329
:103F3300F002366C1211F1851082851183EAF0A329
:103F4300EB123F4822123F4DE022F085108285118B
:103F53008322F0A3E9123F5C22F0850E82850F8352
:103F630002340EF0850C82850D83E004F02274F494
:103F73001203568A088B09EA124005F0EA13135418
:103F83003F123FFEA3A3A3F0EAC41313124005A3F9
:103F9300A3F0EB123FEBF08A0A8B0B7409780A1239
:103FA3000A10E50A123FEBA3F08A0A8B0B740A7816
:103FB3000A120A10E50A5401C0E0EC2418F582ED58
:103FC300122678D0E0F08A0A8B0B740B780A120A57
:103FD30010E50A123FF8F0740C7808120A10E5088D
:103FE300123FF8A3F0022D57123FEF2254018C82A7
:103FF3008D8302340D123FEFA3A322540F8C828DC5
:10400300832254038C828D83A3A322C082C083792D
:10401300008A828B83A3A3A3A3A3A3E09004586085
:104023000FE070228A828B83A3A3E07019098016A4
:10403300E060138A828B8312476B900461E06A709D
:1040430003A3E06B70E7800312081DD083D08202C4
:1040530007CF74F31203568A0A8B0B890CECFEED1F
:10406300FF8A828B8312418E850A82850B83A3A3E9
:104073001241851241B81241E61241851241A7123D
:1040830041E6A3A3E0C0E0EE2411122675D0E012AE
:1040930041EDA3A3A3E0C0E0EE2412122675D0E005
:1040A30012420E600AE50A2408F8E50B1241D58E88
:1040B300828F83A3A3A3A3A3A3A3A3E0601B8E82E6
:1040C3008F83A3124195EE24151226751241CF85D5
:1040D3000882850983E02408F08E828F83A3A3A33B
:1040E300A3A3E060238E828F83A38582088583093F
:1040F300E0F8E50A28F582E50B124177A3A3F085E2
:104103000882850983E004F0EEFAEFFB120D35E92E
:10411300705D8E828F83A3A3A3A3A3122956702558
:10412300E0FC8C08E50A2508FAE50B3400FBEE24D5
:104133001D12439BE50CC39CC0E0EE2417122675A9
:10414300D0E0F0802A124195740E28F8E439123E2B
:10415300F31241F7FCE50CC39C24F2C39AFDEE2451
:1041630017122675EDF0AA0AAB0B7901120A897FA3
:1041730005020563122C7E124181A3A3A322E00250
:1041830054A9E0FA850A82850B8322124778120D1F
:104193002F22858208858309E0F8E50A28F8E50BD4
:1041A3003400F922A3A3A3A3A3E0F9EAF8EE240BB6
:1041B300122C7BE822A3A3A3E0F9EA8E828F83A3C8
:1041C300025847124E7E8E828F83A3A3E8F0A3E9A1
:1041D300F0223400F9EE2413123EFB1234BEE02425
:1041E30008F022F0A3E91241ED22F0850A82850B43
:1041F3008302340EF01241FC22900459E0F9120AB2
:104203008FE9FA850882850983E022F074088E829B
:104213008F83A3125964A3E022C082C0837AD37B25
:104223000479E21218DB7AD37B0402404EC082C0C9
:104233008390046112477402404EC082C08374FEAF
:104243001208AF851082851183AA82AB83794B1242
:10425300425802404B1218DB8510828511831247A6
:1042630078740222C082C083794A1218DB02404E5E
:1042730074F61203569004DBE0FE04F0EEF9120C20
:10428300F3EA7001EB70EEEE60EBF90243AD74F00C
:10429300120356EAFEEBFF8C0E8D0F890874101281
:1042A3000A6DE0F50D7411120A6DE0F50C75090045
:1042B300120E438A0A8B0BA80AA90BE87001E97056
:1042C30013E50C705DA908AC0EAD0FEEFAEFFB120F
:1042D3000E61806CE508601FE82402F582E9124351
:1042E30049E5082AFAE4340013EA13F0700974016B
:1042F30088828983A3A3F0E50C6045E50D701088DF
:10430300828983E0600214F0E49004EAF080319043
:1043130004EAE004F0FA9014A1E06A70237509013D
:104323008003E4601BE5096017120D4DEA6E70020D
:10433300EB6F700CEEFAEFFB7901120BFD12434E9B
:10434300024AEDF582EF1236B4FA227A017B00902D
:1043530004BBE0F912129322C082C08374016A7015
:1043630001EB70077A01123278801490149812438B
:10437300A2EA7001EB6005122029800312434E026A
:10438300404EC082C08390149A1243A202404EC092
:1043930082C08390149C80F1F582EF3400F583EAA8
:1043A300F0A3EBF022740D12081D7F02020563A235
:1043B300F0E492E01243C079521218E12285108290
:1043C300851183F0AA82AB83221243C0794212186B
:1043D300E1221246E422AA82AB83120CA57ABE7BA9
:1043E3000479451218E12274F712035674ED12088A
:1043F300AFE9FE9004BA12478F1244217412120AD5
:104403006DEE1244168510828511831243D97413FD
:10441300023661F0901446E0F97CBE7D04229014CC
:1044230046E0F97ABE7B04120CAB22122C40A3A304
:1044330022F012443922EEFAEFFB9004BBE0F912AA
:104443001191223400FB02366CF582EF12454F22A4
:10445300A3E088828983F0A308A98322A3A3A3A34B
:10446300A3A3A3A3A374FEF0A374FFF02274F41216
:1044730003568A088B097A007B041243521244FDC7
:104483001241CF7409900470F0120D418A0A8B0B0C
:10449300AC0AAD0BE5082413F582E5091226781260
:1044A30047741249546401704E1229457001EF603C
:1044B3004674028E828F83F0E508241DF8E5091205
:1044C30021111247748A828B83A3E0FC8A828B8337
:1044D300A3A3E0FBEC8E828F83A3A3F0A3EB1232A2
:1044E30096F812267C124181124507FAA3E0FB7964
:1044F3004A1218E1124439022D57900442124E7E9B
:1045030090149C22A3F0E5082415F582E5091236E0
:10451300B422EE240F1236B14404F0A3E0F02212C9
:10452300452FA3A3A322124522A3A322F085088229
:10453300850983A3A322EE241712454C120D41EEE5
:10454300241A122C7BEA0243A3F582EF3400F5838D
:104553007401F02274F612035674F31208AFEAFEE4
:10456300EBFF7C0D7D007900851082851183AA8283
:10457300AB8312116DEE241DF582EF124622E0F893
:1045830054206008740C120A6D7401F0E8548060C2
:1045930008740B120A6D7401F0E85440600A740A3F
:1045A300120A6D7401F0800A740A120A6DE0640144
:1045B3007005EE24138003EE2415124C11740212BD
:1045C3000A6DAA82AB831218C91226721246D3123D
:1045D30041CF740A120A6DE06401703312462E70E3
:1045E3003B120D4D8A088B09A808A909EE240B126A
:1045F3005166687003A3E0697022120D41EAFCEB77
:10460300FD7402120A6DAA82AB83124954600D85B0
:104613001082851183AA82AB83120BF70243A8127F
:104623002C7E124629221246E8A3228E828F83A370
:10463300A3A3A3A3A3A3A3A312463F22E0FAA3E049
:10464300FB120DA7E92274F612035674F31208AF96
:104653008A088B09ECFEEDFF7C0D7D007900851047
:1046630082851183AA82AB831256D7A3A3A3A3A3E4
:10467300A3A3A3A31246D3E8F0A3E91246D9A3E068
:10468300FAA2E55008740B120A6D7401F0EAA2E76E
:104693005008740A120A6D7401F0EAA2E6EE50049F
:1046A300241380022415124C117402120A6DAA827B
:1046B300AB831218C9850882850983A3A3E0C0E0F0
:1046C300740C120A6DD0E012495A120BF10243A87E
:1046D300124E7E023F4EF0EE241D122C7B1246E456
:1046E300221246E8221246EC22E0F81246F222A3F6
:1046F300E0F58388822274F712035674E11208AF3F
:10470300EAFEEBFF8E828F83122FA2A2E050568E19
:10471300828F831222D28A828B83A3A3A3A3A3A310
:10472300E054FEF0A3E012478F8A828B83E0241BC0
:10473300124784F98A828B83E0241CFAA3E0124493
:1047430046124774120D3BE9701B741D120A6D1259
:10475300477E7011851082851183AC82AD83EEFA9A
:10476300EFFB120D8902365FA3A3A3A3A3A3A3A305
:10477300A312477822E0FAA3E0FB2212384664042E
:104783002212478822F8A3E012549022123F4DAC24
:1047930082AD8322E9FA790074046A600A740A6AB2
:1047A300600574036A7001090207CF74F612035699
:1047B30074208A828B83F07401A3A3F0120BA98A5D
:1047C300088B09AE08AF09EE7001EF600774018E24
:1047D300828F83F09004AEE07003124539EEFAEF56
:1047E300FB0243ADC082C08374019004D0F0E9A200
:1047F300E350037403F0E9A2E15004E0D2E2F002D3
:10480300404E74F612035679007C008A088B0978AF
:104813000812051DF8FF073848364836483648362B
:10482300482F48334838482C480C80097C048005BD
:104833000C80F67C089004D0E05C6003098003ECF4
:104843006001090243AD74F61203568A828B83E03A
:104853007014A3E07002A3E0600C8A828B8312477A
:10486300731219EF80047A007B000243AD74F512D2
:10487300035674F31208AFEAFEEBFF8C088D09753B
:104883000A12EE7001EF7005790002494590046148
:10489300E06E7003A3E06F7018120D41EAFCEBFDAC
:1048A300AA08AB091249547005750A018003750AF9
:1048B30000E4851082851183F07401120A6DEEF015
:1048C300A3EF12495A120AD7E9602B7403120A6D37
:1048D300AA82AB83120ABFE96401701A750A0174D4
:1048E30003120A6DAC82AD83AA08AB091249546066
:1048F30021750A00801C7412650A70169004ADE0DD
:104903006402700EAC08AD09EEFAEFFB120AF5E98A
:1049130070DFAC08AD09EEFAEFFB120E49E9FA7449
:104923000A6A7005750A01801774A06A7012AC08D0
:10493300AD09EEFAEFFB120E55EEFAEFFB120E6D18
:10494300A90A740D12081D0234A5248DFAE9341343
:10495300FB1218C3E922E412495E2212496222F0D3
:104963008510828511830243C774F7120356EAFE4A
:10497300EBFF7508008E828F83A3A3A3A3A3A3A336
:10498300A3E06017EE24151223CB1226731247748B
:10499300120DB3E9640170037508018E828F83A33E
:1049A300A3A3A3A3A3A3E06018EE241312267512F6
:1049B30049C9FAA3E0FB120DB3E96401700375085A
:1049C30001A9080236641249CF022C55124C180271
:1049D30054A9EA240BF582EB22124E7E8882898346
:1049E300A3A3E02274F012035674F31208AF740306
:1049F300120A6DECF0A3EDF08A0E8B0F890B741D78
:104A0300120A6DE0F50A7E01EE120A6D740AF0E9EE
:104A13007007E50AC333240AF0851082851183AA3F
:104A230082AB83120D9B8A088B09EA7001EB70033A
:104A3300024AE2123A287409124BE0450A124BED7E
:104A4300120A6D124BC6E50B70307A008026EAC35A
:104A530033F8E433F9741E120A6DE028F8A3E03941
:104A6300F988828983124AF788828983122E1FA3C9
:104A73000EAF830AEAC3950A40D4E5082417F582EA
:104A8300E50912444F120D41E508241AF582E509A0
:104A930012439E7405120A6DAC82AD83AA0EAB0F4E
:104AA300120AC5E96021E508124AF2E50912444FEA
:104AB3007405120A6DA882A983E5082418F582E516
:104AC300091226781241CF850882850983A3A3E5BD
:104AD3000EF0A3E50FF0AA08AB09120BA3E9FEEE53
:104AE300F9740D8002740212081D7F080205632405
:104AF30016F58222124181F0A3AE82AF8322FEA378
:104B0300E03400FF022F0474F012035674FE1208FF
:104B1300AF8510828511831243A289088C0E8D0FF5
:104B23007412120A6DE0F50B900E9AE07002A3E086
:104B33006075E50BC333F8E433F9740E28FAE439EE
:104B4300FB1211858A0C8B0DAE0CAF0DEE7001EFCD
:104B5300605574D48E828F83124BBE1241C98E82EC
:104B63008F83A3A3A3A3E508F0AC0EAD0FEE24053A
:104B7300122C33EE240D122675E50BF07413120A72
:104B83006D124BB61207EBE50BC333FCE433FDEEBA
:104B9300240EFAEF124BB012081DEEFAEFFB900E43
:104BA3009A1243D5121A8A024AE8FAE50D3400FB39
:104BB300023C66E0F508A3E0023EEB123F48F8A38F
:104BC300E0F9221223D5FAEFFB124BD0221218C9B7
:104BD300124BD722EE2408FEEF3400FF228E828F81
:104BE30083F0A3E50BC43354E022F0A3AE82AF837A
:104BF300740322A3A3E508F0A3E509F022E0FA8EEB
:104C0300828F83A3A3E022124778120D2922122C4C
:104C13007B124C1822E002368374F7120356E9FE26
:104C23007C007D0078007900800C124CEC2CFCA3F6
:104C3300E03DFD1256121258645037E8FAE9FBEAD8
:104C430075F012A4FAAFF075F012EBA42FFBEA246F
:104C530015F582EB3412F583E064FF60D6124CEC59
:104C63007002A3E060CDEE60C1124CF1E4F0A3F05A
:104C730080C178007900800C124CCB2CFCA3E03D62
:104C8300FD1256121258575038E8FAE9FBEA75F04C
:104C930017A4FAAFF075F017EBA42FFBEA125852E2
:104CA300EB1258257004A3E064FF60D5124CCB705F
:104CB30002A3E060CCEE60C0124CD0E4F0A3F0801D
:104CC300C0ECFAEDFB023664124CD0E022E8FAE9BC
:104CD300FBEA75F017A4FA75F017EBA42FFBEA248F
:104CE300A0F582EB3413F58322124CF1E022E8FAAB
:104CF300E9FBEA75F012A4FA75F012EBA42FFBEAB4
:104D03002421F582EB3412F5832274F6120356EA5A
:104D1300FEEBFF9004D1801388828983E06E7003D9
:104D2300A3E06F603F88828983A3A312358D70014E
:104D3300E970E57A047B001211F18A088B09A8084F
:104D4300A909E87001E9601C88828983124D6E907D
:104D530004D112477488828983A3A31243A29004C7
:104D6300D11241CF0243ADA3A3A3A3EEF0A3EFF06F
:104D73002274F41203567E009004D180070E8882B9
:104D83008983A3A312358D7001E970F1EEC333FA61
:104D9300E433FB124E287001EB7003024E227F00B6
:104DA3009004D1802488828983124C14EFC333FA90
:104DB300E433FBE5082AF582E5093BF583ECF0A330
:104DC300EDF00F88828983A3A312358D7001E970FA
:104DD300D49004B6124E457003A3E06978087019A5
:104DE3001207EFEEF50A780A1207F37C827D047945
:104DF300009004B6124E31801A1207EFEEF50A78CE
:104E03000A1207F37C827D0479009004B61247747A
:104E1300120DBF740312081DAA08AB091211F71271
:104E23000BBB022D571211F18A088B09EA22124794
:104E330078120DC5228E828F83A3A3A3A3A3A3A35A
:104E4300A3A3124E7E900461E06822C082C08380D7
:104E5300128A828B83A3A3124E7A9004D11241CF7C
:104E63001211F79004D11235587001EB70E3024030
:104E73004EF582EF122C7E124E7E22E0024BC1745D
:104E8300F612035690046E123A319004DC124EEB84
:104E93001241CF7ADC7B0479501218E19004DC12C2
:104EA30023D1FAEFFB120E679004DC123A31900E15
:104EB3009CE07002A3E0602D7A067B00121185EA64
:104EC3007001EB602074D58A828B83F0E4A3A3F096
:104ED30074018A828B83123F30124D6A900E9C12AA
:104EE30043D5121A8A0243AD124EEF22E0F8A3E033
:104EF300F990046E22C082C0839004DE74F5F0A39F
:104F0300740DF09004E074EFF0A3740DF09004E2DC
:104F1300740DF0A3740EF002404EC082C08390045F
:104F230061E064FE7004A3E064FF600E90045BE044
:104F3300A2E15006120E4F120DFB120DF502404E68
:104F430074F61203569004AFE0602812117F8A08AA
:104F5300A8089004AFE0FA75F0E8A4CAACF075F0C5
:104F630003A42CFB747F582AFCE43BFD7A007B01ED
:104F73001220310243AD74F012035674FE1208AFCF
:104F8300750F00851082851183E4F0A3F0120B13D3
:104F93007A047900120AEFEAFE7A02790112515A71
:104FA3007A03790312515A120E2BEAF50E2EFF8E55
:104FB3000AEA250AF8E43400F9E87001E97003020B
:104FC30050BA8F0875090074027808120988AA0874
:104FD300AB09123F377002A3E070030250B88F0889
:104FE30075090074027808120988AC08AD0979FFC5
:104FF300851082851183E0FA12116D7508008056C1
:10500300A908120B0D8A0C8B0DEA7001EB60458A1F
:10501300828B83A3A3A3A3E0600464047036050F0B
:105023008A828B83A3A3A3A3A3A3A3A3A3A3E0F92C
:10503300120E5B851082851183120653EFFD850CDA
:1050430082850D83A3A3A3A3A3A3A3A3A3E01251C8
:105053006D12081D050885080A901E24E493F87450
:105063000193F9C3E50A98E4995006E50FC39E40FE
:105073008F750800E508C3950E503CAA087B001203
:105083000E318A0C8B0DEA7001EB60258510828549
:105093001183120653EA240EF582EB125169FEEADC
:1050A300240F1236BA120E5BEFFDEE12516D120889
:1050B3001D050880BF7F0075096A900459E0600CE4
:1050C300F9120A8FE9FA745CC39AF50975F003E5DE
:1050D3000984F50A851082851183E0F50EA3E0F5B6
:1050E3000F750B00E5096006750B20750900E50ACD
:1050F300C39F5004AE0A8008EFFEE50BD2E6F50B22
:10510300AC0EAD0FAA0BEEF9120E07E9F50CE50B89
:10511300A2E6401F1E750800800EE50E2404F50E5E
:10512300E50F3400F50F0508E508C39E40ECEECF0C
:10513300C39FFFE97006E50BA2E650A585108285A3
:105143001183E07002A3E060098510828511831248
:105153003289A90C024AE8120AEFEACEC39EFE2264
:10516300EE2411F582EF1236B422FC850C82850DF4
:1051730083124778120E0174022274F2120356EA64
:10518300FEEBFF8908740E120A6D124774750A004C
:10519300750B00750900800E8A0A8B0BEA2404FA4A
:1051A300EB3400FB0509E509C39D50218A828B83FB
:1051B300E064FF7004A3E064FF70158A828B83129E
:1051C3004D6EEC8A828B83125263E508F002202431
:1051D300E50A7002E50B600E850A82850B83C3E046
:1051E3009EA3E09F50B28A828B83124E7AC3EE98BD
:1051F300EF9950A4EAF8EBF988828983E064FF70A1
:1052030004A3E064FF6010E82404F8E93400F9051E
:1052130009E509C39D40E1880A890BE824FCF8E904
:1052230034FFF988828983E0F50CA3E0F50D850A44
:1052330082850B83E50CF0A3E50DF0888289831248
:105243005257123C9F125257A3F0C3EA98EB99406E
:10525300C60251BEA3A3E0850A82850B83A3A322C2
:10526300A312526822A3F08A82022E2E74F3120331
:105273005674FD1208AF89088A09ECFEEDFF750C20
:105283000175F003E9A42402C0E07401120A6DD091
:10529300E01253287001EB607C1249D51226781274
:1052A300532288828983F0741F55084509A3F0129D
:1052B3005472750900803D8E828F83E088828983D2
:1052C300F0A3A882A9838E828F831244538E828F88
:1052D30083A3A3E05407C4C0E08E828F83A3A3A358
:1052E300E05407FCD0E04C124455EE2404FEEF34A6
:1052F30000FF0509E509C3950840BC8A828B83A397
:10530300A374FC12446AEA2413F582EB12444F128D
:105313000BA3E9F50CA90C740312081D02417212C8
:105323004E7E74082212532DEA22124962120D9BFB
:105333002274F11203568A0A8B0B7508007AFE7BDE
:10534300FF7CFE7DFFE50A241DF582E50B124E77F7
:1053530088828983A3E0F509741F5509F50C12545B
:1053630072E50C600B88828983E0FEA3E0FBEEFA12
:10537300750D00803088828983E0FCA3E0FFECFE9A
:10538300E824020808E91254885407F50EA3A882FA
:10539300A983EFFD900461E06E7003A3E06F7003D7
:1053A300850E08050DE50DC3950C40C9E508700B86
:1053B300A909120E13E9700302546F12547C12549C
:1053C300968A0C8B0DA80CA90DE87001E9600EE418
:1053D3008882898312583FE508F002546F7CFF7D71
:1053E300FF12547C122678124774120E1F8A0C8BFC
:1053F3000DAE0CAF0DEE7001EF7033125953700107
:10540300EF60697C177D00790012116D12547C12D4
:1054130026781254A01241CF90046E1254AEA312F8
:1054230041CDEE240F125968EE240E12444CEE24A3
:105433000E122675E508F0EE240C123829EE24022C
:10544300FAEF3400FB120ABFE97021850A82850B4B
:1054530083A3A3A3A3A3A3A3A3E06010E50A241536
:10546300F582E50B1223CE2402122C33023271E8AB
:1054730024020808E93400F922E50A240BF582E541
:105483000B22F8E50912548C22125490223400F9AD
:10549300023297122C7E124778120AFB221254A46E
:1054A30022E0F8A3E0F98E828F83221254A40258DB
:1054B30048C082C08374FE6A700374FF6B70047902
:1054C300018034746059646060F5E9A2E5500F907F
:1054D3000461124E7AC3EC98ED99401980E1A2E67B
:1054E3009004615008C3E09AA3E09B80EDC3E09A67
:1054F300A3E09B50DA790002404E74F71203567E04
:105503000080041255180E901E2AE493FAEEC39AF3
:1055130040F1023664EE75F017A4248BFAE5F034FB
:1055230013FB120E372274F71203567800790080AA
:1055330003125612901E2AE493FEC3E89EE99400D8
:105543005064E8FEE9FFEE75F017A4FE85F00875D8
:10555300F017EFA425081258D1E06A7003A3E06B9B
:1055630070CFE8FEE9FFEE75F017A4FE75F017EFB4
:10557300A42508FFEE2495F582EF3413F583E06C40
:105583007003A3E06D600A74FF6C700374FF6D70A9
:10559300A0E875F017A4F8AAF075F017E9A42AF9A2
:1055A300E81256A980047A007B0002366474F6126E
:1055B30003567CFF7DFF7AFE7BFF120E1FEA70010C
:1055C300EB704978007900803EE8FCE9FDEC75F06A
:1055D30017A4FCAEF075F017EDA42EFDEC249AF59C
:1055E30082ED3413F583E0701BE8FAE9FBEA75F00A
:1055F30017A4FAACF075F017EBA42CFBEA248BFA92
:10560300EB3413FB12561212565D40BD0243ADE854
:10561300240102547674F71203567A007B00780053
:105623007900802EE8FCE9FDEC75F017A4FCAEF0E0
:1056330075F017EDA42EFDEC125852ED125825709B
:1056430004A3E064FF6008EA24010AEB3400FB12C0
:10565300561212565D40CD023664901E2AE493FC26
:10566300C3E89CE994002274F61203567E007D0081
:1056730080020E0D901E2AE493FCEDC39C501CED9A
:1056830012581D7004A3E064FF60E88E08EA650801
:105693007001EB70DDED1256A580047A007B0002E9
:1056A30043AD75F017A4248BFAE93413FB2274F786
:1056B300120356EAFEEBFFEE7001EF600E1256D1B5
:1056C3001244688E828F83A312445F0236647C1770
:1056D3007D00790012116D0254A974F7120356EA82
:1056E300FEEBFF7508008018A808E875F017A4A959
:1056F300F01259DC7003A3E06F60031259E205084E
:10570300901E2AE493FAE508C39A40DC02366474D7
:10571300F6120356120E1F8A088B09A808A909E876
:105723007001E9600AE8240DFAE93400FB80047A89
:10573300007B000243AD74F4120356EAFEEBFF8CC8
:105743000A8D0B7508007509008036E50975F01799
:10575300A4248DFAE5F03413FB120ABFE96020A8F4
:1057630009125A207003A3E06F700375080AAC0A8C
:10577300AD0BE875F017A412494D60034308A0056B
:1057830009901E2AE493FAE509C39A5004E50860D8
:10579300BA0223B374F61203567E008024EEF91284
:1057A3000B0DEAF8EBF9EA7001EB6014E824071239
:1057B300582D500CE488828983A3A3A312583FF089
:1057C3000E8E08901E24E493F8740193F9C3E50840
:1057D30098E49940C87E00803212581C7004A3E0FC
:1057E30064FF6026EE75F017A4248BF8E93413F9EF
:1057F300E8240C12582D5012E8240FF582E91238D0
:105803002CE8240EF582E912382C0E901E2AE4931C
:10581300FAEEC39A40C30243ADEE12584CE9125854
:1058230025223413F583E064FE22F582E91236B4AF
:10583300FA74012AF09004B0E0C39A22A3A3A3A3AD
:10584300A3123C9DA3A302340C75F017A4A9F02462
:105853008BF58222901E2AE493FAC3E89AE9940016
:1058630022901E24E493FA740193FBC3E89AE99B04
:105873002274F41203568A088B098C0A8D0B7E005E
:105883007F008008EE24010EEF3400FF901E2AE40F
:1058930093F8C3EE98EF94005031AC0AAD0BEEF8D9
:1058A300EFF9E875F017A4F8AAF075F017E9A42A40
:1058B300F9E812494D60CDEE75F017A4FEAAF07514
:1058C300F017EFA42A1258D1124BF8022D57FFEE0E
:1058D300125852EF3413F58322E9FA7907C3940D72
:1058E300400479018019EAC3940740047903800FC7
:1058F300EAC39403400419198005EA70027900028F
:1059030007CF74F01203568A0E8B0F8C0A8D0B8906
:10591300081259537001EF60341256D1E50EF0A30B
:10592300E50F125960A3A3A3A3E50AF0A3E50BF0C7
:10593300E508600AEE240F122675E5088008EE24B8
:105943000F1226757401F0EE240E125968024AED07
:10595300120E258A0C8B0DAE0CAF0DEE221259647C
:1059630022F002340812454CEE240D122C7B7402F3
:10597300F02274F51203568A088B09ECFEEDFF75CD
:105983000A008014E875F017A41259DC7003A3E031
:105993006F60031259E2050A901E2AE493FAE50A9E
:1059A300C39A5024A80AE875F017A4A9F01259CE97
:1059B300E065087004A3E0650970C9E875F017A4F1
:1059C3001259CE124D6E80CE0234A51259D2222422
:1059D30095F582E93413F583221259D2E06E22E859
:1059E3001256A5120E372274F7120356EAFEEBFF86
:1059F3007508008019A808125A207003A3E06F707D
:105A03000BE8125A2C7005E5081255190508901E6B
:105A13002AE493FAE508C39A40DB023664E8125895
:105A23004CE93413F583E06E2275F017A4248DFA44
:105A3300E93413FB120ABFE922C082C0839004E455
:105A43007479F0A3740EF09004E6747FF0A3740EDF
:105A5300F09004E87485F0A3740EF002404E74F4E1
:105A6300120356EAFEEBFF122F9F70358E828F834F
:105A7300A3A3A3A3A3A3A3A3A31206539004401217
:105A830043D57808120A2EAA08AB09AC0AAD0B8ECF
:105A9300828F83A3E0F9120C09740212081D120B02
:105AA300BB022D57C082C0839004B8125B58F0909C
:105AB30004B8E07002A3E070057901120DCB024037
:105AC3004E74F612035674FC1208AFEA2408F8EB7E
:105AD300122111125B581232967002A3E09004B89F
:105AE300700BE4F0A3F07901120DCB8063C3E09453
:105AF30015A3E0940040597900120DCB8A088B0955
:105B0300AC08AD09ECF8EDF9E875F064A4F8AAF077
:105B130075F064E9A42AF99004B812477412020DCF
:105B2300E8941AE994004028900E94E07002A3E0F0
:105B3300601E9004B81246D31241CF7402120A6D4C
:105B4300ECF0A3ED12495A900E941243D5121A8A1F
:105B530074040243AAE02401F0A3E0340022C082CB
:105B6300C08374F81208AF851082851183AC82ADAF
:105B730083758387758219740812074B8510828594
:105B83001183AC82AD83124954640170047900809F
:105B9300027901740802404BC082C0838A828B83DE
:105BA300E0D2E7F0121383027653C082C0837900F8
:105BB300125C35C082C08390042D127CE3D083D065
:105BC30082C3E09CA3E09D500C127C3CFAA3E0123C
:105BD3005CA660010902765374F7120356125C3512
:105BE300125DACAEF075F00BEDA42EFD90042FE02A
:105BF3002CFEA3E03DFF7401696005740269702007
:105C03008A828B83A3127D02127E4F7402697018FD
:105C1300125F961260A37010E48E828F83F0800867
:105C2300EA2403FCEB12608BEEFAEFFB120A9502F7
:105C33006828127D4EEB127D382274F41203568AC3
:105C4300088B09127D0879008A828B83E0604E7E7F
:105C5300007F008043125CA3703B125DB6F50AA37C
:105C6300E039F50B850882850983E08C82850B83F7
:105C73001271D5F8A3E0F98C82850B831260ABFC1B
:105C8300E509126024126093127D3DAA0AAB0B1240
:105C93000A95127D77126324125F9E40B80269C988
:105CA300EEFAEFFBEA75F00BA4FAACF075F00BEB30
:105CB300A42CFB90042F127E88F583E0540F2274EA
:105CC300F51203568A088B09740B120A6D127D7C38
:105CD300750A01EC7001ED6026EC126179ED127921
:105CE300667901120AA1EE7001EF606E8E828F83D6
:105CF300A3127D107902EEFAEFFB120AA1805BEE8C
:105D03007001EF6031126178EF127966EE2403FAC5
:105D1300EF12609D700CAA08AB09120AA7E9F50AF5
:105D230080CAE5082403FAE50912609D702C790303
:105D3300AA08AB0980C48A828B83A3E064FE700443
:105D4300A3E064FF700512609A700CAA08AB0912F5
:105D53000AA7E9F50A8003750A000268AB74F71213
:105D6300035690042D127BCFEA7001EB6031EA7584
:105D7300F00BA4FAACF075F00BEBA42CFBEAFEEBF2
:105D8300FF1211F190042F127BCF90042FE07002C9
:105D9300A3E06012EEFCEFFD790012116D80079015
:105DA300042FE4F0A3F0026828127CE7EC75F00BF3
:105DB300A4FC22EEF8EFF9125DC4E02822EEF8EF1E
:105DC300F9E875F00BA4F8AAF075F00BE9A42AF929
:105DD30090042F2290042D127982C3EE98EF99221A
:105DE300C082C083EC7001ED60051218C980097C84
:105DF300087D00790012116D02765374F612035672
:105E03007900EA7001EB60177C008C08EA25081220
:105E13007D70600479017C080CECC3940840EB02AC
:105E23006C4274F712035674F31208AFECFEEDFFE5
:105E3300E4851082851183F07401120A6D126E6875
:105E4300120AD77403120A6DAC82AD83EEFAEFFB2C
:105E5300120AB9EEFAEFFB120ABF02682374F712B3
:105E6300035674F31208AFECFEEDFFE48510828550
:105E73001183F0EAFCEBFD7403120A6D126E9F743A
:105E830001120A6D12617D12797074FE68700374D9
:105E9300FF69600479018002790002682374F712B4
:105EA3000356EAFEEBFF7508008E828F83E06017CE
:105EB300125ECD7012125ED88A828B83FCE05C7016
:105EC30006E04CF0120A95027141120A9BE9F508AB
:105ED3007401650822EE127D4FEF12797E125DC4C4
:105EE300E028FAA3E039FB8E828F83E02274F41258
:105EF30003568A088B097C007D00125F961260931B
:105F0300E508126179E509127D0C7900850882851F
:105F13000983A3E064FE7004A3E064FF60727E0063
:105F23007F008067125CA3605FEEFAEFFBEA75F017
:105F33000BA4FAACF075F00BEBA42CFB90042FE050
:105F43002AF50AA3E03BF50B850882850983A31292
:105F53007CFA850A82850B83A3E06A7003A3E06B56
:105F63007026E50A2403FAE50B12609D7014E50A16
:105F73002403FCE50B3400FDE5082403FAE50912CC
:105F83006093127D3D127D77126324125F9E4094CD
:105F93000269C9EA24030A0A0AEB2290042D127C3F
:105FA300FEC3EE9AEF9B2274F21203568A0A8B0BFE
:105FB3008A828B83A3127D10127D087508001260FC
:105FC3009A70597E007F00804E125DC0127E79E088
:105FD300540F6040125DB6F50CA3E039F50DE50CE6
:105FE3002403FCE50D1260243400FB1218C3E9649A
:105FF300017021850C82850D83A3127CDC850A82C6
:10600300850B83A3E8F0A3E9127C94127D487508FD
:1060130001127D79126324125DD740ADA90802767F
:10602300433400FDE50A2403FAE50B2274F5120359
:1060330056EAFEEBFF8E828F83A3127D107C007DD8
:1060430000EE24030A0A0A126092EEFAEFFB120A28
:106053009BE9F50A7401650A702B127CD3125DBAB1
:10606300F508A3E039F509850882F583A312617D5C
:106073001260ABFAE50912609D700AE5082403FC7F
:10608300E50912608B0268AB3400FDEE2403FAEFDE
:106093003400FB120AB922125F961260A364012234
:1060A3003400FB120ABFE922A3E8F0A3E9F0E508F4
:1060B30024032274F212035674E61208AFEAFEEBCD
:1060C300FF126178EF127D0C750801750A00750BDC
:1060D30000750C00750D00E4851082851183F0EEC8
:1060E3002403FCEF3400FD7403120A6D127046643E
:1060F30001702D740B120A6D127B7E126179EF12FF
:10610300796D7401120A6D12617DA3E0687003A3B7
:10611300E069605385108285118385820A85830B2C
:10612300740D120A6D12618B127CDC740E120A6DEF
:10613300127970740D120A6DAA82AB83120AD7E921
:106143006401700B740D120A6D85820C85830D78C2
:106153000C1207EFAC0AAD0BEEFAEFFB120AAD74AB
:106163000212081DE9F508EEFAEFFB120AD1A9089D
:10617300741A027640EE127D4F2212618122E0F8FA
:10618300A3E0F98E828F8322E4F08E828F83A32291
:10619300901E24E493FC740193FD2274F7120356BA
:1061A300E9FEEAFF7C007D0078007900802DE8FAA3
:1061B300E9FBEA75F012A4FA85F00875F012EBA476
:1061C3002508126335C39E400FE0FAEFC39A4008D7
:1061D300EC24010CED3400FD126602901E241265BE
:1061E3008940CBECFAEDFB026828EE240DF582EF33
:1061F300127D382274F212035674F31208AFEAFECA
:10620300EBFF8C088D09750A00AA08AB09120B0174
:106213008A0C8B0DA80CA90DE87001E960408882F7
:106223008983E06E7003A3E06F603388828983A360
:10623300A3A3A3E0C39405502588828983127D48D4
:106243007401851082851183F0120A6D127D48ACAA
:1062530008AD097403120A6D126268750A01A90A6E
:10626300740D027640126EAA120AE922C082C0831C
:10627300EAFCEBFD7A007B00120B07027653C08227
:10628300C0837C007D0080F074F412035674F31213
:1062930008AF8A0A8B0B8C088D097E007F00802152
:1062A3001264A1120A6D12632960137403120A6D3A
:1062B300AC82AD83AA0AAB0B1218C3E97038126320
:1062C3002412631B504912634A60F3E50A7002E526
:1062D3000B70CD74FF6508700474FF650960DFEE11
:1062E300F8EFF9E875F012A4F812649565087004E4
:1062F300A3E0650970C8EE75F012A4FEAAF075F06C
:1063030012EFA42AFFEE2411FAEF3412FB80047A71
:10631300007B00740D0269C6901E24126B69025D36
:10632300DE126342FF22E8F0A3E9126EC4120AE30D
:10633300E922FBEA2415F582EB3412F583E022EE21
:1063430024010EEF340022EEF8EFF9E875F012A401
:10635300F8AAF075F012E9A42AF9E8127E21E912ED
:10636300633C64FF2274F71203567A007B008009B2
:1063730019EA24010AEB3400FB126193C3EA9CEB94
:106383009D503AEAFCEBFDEC75F012A4FCAEF075FF
:10639300F012EDA42E127E1FED12633CC394055040
:1063A300D0E970CCEA75F012A4FAACF075F012EBF8
:1063B300A42CFBEA2411FAEB3412FB80047A007B51
:1063C3000002682874F712035674F31208AF7E00B4
:1063D3007F00026464E508127D20127CF8EEF8EF7A
:1063E300F9E875F012A4F8ACF075F012E9A42CF9F1
:1063F300E8127E096A7003A3E06B6044E50875F058
:1064030017A4F8AAF0EAF9E8248BF582E93413F526
:1064130083126FC1120A6DE0687003A3E069602004
:10642300E50875F017A4F8EAF9E8248DFCE93413BC
:10643300FD7403120A6DAA82AB831218C3E96011BB
:10644300E50875F017A4248BFAE5F03413FB120E5C
:10645300370508901E2A127D6150030263D8126328
:106463002412631B5029EEF8EFF9E875F012A4F833
:10647300AAF012649564FF7004A3E064FF60DF1266
:1064830064A1120A6D12632960D475080080C402E6
:10649300682375F012E9A42AF9E8127E0D2274012B
:1064A300851082851183F0EEF8EFF9E875F012A4F8
:1064B300F875F012E9A42AF9E82413F582E93412F5
:1064C300127980740B2274F6120356126C47FC7413
:1064D3000193FDEC8508F0A4CCAAF08509F0A42A69
:1064E300FA8508F0EDA42AFD79FF7AE77B131211F0
:1064F3006D900432742BF0A3740BF0900434742564
:10650300F0A3740BF0900436744FF0A3740BF09067
:1065130004387461F0A3740BF090043A7467F0A329
:10652300740BF090043C746DF0A3740BF090043E74
:106533007473F0A3740BF0E4900431F0026C42C066
:1065430082C0837800790080031266021265865048
:106553001CE8FAE9FBEA75F00EA4FAACF075F00E4C
:10656300EBA42C12657770E1126A0B80047A007B2E
:1065730000027653FBEA24E7F582EB3413F583E05C
:1065830064FF22901E22E493FA740193FBC3E89AFA
:10659300E99B2274F71203567A007B007800790096
:1065A3008045E8FCE9FDEC75F00EA4FCAEF075F057
:1065B3000EEDA42EFDEC24E7F582ED12657E60243A
:1065C300E8FCE9FDEC75F00EA4FC75F00EEDA42ECD
:1065D300FDEC24ECF582ED3413F583E0FCEA2CFAB0
:1065E300EB3400FB126602901E221265F540B302E3
:1065F3006828E493FC740193FDC3E89CE99D22E8B9
:10660300240108E93400F92274F112035674FC12D0
:1066130008AF7402120A6D127BCF890E8C088D0BA2
:106623007E007F00120B8B7402120A6D127CFA1229
:106633000B91127BC97402120A6D127CC470077528
:106643000A018E0980058E0A850809851082851145
:1066530083E064FE7004A3E064FF700302677E8E30
:10666300088002050885080C901E22127E2640032E
:10667300026711A808E875F00EA4A9F0126AFB6579
:106683000E70E0E875F00EA4126AC8650A70D4852E
:106693001082851183127CDCE50875F00EA424E9D1
:1066A300F582E5F03413F583E0687003A3E06970C5
:1066B300B2A808E875F00EA4A9F024EBF582E9343A
:1066C30013F583E06509709BE875F00EA424E7FEDB
:1066D300E93413FF750800E508C3950B400302670F
:1066E3007EE508C333F8E433F97413120A6D1267B5
:1066F30095120B37E97013E508C333F8E433F974E3
:1067030013120A6D126795120B43050880C9120B09
:106713001F8A0C8B0DAE0CAF0DEE7001EF605C8E1B
:10672300828F83E50EF0A3E50A1276348E828F837F
:10673300A3A3E8F0A3E91267A6E509F0901E26E4F7
:1067430093C3950B5004E493F50B8E828F83A3A31D
:10675300A3A3A3E50BF07413120A6D126AD0750A92
:106763000078081207EBE50BC333FCE433FDEE249A
:1067730006FAEF340012678E12081DEEFAEFFB746F
:1067830004800012081D7F07020563FB1211617468
:106793000322127E7D12679C22E0FCA3E0FDEEFA49
:1067A300EFFB221267AA22F08E828F838001A3A3BC
:1067B300A3A3A322C082C083901E2012619679FFF7
:1067C30012116D790102765374F7120356EA7001C0
:1067D300EB60498A828B83A3A3A3A3A3A3E582705F
:1067E30002E58360377E0080010E8A828B83A3A338
:1067F300A3A3A3E0FFEEC39F5022EEC333F8E43319
:10680300F9EA28F582EB39F583A3A3A3A3A3A3E0B5
:106813006C7003A3E06D70D179018002790080056B
:10682300740D12081D7F0102056374F5120356EA05
:106833007001EB605F8A828B83A3A3A3A3A3E060B1
:1068430063EA2406F8EB3400F98A828B83A3A3A3BB
:10685300A3A3E0F509750800800DEA2405F582EB92
:10686300127CED603F0508E508C395095026E5084D
:106873001268F3E06C7003A3E06D60DE1268F91236
:106883007D7C88828983127D48E824020808E934E4
:1068930000F980D18A828B83A3A3A3A3A3E060041E
:1068A3007901800279008002A90A7F0302056374DB
:1068B300F7120356EA7001EB60318A828B83A3A33C
:1068C300A3A3A3E0C0E0901E26E493FED0E0C39E02
:1068D3005019EA2405F8EB127E9B1268F3127E4FDF
:1068E30088828983E004F0790180027900026828B4
:1068F300C333FEE433FF127E910267B174F41203D3
:10690300568908EAFEEBFF8C098E828F83A3A3A32B
:10691300A3A3A3A3A3E0640170098E828F83127CD7
:10692300E38003126B0674FE6C700374FF6D7007D3
:106933007A007B000269C17800790080141269CE65
:106943006401700A1269EC7003A3E06D606D126656
:106953000212658650DAE8FAE9FBEA75F00EA4FA4A
:1069630085F00A75F00EEBA4250AFBEA24E7F5820D
:10697300EB3413F583E0650870D48E828F83A3A371
:10698300A3A3A3A3A3A3E0640160B21269CE70BE64
:106993001269EC7003A3E06D70B4E8FAE9FBEA75E1
:1069A300F00EA4FA75F00EEBA4250AFBEA24EBF52E
:1069B30082EB3413F583E065097093126A0B80064A
:1069C30012731C12081D7F04020563E8FAE9FBEA4F
:1069D30075F00EA4FA75F00EEBA4250AFBEA24E881
:1069E300F582EB3413F583E022E8FAE9FBEA75F06C
:1069F3000EA4FA75F00EEBA4250AFBEA24E9F5824E
:106A0300EB3413F583E06C22126A0F22E875F00E63
:106A1300A4F8AAF075F00EE9A42AF9E824E7FAE944
:106A23003413FB2274F21203568A0A8B0B8A828B6D
:106A330083A3A3A3A3A3A3A3A3E0640170098A82EE
:106A43008B83126AD08007120B798A088B0974FE34
:106A53006508700474FF650960687E007F00805AD2
:106A6300850A82850B83A3A3A3A3A3A3A3A3E064A3
:106A7300017041EEF8EFF9E875F00EA4F8AAF0758D
:106A8300F00EE9A42AF9E8126AC864017029EEF845
:106A9300EFF9E875F00EA4F875F00EE9A42AF9E809
:106AA30024E9F582E93413F583E065087004A3E073
:106AB30065097003126AD8126324901E2212631EA2
:106AC300409E02764324E8F582E90269E6E0F50890
:106AD300A3E0F50922EEF8EFF9126A0F120B312247
:106AE300EEF8EFF9E875F00EA4F8AAF075F00EE9E8
:106AF300A42AF9E8126AFB2224E7F582E93413F5A4
:106B030083E022120B798A0A8B0BAC0AAD0B227439
:106B1300F3120356890CEAFEEBFF750A00750B00AE
:106B23007508007509008029E50875F00EA4F8AA18
:106B3300F075F00EE509126AF3650C7011EEFCEFC7
:106B4300FDAA82AB83120B37E96003126BEE126B63
:106B530072901E22126B69E50898E5099940C9AA4B
:106B63000AAB0B0272D0E493F8740193F9C322E5E4
:106B7300082401F508E5093400F5092274F112032C
:106B830056890EEAFEEBFF8C09750800750A00753D
:106B93000B0080050508126BEE901E22127E18E58D
:106BA3000B995040E50A75F00EA4F8AAF075F00EA3
:106BB300E50BA42AF9E824E7F50CE93413F50D8570
:106BC3000C82F583E0650E70CDEEFCEFFDAA0CABF5
:106BD3000D120B37E960BFE508C3950940B6AA0C4F
:106BE300AB0D80047A007B00026789E50A2401F576
:106BF3000AE50B3400F50B2274F6120356750800F0
:106C030075090078081207EF126C47126E29758315
:106C13001E758220E49328FCA3E49339FD7A417B1B
:106C230000121257740212081DE9FE6003120B676B
:106C3300EEF9800B126E5412081D740212081D7FA8
:106C430002020563901E20126C53901E22E49322CD
:106C5300E493F508740193F5092274F6120356744C
:106C6300FE1208AF126C801207EF75080275090057
:106C730078081207EF7C007D007A4180B785108287
:106C8300851183E4F0A3126E5C85820885830978FD
:106C9300082274F412035674E71208AF7E007F00D3
:106CA30085108285118385820885830978081207F8
:106CB300EF7508028E0978081207EF7C007D007AD1
:106CC30041126D6812081DE96003026D518E088040
:106CD300757402120A6D85820A85830B780A12077E
:106CE300EF901E20120680126E17126D6812081D97
:106CF300E970507410120A6DAC82AD837404120AE9
:106D03006D127CFA120B7FE960397408120A6D85E3
:106D1300820A85830B780A1207EF7409120A6DE061
:106D2300FD7408120A6DE0FC7412120A6DAA82AB9C
:106D3300837404120A6DE0F9120B2B740212081DFE
:106D4300126324126B72126D5AE509994083EEFAAD
:106D5300EFFB74190269C68510828511831279824B
:106D6300C3E50898227B0012126374042274F5129F
:106D7300035674F01208AF851082851183E4F0A3E3
:106D8300F0FE8057126AE364FF604D8582088583B5
:106D930009750A0078081207EB901E201261967499
:106DA30005120A6DAA82AB8312678F12081D740243
:106DB300120A6D85820885830978081207EF901EF1
:106DC300201206807404120A6D126AD0126E171212
:106DD3006E5412081D126E44126342FF901E22125B
:106DE300631E40A0851082851183858208858309EF
:106DF30078081207EF75080275090078081207EF83
:106E03007C007D007A41126E5412081D7410120822
:106E13001D0268AD901E20E493126E29740228FCB3
:106E2300E439FD7A4122F8740193F9E88508F0A466
:106E3300C8AAF08509F0A42AFA8508F0E9A42AF97A
:106E430022851082851183E02401F0A3E03400F051
:106E5300227B0012125D740422126E6022F08510F0
:106E63008285118322EAF0A3EB126EC422C082C092
:106E73008374F31208AF12704B70128A828B8312E1
:106E83006FC1120A6D126EBC120AD7800CEAFCEBBA
:106E9300FD7403120A6D126E9F027648126EA322CE
:106EA300126EAA120ADD22AA82AB83120AB98510D6
:106EB30082851183AA82AB8322E8F0A3E9126EC410
:106EC30022126EC822126E6080EA74F7120356749F
:106ED300F31208AFECFEEDFF740485108285118375
:106EE300F0740B120A6DEAF0A3EB12632DF5086040
:106EF3001D74038E828F83A3A3A3A3A3A3A3A3F0D1
:106F0300120A6DAC82AD83EEFAEFFB1218C9A90821
:106F1300026823C082C08374F31208AF740485101F
:106F230082851183F0740B120A6D126E68120AE3E4
:106F3300740102764A127CFE740D2274F612035613
:106F430074F31208AF900431E0706E7404851082FC
:106F5300851183F0900461126FC1120A6D1279706A
:106F6300120D41EAFCEBFD7403120A6D1262681202
:106F73000D4D8A088B09A808A9097401120A6DE04E
:106F8300687003A3E069602B74FE68700374FF6983
:106F930060217401120A6D1279707403120A6DAACA
:106FA30082AB83120D53851082851183AA82AB8332
:106FB300120AE97401900431F0740D026C3F1279E6
:106FC30082740122C082C08374F31208AF12704B23
:106FD3008A828B83701E126FC1120A6DE8F0A3E9D7
:106FE300127D18705B851082851183AA82AB831290
:106FF3000AE9804CA3A3A3A3A3A3A3A3E064037000
:1070030010EAFCEBFD7403120A6D127046703180B6
:10701300D48A828B83A3A3A3A3A3A3A3A3E0640122
:1070230070128A828B83127CDC740B120A6DE8F077
:10703300A3E9800B740B120A6D74FEF0A374FFF0C6
:10704300027648126EA3E9227404851082851183A7
:10705300127DF4A3A3A3E064022274F5120356EA9B
:10706300FCEBFD7A007B008A088A097800790080AE
:1070730003126602901E22E493FE740193FFC3E899
:107083009EE99F5038E8FEE9FFEE75F00EA4FE85F9
:10709300F00A75F00EEFA4250AFFEE24E7F582EF60
:1070A30012657E60CCAE08AF0974012EF508E43F8B
:1070B300F509EC6E7002ED6F70B7126A0B0268ADE2
:1070C300C082C083900448748DF0A3740CF00276E0
:1070D3005374F7120356EAFEEBFF900470E0640862
:1070E3006019E0640460148E828F83E0640170444D
:1070F300127146127CA4E0640670398E828F83A3DA
:10710300A3E064FE7004A3E064FF60288E828F8393
:10711300A3A3127E2F7003A3E069700BEE2415F571
:1071230082EF127D736008120D0BE9F508800812D7
:107133000D1180F67508C2EEFAEFFB1211F7A908DC
:10714300026828EE240B127D352274F41203568A4A
:10715300088B098A828B83E0F8A3E028FAE43400E1
:10716300FB1211F18A0A8B0BAE0AAF0BEE7001EF23
:107173006059850882850983E0FC7D00790012113E
:107183006D8E828F83A3A3127D10120D478E828F83
:1071930083A3A3A3A3127D54F8EE28F8EF3400F9D8
:1071A300127146E8F0A3E91271D5C0E01261EDD087
:1071B300E0F0120D59EE240E1261F0E91274ADE005
:1071C300C0E0EE24111261F0D0E0F0EEFAEFFB0222
:1071D30069C91274B2E02274F412035674EB1208F4
:1071E300AF8A088B098C0A8D0B9004717808120AF8
:1071F3001FE9900477127316120A1F7405120A6DA1
:10720300E9F07404120A6D7401F07407120A6DE454
:10721300F074029004700269C374F412035674EBA1
:107223001208AFEAFEEBFF900440E07002A3E070A7
:10723300687A077B001211F1900440127BCF90040F
:1072430040E07002A3E0604D900440127CE38F8322
:107253008E82740712074B8E828F837808120A2E50
:107263008510828511837808120A1F8E828F83A36B
:10727300A3A3A3E0C0E07405120A6DD0E01272A3C9
:10728300E0C0E07404120A6DD0E0F07407120A6DD6
:107293001272D5800679108002790174150269C6CD
:1072A3001272A7221267AAA322C082C0839004404D
:1072B300E07002A3E0600D900440127D69900440E9
:1072C300E4F0A3F0120C9F120DDD0276537F05024A
:1072D3000563E41272DA22126EC81218ED2274F4F6
:1072E30012035674EB1208AF8A088B098C0A8D0BB4
:1072F3007401900470127316120A1F7405120A6D3A
:10730300E9F07404120A6D7403F07407120A6DE451
:107313000269C3126E5C7808221272DA7415227441
:10732300F412035674FC1208AFE9851082851183A9
:10733300F0EAFEEBFF127CE0120C998A088B09EA53
:107343007001EB700579CA0274A28A828B83A3A3AE
:10735300A3A3A3A3A3A3A3E064FE7004A3E064FF19
:10736300700579C30274A290046E127CFA120E3D6A
:10737300E508240CF582E509127D7304900481F07D
:10738300EEFCEFFD7A827B041218C97402120A6DB7
:107393007402F07401120A6DAA82AB83120D9B8AE8
:1073A3000A8B0BAE0AAF0BEE7001EF7003027498F9
:1073B300127CD3740688828983F0A3A882A9839060
:1073C300045B127CA0F0EE2417F582EF127C8AEEA8
:1073D300241A1261F0127BCFEE24131261F07401B0
:1073E300127D2D7440F0A3E41274ADA3A3A3A3A351
:1073F300A3A31274A7127B83120BA3E9F50A6003FC
:1074030002749B7409900470F0E5082409FEE509F1
:107413003400FFEEFAEFFB794B1218E18E828F8373
:10742300127CDC900464127970900463E0FA851096
:1074330082851183E06A600CE090046312763C79E4
:10744300E11218E190149C127CDC90149EE06870A9
:1074530003A3E069601A90044212797090149E129B
:107463007CFA120D7190149E127CE37A01127E3E17
:107473007A007B049004BBE0F912129390149E12DD
:107483006AD074027808120988AC08AD09FA7B0443
:10749300127E408003750A10E4900E5AF0A90A7414
:1074A300040269C6126181A3A3221274B2A322F05B
:1074B300850882850983A32274F012035674E212AD
:1074C30008AF127E498A0C8B0D742E120A6DE0F5FB
:1074D30008900470E064046005E06408700579C2F4
:1074E30002761D851082851183E0FC120C998A0AAD
:1074F3008B0BAE0AAF0BEE7001EF700579CA027603
:107503001D8E828F83A3A3A3A3A3A3A3A3A3E0643A
:10751300FE7004A3E064FF700579C302761D740353
:1075230090047012763C79501218E1EE2409F50AA2
:10753300EF3400F50BAA0AFB794B1218E185108290
:10754300851183127622127970EE2402F50EEF3440
:1075530000F50F850E82F583E0900463127629907F
:107563000464127970E50890045BF0AC0CAD0D7AFD
:10757300827B041218C974CE55084480C0E074128B
:10758300120A6DD0E0F0740F120A6D74021276299C
:107593007407120A6DE8F0A3E91276347410120A24
:1075A3006D127970850E82850F83E0C0E074051239
:1075B3000A6DD0E0F0741B120A6DE41267A6E09026
:1075C3000476F07A767B0479541218E18E828F83E5
:1075D300A3A3A3E0900475F07A757B04794712188E
:1075E300E1900475E0C3940F50247405120A6DE012
:1075F300C0E07402120A6DD0E0F07404120A6D74D4
:1076030001F07402120A6DAA82AB831218F3740597
:10761300120A6DAA82AB831218E7741E027D8212CE
:10762300798290046E22F0850A82850B8312798217
:1076330022127E55F8A3E0F922126EC42212081D0D
:107643007F06020563740B120A6D126F3812081D50
:10765300D083D0820207CF74F412035674F9120850
:10766300AF8A088B098C0A8D0B851082851183786C
:1076730008120A1F7404120A6DE9F07405120A6DE8
:10768300E4F07406120A6DE412763C120BB574072B
:107693000269C674F41203568A088B098A828B83A3
:1076A300127D7CEE7001EF70030277B490040FE05B
:1076B3007002A3E060158A828B83A3A3E0F9EEFA3C
:1076C300EFFB90040F127CA4121A8A8E828F83A37D
:1076D300A3A3A3A3A3A3A3A3E06402707F8E828FBB
:1076E30083A3A3A3A3A3A3E0540270030277838518
:1076F3000882850983A3A3E064E970030277838E7C
:10770300828F83A3A3A3A3A3A3A3A3A3A3E0701420
:107713009014ADE0048E828F83A3A3A3A3A3A3A39A
:10772300A3A3A3F08E828F83A3A3A3A3A3A3A3A343
:10773300A3A3E014F074048E828F83A3A3A3A3A353
:10774300A3A3A3A3F09014AE1274A7A3A3E8F0A37A
:10775300E9127E667001EB7003127DFC8E828F83CB
:10776300A3A3A3A3A3A3A3A3A3E0640260128E8293
:107773008F83A3A3A3A3A3A3A3A3A3E0640670314E
:107783008E828F83A3A3A3A3A3A3E0A2E0502285A9
:107793000882850983A3A3E0F9EEFAEFFB12196BC4
:1077A3008E828F83A3A3A3A3A3A3E054FEF0A3E03D
:1077B300F00269C974F012035674DD1208AF8A0C23
:1077C3008B0D8C0E8D0F7433120A6D7808120A2EEE
:1077D3007F00740E120A6DAC82AD83121227740EF1
:1077E300120A6DE0A2E5500D0F127CF3121977E92E
:1077F3006003027947740E120A6DE0A2E6500E741C
:107803000F120A6DE0540370047E0180027E00743F
:107813000E120A6DE05403FA74026A7009127CF3C3
:10782300120A8302794774016A7043EE6003127986
:107833004C740E120A6DA882A9837403120A6DE8B0
:10784300F0A3E91279768510828511831279708508
:107853000C82850D83A3A3A3A3A3A3E0C0E07402BA
:10786300120A6DD0E012763C121A67027947EA6079
:1078730003027947740D120A6D7402127976740546
:10788300120A6D127970EE6008740E120A6D127985
:107893004C740E120A6DE0540C64047071E50C24F0
:1078A3000FF582E50D127D73C0E07420120A6DD0CE
:1078B300E0F0900411E07002A3E070030279471234
:1078C3000D478A0C8B0DA80CA90D7405120A6DE0E7
:1078D300687003A3E069706C78081207E7EFF50896
:1078E30078081207F3780E1207EFEEF97415120AEF
:1078F3006DAC82AD83740C120A6DAA82AB839004C3
:1079030011127CA4121A8A740712081D8036AA0C5D
:10791300AB0D121A1FE9602C78081207E7780E12D4
:1079230007EF90046E120653EFF9740D120A6DAC53
:1079330082AD837416120A6DAA82AB8312195F7427
:107943000812081D7423027D82127959127D3812A0
:107953007CFE120A7722AC82AD83E50C240BF58200
:10796300E50D2212797E127D4EEB127D38E8F0A3ED
:10797300E9F022F012795D12797E223400F583E07A
:10798300027637C082C08312135F027653C082C06F
:1079930083121365027653C082C08312136B02767F
:1079A30053C082C083121371027653C082C0831204
:1079B3001377027653C082C08312137D0276537409
:1079C300F412035674F91208AF8A088B098C0A8DD6
:1079D3000B7413120A6D127CFA900E98E07002A3D6
:1079E300E06027E9851082851183F07401120A6D26
:1079F3007808120A1FEAF8EBF97405120A6D126E81
:107A0300BC900E98127CA4121A8A02769174F71213
:107A13000356901444E0F97F00800B127C59540DF7
:107A230064017001190F127C515003E970ED026873
:107A33002874F7120356901445E0F97F00800B1267
:107A43007C59548D64817001190F127C515003E9E4
:107A530070ED02682874F2120356890AE975F0067C
:107A6300A4F8A9F0740C28FEE439FFEA2EFAE43FE7
:107A7300FB1211F18A088B09EA7001EB6029EEFC15
:107A8300EFFD790012116D127D8AE50AF0E5082EEB
:107A9300F8E5093FF9850882850983A3A3A3A3A376
:107AA300A3A3A3A3127970AA08AB0902764374F6C1
:107AB3001203568A088B09120C27901443E0FAE943
:107AC300C39A400990044A127CFA120C2DE508244B
:107AD30002FEE5093400FF90044C127D95F09004FA
:107AE3004CE004F0AA08AB09120C338E828F83E0BA
:107AF300026C34C082C083790090044A8001091269
:107B03007CFA8A828B83E5827002E58370F00276C9
:107B13005374F7120356EAFEEBFFEE7001EF605861
:107B230090044AE07002A3E0604E90044A127CB5D0
:107B33007A007B00800FAA82AB83127CB5E582704A
:107B430002E5836033EE65827003EF658370E7902F
:107B5300044A127B7E687002EF698E828F837008FD
:107B6300127CDC90044A8003127E5A127B83121A21
:107B730037EEFAEFFB1211F7026828127982EE2230
:107B8300E8F0A3E9F00267A1C082C08390044A80B1
:107B93000488828983127CDCE87001E9600B8882A7
:107BA3008983E07002A3E070E88A828B83E4F0A308
:107BB300F0E87001E9600688828983800390044AB3
:107BC300127BCF027653851082851183EAF0A3EBF3
:107BD300F02274F7120356E9FC90044A80048A8267
:107BE3008B83127C4C7001EB60177E0080010E12B8
:107BF3007C3CFDEEC39D50E6EE127C726C70EF8010
:107C0300047A007B0002682874F7120356E9FD7FAB
:107C13000080010F127C3CFEEFC39E5019EF127CD3
:107C2300726D70EFEF75F006A4F8A9F0127D9974E8
:107C330011127C814CF0026828127C4022EA240B4A
:107C4300F582EB3400F583E022127CFEEA22127CFB
:107C530040FCEFC39C22EF75F006A4FCADF0EA2CC8
:107C6300FCEB3DFD74112CF582E43DF583E02275B8
:107C7300F006A4F8A9F0EA28F8EB39F9741028F50E
:107C830082E439F583E022127D387401F0120D414C
:107C930022F0E50A127D4FE50B127D3822E0027CCB
:107CA300BA127CA822127CAC22E0F8A3E0F5838808
:107CB300822212798280008882898322FAA3E0FBE0
:107CC30022127E38A3A3A3E06401228A828B83223B
:107CD300EE127D4FEF3400F5831279822290046E09
:107CE300127CE722E0FCA3E0FD22127C4614F02282
:107CF3001279593400F583127CFE22E0027CBF1214
:107D03007CE702618D127D4EEB3400F58374FEF047
:107D1300A374FFF022126EC4120AD7E92275F0177A
:107D2300A4248BF582E5F0341322F0EE240F127DA8
:107D33003522F582EF3400F58322E508127D4FE505
:107D4300093400F583EEF0A3EFF022EA240BF58269
:107D530022EAF0A3EBF0850882850983E022E4930D
:107D6300FAE508C39A22127CFE1211F722F582EB80
:107D7300127C4622790190042DE0FEA3E0FF22123B
:107D8300081D7F08020563E508127D4FE509127D92
:107D93003822E0026186EA28F8EB39F92274F312FB
:107DA300035689088A09ECFEEDFF750C0080020575
:107DB3000CE50CC39508502AE50CC333F8E433F9FA
:107DC300EE28F582EF39F583C082C083120D478A0E
:107DD3000A8B0BD083D082E0650A7004A3E0650BA5
:107DE30070CDE509650C7004790180027900027297
:107DF300D0F08A828B830267B17A207B009004BB28
:107E0300E0F91211B522127E0D222411F582E93414
:107E130012F583E022126B69E50A9822FDEC241522
:107E2300F58222126B69E50C98E49922127982900B
:107E33000461E06822127CAC0267B17B009004BB52
:107E4300E0F912128D22851082851183ECF0A3EDE7
:107E5300F022126E60E022127E5E22E0F8A3E0F9C7
:107E6300027CCEF07A20127E6D227B009004BBE070
:107E7300F9121299EA22127E7D22E028FAA3E03950
:107E83008A82F58322E02AFCA3E03B8C8222EA2E3D
:107E9300F582EB3FF583A3223400F988828983E0DE
:107EA3002274F7120356E9FE8A08EBFF127FB174BE
:107EB300BA28F582740F39F583127ED3E5824583A0
:107EC3006009EFFBAA08EEF9121A8A7F0102056323
:107ED300E0F8A3E0F98882898322E9600924FE603F
:107EE3000914600A800C7901800A790280067900FE
:107EF300800279030207CFC082C0837903127F9C7B
:107F03007033E5E4A2E5500C53E4DF7B027A027997
:107F1300031215D5E5E4A2E6500C53E4BF7B027AC5
:107F23000479031215D5E5E4A2E7502253E47F7BDD
:107F3300027A0880147903127F967012E5E4A2E4B2
:107F4300500C53E4EF7B047A0179031215D5D083E7
:107F5300D0820207CFC082C0837900127F9C701B3E
:107F6300A2D9500BC2D97B027A0279001215D5A28D
:107F7300DA501EC2DA7B027A0480117900127F96EE
:107F8300700FA2D8500BC2D87B047A017900121566
:107F9300D580BB127FA2640422127FA26402221244
:107FA3007FB174B628F582740F39F583E022121578
:107FB300DBE975F00AA4F8A9F022C082C083790234
:107FC300127F9C701BA2DC500BC2DC7B027A02790D
:107FD300021215D5A2DD501EC2DD7B027A04801188
:107FE3007902127F96700FA2DB500BC2DB7B047AFF
:097FF3000179021215D5027F513B
:108000000000000000000000000000000000000070
:10801000000000F800000000000000333000000005
:1080200000100C06100C060000000000000000000C
:1080300040C07840C0784000043F04043F0404007E
:10804000007088FC08300000001820FF211E00008E
:10805000F008F000E018000000211C031E211E00A3
:1080600000F00888700000001E2123241927211029
:1080700010160E00000000000000000000000000CC
:10808000000000E018040200000000071820400073
:1080900000020418E0000000004020180700000063
:1080A000404080F0804040000202010F01020200C7
:1080B000000000F0000000000101011F01010100AB
:1080C000000000000000000080B070000000000010
:1080D0000000000000000000000101010101010199
:1080E0000000000000000000003030000000000030
:1080F0000000000080601804006018060100000005
:1081000000E010080810E000000F102020100F0001
:10811000001010F8000000000020203F2020000088
:1081200000700808088870000030282422213000E0
:1081300000300888884830000018202020110E00E8
:108140000000C02010F8000000070424243F240091
:1081500000F80888880808000019212020110E0066
:1081600000E0108888180000000F112020110E0078
:1081700000380808C83808000000003F0000000070
:108180000070880808887000001C222121221C0031
:1081900000E010080810E0000000312222110F005A
:1081A000000000C0C00000000000003030000000EF
:1081B000000000800000000000008060000000005F
:1081C0000000804020100800000102040810200078
:1081D00040404040404040000404040404040400C3
:1081E0000008102040800000002010080402010058
:1081F000007048080808F000000000303601000058
:10820000C030C828E810E0000718272423140B000A
:108210000000C038E0000000203C23020227382084
:1082200008F8888888700000203F202020110E0068
:10823000C03008080808380007182020201008005F
:1082400008F808080810E000203F202020100F0048
:1082500008F88888E8081000203F20202320180014
:1082600008F88888E8081000203F2000030000007C
:10827000C03008080838000007182020221E02001D
:1082800008F808000008F808203F210101213F20DC
:10829000000808F8080800000020203F2020000007
:1082A00000000808F8080800C08080807F000000F7
:1082B00008F888C028180800203F20012638200030
:1082C00008F8080000000000203F20202020300097
:1082D00008F8F800F8F80800203F003F003F2000B1
:1082E00008F830C00008F808203F200007183F00B9
:1082F000E01008080810E0000F10202020100F00E8
:1083000008F808080808F000203F210101010000DA
:10831000E01008080810E0000F18242438504F001F
:1083200008F8888888887000203F2000030C3020DF
:1083300000708808080838000038202121221C001D
:10834000180808F8080818000000203F2000000066
:1083500008F808000008F808001F202020201F004F
:108360000878880000C83808000007380E010000AF
:10837000F80800F80008F800033C0700073C030079
:10838000081868808068180820302C03032C3020DF
:108390000838C800C83808000000203F200000004E
:1083A00010080808C83808002038262120201800A6
:1083B000000000FE020202000000007F404040007A
:1083C000000C30C000000000000000010638C000B2
:1083D00000020202FE000000004040407F0000005A
:1083E000000004020202040000000000000000007F
:1083F000000000000000000080808080808080807D
:108400000002020400000000000000000000000064
:1084100000008080808000000019242222223F205A
:1084200008F8008080000000003F112020110E009D
:108430000000008080800000000E1120202011002C
:10844000000000808088F800000E112020103F20DE
:108450000000808080800000001F22222222130062
:10846000008080F0888888180020203F20200000AD
:108470000000808080808000006B94949493600062
:1084800008F8008080800000203F210000203F206D
:1084900000809898000000000020203F202000006D
:1084A000000000809898000000C08080807F00005D
:1084B00008F8000080808000203F24022D3020003A
:1084C000000808F8000000000020203F20200000E5
:1084D0008080808080808000203F20003F20003FFF
:1084E0008080008080800000203F210000203F200D
:1084F0000000808080800000001F202020201F00BE
:10850000808000808000000080FFA12020110E00EC
:108510000000008080808000000E112020A0FF80DD
:10852000808080008080800020203F21200001008A
:1085300000008080808080000033242424241900DF
:10854000008080E0808000000000001F20200000EC
:108550008080000000808000001F202020103F202D
:10856000808080000080808000010E3008060100BD
:1085700080800080008080800F300C030C300F0062
:1085800000808000808080000020312E0E3120008D
:10859000808080000080808080818E7018060100BD
:1085A00000808080808080000021302C22213000DB
:1085B00000000000807C020200000000003F4040FC
:1085C00000000000FF00000000000000FF000000AD
:1085D0000002027C800000000040403F00000000DC
:1085E0000006010102020404000000000000000077
:1085F000000000000000000000000000000000007B
:1086000000000000000000000000000000004E4DCF
:108610002D656E65726779206E6F742075700053DA
:10862000746172744465766963652045525200E155
:108630000F510C1B156D1AC5190B13C513DB124D09
:1086400061746368204465736320526571004173EF
:10865000736F6320436E66206661696C004D4F4402
:108660004520756E6B6E6F776E00456E657267792B
:10867000204C6576656C000B050F010000025587E4
:108680000255875363616E204661696C6564004ED4
:108690006F6E204D61746368656400000000000027
:1086A00000000000000000000000000000000000CA
:1086B00000456E644465766963653A000000000019
:1086C00000000000000000000000000000000000AA
:1086D0004E574B204944203A200000000000000083
:1086E000000000004173736F6320436E66005365A2
:1086F0007269616C417070005273702053656E74C2
:1087000000FFFFFFFFFFFFFFFF506172656E743ACD
:108710000053756363657373000000000000000080
:1087200000FFFFFFFFFFFFFFFF506D322E353A20A5
:108730000054656D703A200048756D693A20004913
:108740004545453A20000BEE0D77860002050200F4
:108750000000580000010000006400000000000C50
:108760000000F8FF0730000000000000FF000000DC
:10877000001027000000E1F505010000003A20008C
:1087800030000874F7120356E9FE120B19EE90142C
:1087900041F090040B7461F0A3741AF090040D740E
:1087A0005BF0A3741AF090040F7455F0A3741AF0E0
:1087B000900411744FF0A3741AF00299E4C082C0BF
:1087C00083E4900401F0E9900400F07C347D0F7A9A
:1087D000027B041218C99014B1E090040AF0121A36
:1087E0002B029DA874F4120356EAFEEBFF74805F1F
:1087F000F9E47001E97026EE5402605F7401901490
:1088000040F074026EFA8066E06402700990042100
:10881000129FBB121A8AAA08AB0912118B9004008E
:1088200012AFF87001EB602B8A828B83E0640170D9
:10883000D712AFEF12064F1288711207EF12919DF7
:108840001298CC12065312B00312110D74081208BC
:108850001D80C3EEFA74806FFB8013EE5408600A2B
:10886000121A2574086EFAEF80EE7A007B000289F6
:1088700086EA240FF50AEB3400F50B780A2274F42B
:108880001203568A088B098A828B83A3A3A312AF93
:108890003C2409FA12A2C87001EF700302892A74FD
:1088A000028E828F83F0E4A312989312A028850889
:1088B00082850983A3A3129FEDF0E5082403F8E560
:1088C000091292912410129B708E828F83A3A3A30E
:1088D000A3F0EE2409FA12892C129D4FF5838882A9
:1088E000E0A2E5500474018001E48E828F83A3A38B
:1088F000A3A3A3F0E5082403F888828983129D07C7
:1089000012B5AAEB1298CC129D371207EB12B5D50F
:10891000EB129CFF8E828F83A3A312A24212081D2A
:10892000EEFAEFFB90040012A2B3805AEF3400FB82
:108930008E828F83A3A32274F41203568A088B09B4
:10894000ECFAEDFB740C120A6DE0FC120B498A0A7A
:108950008B0BAE0AAF0BEE7001EF6023AC08AD09D4
:10896000120B37E96019AC08AD09EEFAEFFB120BF8
:108970003DE97007EEFAEFFB120B317900800279C6
:10898000B4800312081D7F0402056374F0120356BD
:1089900074F51208AFEAFEEBFF8C088D09750CB375
:1089A000750D00851082851183E4F0A3800312B059
:1089B000CD12B45AC082C083901E22E493F8740191
:1089C00093F9D083D082C3E098A3E0994003028A50
:1089D000E585108285118312A870120B978A0E8B81
:1089E0000FEA7001EB60C78A828B83A3A3A3A3A3C2
:1089F000E0250DF50DF50AC3EE950AEF940050AE93
:108A00007C157D007900AA08AB0912116D850E82D4
:108A1000850F83A3A3A3A3A3EEC3950DFAE02AC3F6
:108A200033F8E433F9E50E28F582E50F39F58312C2
:108A3000B0B4850882850983A3A3A3A3A3129D3B99
:108A4000EAFCEBFDAA08AB091218C9850E82850F56
:108A500083A3E06401700A12A96F740112A254800A
:108A60004A7402120A6DAC82AD83850E82850F8333
:108A700012A86E120B7FE96043740A120A6DE0C0FF
:108A8000E012A96FD0E0F0740A120A6DE06403707E
:108A9000157402120A6DAC82AD83E508240BFAE569
:108AA0000912988080167402120A6D12B0BAE50895
:108AB000240BF582E5091298CC12A036850E82852A
:108AC0000F83E0850882850983A3A3A3A3A3A3A39F
:108AD000A312A254A3A3E0C0E012A94C1298CCD0D8
:108AE000E0F0750C00A90C740B02AEF7C082C083D5
:108AF0008A828B83A3A3A3A3A3A3E0540860298A3B
:108B0000828B83A3A3A3A3A3A3E0540260178A824A
:108B10008B83A3A3A3A3A3A3A3A3A3E064066005DD
:108B200074E9697003121A43029DA874F112035686
:108B300074EF1208AF740F120A6D12A06C74081251
:108B40000A6DE9F0ECFEEDFF7423120A6D7808124D
:108B50000A2E7405120A6DE4129FC2128DF8120BD0
:108B6000557406120A6D12A06C7406120A6DE0703C
:108B700002A3E07003028D91EE241012A78D7406FB
:108B8000120A6DE0F9120C1B7401120A6D12A06C2E
:108B90007401120A6DE07002A3E07003028D91EE81
:108BA0002406F50CEF3400F50D7C00850C82F5836E
:108BB000128DEE120A6DEAF0A3EB129F2CC0E07446
:108BC00001120A6D12990CA3A3D0E012A2B974018C
:108BD000120A6D128DDD1298D5E0F87401120A6D3B
:108BE000128DDDA3A3A3E812A0237401120A6D1253
:108BF0008DE3A3A3E412B5C7F50CA3E0F50D750E44
:108C000000780C1207EBEE12B5D6EF129CFF74043D
:108C1000120A6D1299E912A24212081DE48510820F
:108C2000851183028CE67403120A6D129C7BFAA3F1
:108C3000E0FB120B85850C82850D83A3EAF0A3EB84
:108C4000F07403120A6D128DE312ABDF12A2E6E09C
:108C5000A2E6500F850C82850D83A3A3A3A3A3E0F6
:108C6000D2E1F07405120A6DE0705A850C82850D10
:108C70008312B0B9900461E0687003A3E0697045A5
:108C8000850C82850D83A3A3A31298BF78081207D1
:108C9000E77424120A6D12065390046E1206537480
:108CA0002A120A6DE0F97417120A6D12B5DB121957
:108CB0005F740812081D850C82850D83A3A3A3A3EE
:108CC000A3E04405F0851082851183E004FC8E82C8
:108CD0008F83A3A3A3A3A3A3128DEE120A6DEAF0C0
:108CE000A3EB129FC704F07403120A6DE07002A395
:108CF000E0606F851082851183E0FA7406120A6DB8
:108D000012B0BAC3EA98E49950588510828511834D
:108D1000E075F006A4F8A9F07401120A6D1290280B
:108D2000F50CE439F50DE4850C82850D83F07403B0
:108D3000120A6D12993E64016003028C26740512BA
:108D40000A6D740112A29DF07403120A6D129C79CF
:108D5000F8A3E0F9850C82850D83A3E8F0A3E9026E
:108D60008C407401120A6D12A870120C2174011249
:108D70000A6D1206537424120A6DE0FC740A120A7A
:108D80006DE0F9EEFAEFFB121A49740212081D8029
:108D9000478E828F83A3A3A3E0C0E0740C120A6DF8
:108DA000D0E012938BC0E0740D120A6DD0E0F07425
:108DB00006120A6DE07002A3E07009740E120A6DCB
:108DC00074B98007740E120A6D7401F07409120AE6
:108DD0006DAA82AB83121965741102B64012992FE5
:108DE000A3A322128DE722129D77A3A3A322E01250
:108DF0008DF8120B5B740322FAA3E0FB8E828F8343
:108E0000A3A3A3E0F92274F012035674F01208AF82
:108E10007402120A6DE9F08A0C8B0D8C0F7420120B
:108E20000A6D12A870120C0FE9F50E7420120A6D6B
:108E300012A870120C15E50E700302901A750B0043
:108E4000800F8E828F83A3A3A3A3A3E0D2E3F005B8
:108E50000B7420120A6DE0240B129D0CFAE50BC373
:108E60009A400302900DE50E700302900DE50B751C
:108E7000F006A4F8A9F07420120A6D129028FEE4FE
:108E800039FF8E828F83A3A3A3A3A3E0A2E040BFF8
:108E9000750800851082851183740812A023E50FE0
:108EA00060037508207C087D0079007403120A6D48
:108EB000AA82AB8312116D8E828F83E060244308F7
:108EC0000C851082851183740C12A0238E828F83EF
:108ED000A312ABF412A0327403120A6D74FFF0A354
:108EE00080297402120A6DE06011E508D2E6F508E7
:108EF000851082851183740A12A0238E828F8312BB
:108F0000B0B97403120A6DE8F0A3E9F07405120A0F
:108F10006DE50812A266C0E07407120A6DD0E0F099
:108F20007408120A6D7401F07403120A6DAA82AB00
:108F300083121983740F120A6DE06003028FF074BC
:108F40000B120A6D1299568E828F83A3A3A3A3F0EE
:108F5000740B120A6D12B5E312A870E81298F1E9C9
:108F60001298CC129F197420120A6DE0129033C02F
:108F7000E0740B120A6D12B436D0E0129F2CC0E0E0
:108F8000740B120A6D12967DD0E0F0740B120A6D0C
:108F900012ABF412B43D12A273E012A05F12B2B68B
:108FA000E50D12B5B5C0E0E8242EF582E91298CCA3
:108FB000D0E0F0740B120A6D12A870850C82850D3A
:108FC0008312901F2424F582EB1298CC12A27A12FD
:108FD00007EB129CF7EA242BF582EB1298CC12A235
:108FE0004212081D7403120A6DAA82AB8312197D06
:108FF0008E828F83A3A3A3A3A3E0D2E0F0740F1209
:109000000A6DE06003028E42150E028E4F790074E5
:1090100020120A6D12A870121A3D741002AEF7A346
:10902000A3A3A312B0BEEA22E028F8A3E039F974A2
:109030000C2822F81290382212B5FFA3A3A3E02235
:1090400074F212035674EB1208AFEAFEEBFF890AC2
:109050008E828F83A3A3A3A3A3A3A3A3E0F9120CDF
:10906000398A088B09EA7001EB70030290F4E50A73
:1090700070047C0480027C088E828F83A3A3A3A348
:10908000A3A3A3A3E0F9120C3F12B5AF7002A3E0B3
:109090006062EE12B5D0EF12A0A5A3A312A86E7461
:1090A00006120A6D1290F912A8707408120A6D1255
:1090B00090F9A3A3E0C0E07410120A6DD0E012A0F2
:1090C0000312A86E740E120A6D12A06C7411120AAB
:1090D0006DE412A9AEFA78081207EF74205AFC74F6
:1090E000405AF97402120A6DAA82AB83121A4974AB
:1090F0000212081D7415029878EAF0A3EB129CEE98
:10910000A3A3A32274F712035674FA1208AFE9FC62
:109110007E017F017D0080037F000D12919D12B5BD
:10912000B5F8EDC3985027ED75F006A4F885F00862
:10913000A908EA28F8EB39F974111298B6A2E050A0
:10914000D7540C60D3E0A2E250D07E0080CC8A825B
:109150008B83A3A3A3A3A3A3E0703D74016F600559
:1091600074016C703374018A828B83A3A3A3A3A3BD
:10917000A312B2F4E0C0E07403120A6DD0E012B2A0
:10918000EEE0C0E07404120A6DD0E0F07405120A3B
:109190006DEE129D6612196574060299E1EA240BC0
:1091A000F582EB22C082C0837901121A3D029DA88C
:1091B000C082C083EA7001EB60189004ADE06402E5
:1091C0007010E4901440F0EAFCEBFD7A0212986D06
:1091D00080127401901440F07A027B00900400E049
:1091E000F9121293029DA8C082C0839014BCE0754E
:1091F000F005A4FCADF079007A1F7B1412116D7B91
:1092000000800CEB12936374FEF0A374FFF00B90DC
:1092100014BCE0FAEBC39A40EA029DA8C082C08366
:109220007B007A0080037B010A9014BCE0FCEAC357
:109230009C5055EA75F005A4F8ACF0ECF9E81293EF
:109240007E7004A3E064FF60DFEA129372E82403F7
:10925000080808E912929124FFF0A3E034FF12A954
:10926000AE7002A3E070BFEA75F005A4F8ECF9E86F
:109270001293768882898374FEF0A374FFF0E488E9
:10928000828983A3A3F080A0EB6003129867029DFC
:10929000A8129D612274F6120356EAFEEBFF9014A9
:1092A000BCE0700302935E8E828F83A3A3A3A3A36B
:1092B000A3A3A3A3129FD06402600F8E828F83A307
:1092C000A3A3A3A3E0700302935E7C0080010C9033
:1092D00014BCE0FAECC39A5034EE240B1298C91275
:1092E000B0BAEC129363E0687003A3E06970DFEE3C
:1092F000241212B5B2FBEC75F005A42421F582E529
:10930000F03414F583E06B70C5790080537C0080E5
:10931000010CECC39A50F2EC75F005A4A9F012937D
:109320007E7004A3E064FF70E8EC129372EE240BED
:109330001298C9129F13EAF0A3EB12938B888289CB
:1093400083A3129CE9740C12A0237A08FB900400FA
:10935000E0F9121299EA7001EB7003129867790133
:1093600002984775F005A4241FF582E5F03414F542
:10937000832275F005A4241FF8E93414F922241F70
:10938000F582E93414F583E064FE22F0EE24121233
:10939000A9812274F212035674F31208AFEAFEEBAD
:1093A000FF8E828F83A3A3A3A3A3A3A3A3A3A3E05E
:1093B000F50A901440E0700579BA029678750801B4
:1093C000750900750C00750D007C087D007900851D
:1093D0001082851183AA82AB8312116D7405120A63
:1093E0006D7401129684540460127402120A6DE0C6
:1093F000D2E612968454087003750803E054106096
:109400000674404508F508E0540860227402120A08
:109410006DE044C01296845420600A7403120A6DF1
:10942000E0D2E080087403120A6DE0D2E1F08E828F
:109430008F83A3A3A3A3A3A3A3A3E07018120D4734
:1094400085108285118312A06C7402120A6DE0D21D
:10945000E2F00294F8640F70137402120A6DE0D205
:10946000E3F012A00A4508F5080294F88E828F8373
:10947000A3A3A3A3A3A3A3A3E064028E828F8370FC
:1094800005129D1780CBA3A3A3A3A3A3A3A3E0646A
:10949000037013851082851183AC82AD83EEFAEFE1
:1094A000FB1219F580528E828F83A3A3A3A3A3A3DB
:1094B000A3A3E0640170419004B1E0601C74021247
:1094C0000A6DE0D2E312A2D785108285118312A023
:1094D00036750910750AFF80187402120A6DE0448F
:1094E0000C12B45A74FDF0A374FFF074044508F52F
:1094F000088E828F831298A8EE241512B5B2A2E0CE
:1095000050257402120A6DE0540C701B8E828F83FA
:1095100012A8701214C1E9700579BB029678740222
:10952000120A6DE0D2E5F0EE241112B5B2C0E0747B
:1095300004120A6DD0E0129D2A120A6DE060030247
:1095400096717408120A6D12B0AF1298F1E912A563
:10955000DBA3E509F0EE241812B5B2C0E0E812B5BD
:10956000A5E91298CCD0E0F0EE241912B5B2C0E013
:109570007408120A6D12AF2FD0E0129D486401707A
:10958000149004B1E0C0E07408120A6DE0241512D2
:10959000992BD0E0F07408120A6D12A23A2417FA3F
:1095A000EF3400FB8A828B83E0FCE8241CF582E91F
:1095B0001298CCECF0A3E412A36CE0C0E0E8242203
:1095C000F582E91298CCD0E0F07408120A6D129678
:1095D0007DE50AF07408120A6D12B0AF2424F582FA
:1095E000E91298CCE50CF0A3E50D12AF58FCA3E00E
:1095F000FDE82426F582E91298CCECF0A3ED12B533
:10960000B9FCA3E0FDE82428F582E91298CC12B059
:10961000C2C0E0E8242FF582E91298CCD0E0F0EE49
:10962000241B12B5B2C0E07408120A6D12B42FD018
:10963000E0F0EE241A12B5B2C0E07408120A6DE030
:10964000242E12992BD0E012B45212A2941207EBDE
:10965000EE24111298C912A014740B120A6D12A2F2
:109660003F12081D851082851183AA82AB831219CF
:109670007D740C120A6DE0F9740D029878E02423D1
:1096800012994522F0EE241512A9812274F71203D3
:10969000567E638A828B83E0600C7905120A8FE91B
:1096A000FA7456C39AFE900459E0F9120A8FE9FA47
:1096B000EEC39A24F2F90299E474F612035674FE8A
:1096C0001208AF85108285118312A06CECFAEDFBB5
:1096D000740C120A6DE0FC900432E07002A3E060AA
:1096E0002F85108285118385820885830978081269
:1096F00007EF7D01900432129FBB121A8A74021286
:10970000081DEA7001EB60047900800679B28002DE
:1097100079B602984274F71203567409120A6DE082
:10972000FE90040BE07002A3E06018EEF5087808E4
:109730001207F390040B129FBB121A8A74011208CD
:109740001D800279B60299E474F512035674F8127A
:1097500008AF8A088B09ECFEEDFF750A011297B479
:10976000129887700D90046112ABEAE8F0A3E9F05B
:10977000803B851082851183AA82AB83120D5385AD
:109780001082851183AC82AD83AA08AB0912988739
:10979000700D120D4D8E828F83EAF0A3EB80D0EE18
:1097A000FCEFFDAA08AB09120ACBE9F50AA90A7475
:1097B00008029D871297B822120D41EAFCEBFDAA20
:1097C00008AB092274F6120356EAFEEBFF7A0C7B13
:1097D000001211F1EA7001EB6066EE242012B5B2BE
:1097E0008A828B83F0EE242112984CF0EE24221210
:1097F000984CA3F0EE242312984CA3A312A7B31203
:10980000985512988E24281298C9129855A3A3E847
:10981000F0A3E912A7BB8A828B83A3A3A3A3A3A36C
:10982000A3A3F0EE242F12B5B2C0E012919D1298BE
:10983000CCD0E012A03A8A828B83A3A3A312A030DB
:109840008005740212081D7F0202056312A9818A35
:10985000828B83A32212B0BE8A828B838004A3A34F
:10986000A3A3A3A3A3A3227CF47D017A087B009089
:109870000400E0F912128D2212081D7F0602056312
:109880003400FB1218C9221218C3E9640122129F86
:10989000DBEE2212989722F0850882850983E02268
:1098A000F508EF3400F50922E0F50CA3E0F50D22F0
:1098B00012A370A3E02228F582E439F583E0221296
:1098C000A5E8A3A3F022EE240CF582EF12A9A922A9
:1098D000FEA3E0FF22129FDBEE241212A9A622248F
:1098E00006FAEF3400FB22F582EB12A9A97401F00D
:1098F00022240FF58222F582ED12A9A9E4F022F5C7
:109900008312A018EC22850882F58322E0F81299D0
:109910001222A312B600A322C082C08312B5CFEBDD
:109920001298F9029DA879010207CF1299452212D7
:109930009935A3A322E0FAA3E0F5838A8222129D3F
:109940007222E0242BF812994A22A3E012995022A5
:109950003400F902A0AFE0240E12995D22F81299AA
:109960004AE022C082C083EA240C1298E7029DA834
:10997000029926C082C08390041974E3F0A374197D
:10998000F090041B74D7F0A37419F090041D74B305
:10999000F0A37419F090041F74DDF0A37419F002A1
:1099A0009DA874F7120356EAFEEBFF8E828F831296
:1099B0009C79A2E550298E828F8312A87090041999
:1099C000129FBB121A8A8E828F831299E9A3E070CC
:1099D00002A3E0700A8E828F83129C7BC2E5F08026
:1099E0000312081D7F01020563128DE7029861745E
:1099F000F5120356129B4A12B0AF2420F582E912E9
:109A0000B5B5FE74035EFF129F0C1298CC12A23AF9
:109A100088828983F0A3A882A983EF600874026F0B
:109A20006003029AB9740C5EF50A60167408650A40
:109A300060107404650A701C74026F7005EEA2E475
:109A4000402D8A828B83A3A3A3A3A3A3A3A3E02473
:109A500023129B98740C650A7010129B45242412E3
:109A60009B802424129B55129B9B74026F7005EE01
:109A7000A2E44045129B452426129B802426129B7B
:109A80005AA3129BB1129B5A129BB1129B55129B67
:109A90009BE50A60127408650A600C740C650A6024
:109AA000067404650A70128A828B83A3A3A3A3A3FE
:109AB000A3A3A3E02422129B988A828B83A3A3A34F
:109AC000A3A3A3A3A3129B677005EEA2E150198A7A
:109AD000828B83A3A3A3A3A3A3A3A3E0242E12AFEB
:109AE0001A88828983F0800E900401129B91900461
:109AF00001E00412A9B3A3A882A983EEA2E7504211
:109B0000129B452421129B5A129B9B8C828D83129F
:109B10009B67602E8A828B83A3A3A3A3A3A3A3A383
:109B2000E02430129B98EEA2E150178A828B83A327
:109B3000A3A3A3A3A3A3A3E02431129B70888289CB
:109B400083F0029D8A129B4AE022EA2408FCEB344F
:109B500000FD02B2D5129B9FA322129B5E22F50844
:109B6000A3E03400029906E0242112AF1E54032220
:109B7000129B75E022FAA3E03400FB8A828B8322D9
:109B8000129B5E129B91A3A882A9838C828D83E095
:109B900022E088828983F022129B9F129BA92212C5
:109BA0009BA322129D8F02B2D5129B91A308A98379
:109BB00022129BA98C828D83E024282274F7120341
:109BC000568A828B83129C79FC74035CFD74018A33
:109BD000828B83A3A3F0ED600574026D7061740C39
:109BE0005CFE601474086E600F74046E701374026F
:109BF0006D7005ECA2E4401D74028A828B83A3A3DE
:109C0000F0740C6E700A8A828B83A3A3E02402F0A6
:109C100074026D7005ECA2E440258A828B83A3A3B5
:109C2000E02404F0EE600F74086E600A740C6E603D
:109C30000574046E70098A828B83A3A3E004F0ECA0
:109C4000A2E750298A828B83A3A3E00412B0C61234
:109C50009033540360178A828B83A3A3E004F0EC53
:109C6000A2E150098A828B83A3A3E004F08A828B4D
:109C700083A3A3E004F00299E4E0F8129912A3E0B0
:109C800022C082C0838A828B83A3A3A3A3A3A3A39E
:109C9000A3A3A3E07002A3E060118A828B83A3A335
:109CA000A3A3A3A3A3A3A3A3129CAE029DA812A245
:109CB0004E1211F72274F7120356EAFEEBFF8E8262
:109CC0008F8312A366E4F0129CE9A3A3A3A3A3A32A
:109CD000A3F0A3F0E812B5D0E91298F912199BEE9F
:109CE000FAEFFB1219A70299E4A3129CEE22F08866
:109CF000828983A3A3A322E50C2410F582E50D122B
:109D0000A9A9E0FC7D002212A24EEA22F812995E77
:109D10002212995D0298A9129D1B22129FE1E8F080
:109D2000A3E922F5838882227401129D6A129D3173
:109D300022121983740C2212A28C22A3A3A3A3E8DB
:109D4000F0A3E9F0120D412212A7A8A3A3E022126A
:109D50009D56F8A3E022EAF0A3EBF088828983E025
:109D600022129950E022129D6A2212B45EAA82AB9E
:109D70008322129D77E022E0F8A3E0F5838882A396
:109D80002212116174032212081D7F03020563FC75
:109D9000A3E03400FD22F509750A00780822129D1F
:109DA000A222E012B5FEE022D083D0820207CF02C9
:109DB00007CF74F612035674FA1208AFEAFEEBFFEF
:109DC0007403120A6D12B2E87403120A6DAA82AB10
:109DD0008312198F12B5AF6003029F07743285108A
:109DE00082851183F07405120A6D12A5E2FAE02A49
:109DF000C0E07401120A6DD0E0129F31C0E074021D
:109E0000120A6DD0E01298B07002A3E060308E822A
:109E10008F83A3A3A3A3A3A3A3A312B0AD2417F579
:109E200082E912B5B5C0E0E82416F582E91298CCB3
:109E3000D0E0FAE02AFA7401120A6DE02AF08510E7
:109E400082851183AA82AB83120BA98A088B09A889
:109E500008A909E87001E97003029EFA8E828F83D7
:109E6000129F13A3A3129F198E828F83A3A3E0C016
:109E7000E0E82420F582E91298CCD0E0129F2CC0B3
:109E8000E0E82421F582E91298CCD0E0129F27C0A7
:109E9000E0E8242AF582E91298CCD0E0F0740512AB
:109EA0000A6DE0FA129F0C12A78812A5ECE8242B89
:109EB00012A0667405120A6DE0C0E0E8242DF58258
:109EC000E91298CCD0E01298B07002A3E06019E8D3
:109ED000242BFAE912892DA3A3A3A3A3A3A3A3E090
:109EE0002416129B9F12B5E98E828F83A3A3A3A38E
:109EF000A3A3A3A3E8F0A3E9800CEEFAEFFB1219E9
:109F0000951298C67410F07406029844E8240BF574
:109F100082E92212A24E02A0AFEAF0A3EBF0E824FD
:109F200012F582E90298EA129F37E02212B0DCE0D3
:109F300022129F37A3E02212B0E0A32274F712038B
:109F400056129F747002A3E06006129FB4121A8A20
:109F500012B5AF70158E828F83A3A3A3A3A3A31200
:109F6000A86E120BA31298C6E9F0EEFAEFFB1219D5
:109F7000950299E4EAFEEBFF1219A18E828F83A36A
:109F8000A3A3A3A3A3A302903B74F6120356EAFE75
:109F9000EBFF8C088D091214C1E97004790180115E
:109FA000AC08AD09EEFAEFFB90041F129FBB121A2A
:109FB0008A029847EEFAEFFB90041BE0F8A312B672
:109FC000002212A7A8E022129FCB2212B45EE02248
:109FD00012A24E120DA7E922129FE1E8F0A3E9F0C8
:109FE00022E0F8A3E0F985108285118322129FF107
:109FF00022E08E828F8302985EF085088285098335
:10A00000029862129FF9A3A3A3228E828F83129FCC
:10A01000D874042212A01822E0FCA3E0FD22F8A3C9
:10A02000E0F922F0A3E4F022F8A3E0F98E828F8316
:10A03000A3A3A3A3A3A3129FDB2212A03E2212A2DA
:10A04000EAA3A312A2E222C082C08312A05874899C
:10A05000F0A37419F0029DA81219AD90042122FA00
:10A06000A3E0FBE82428F582E912A9A9EAF0A3EB12
:10A07000F022C082C083E9FC12B5CFEB12B5B570F7
:10A0800002A3E0601712A09FA3E05403700EECFB44
:10A09000129F0C1298CC12A0DF12A0D9029DA8EA40
:10A0A000240CF582EB12A9A912A0AC2212A2E2881C
:10A0B00082898322C082C083EAF8EBF9888289838F
:10A0C000A3A3A3A3A3E0FB88828983A3A3A3A312D2
:10A0D000A0DFA312A0D9029DA8E0F912110722E087
:10A0E000FA88828983A3A32274F012035674FD12A6
:10A0F00008AF7401120A6D12AC2A8A0C8B0D74150C
:10A10000120A6DE0F50EA3E0F50F12B5D5EB12B50E
:10A11000B5242CFA12A2AC7001EF700302A21B74DA
:10A12000018E828F83F0850C08850D09750A0078F1
:10A13000081207EB7C157D00EE241712A22C1208E2
:10A140001D7401120A6D12B6481207EB7C097D00DE
:10A15000EE240212A22C12081D7413120A6D12A210
:10A160003A240B12AC04E0C0E0EE240F1298C9D0E0
:10A17000E012A254E0C0E0EE24111298C9D0E0121F
:10A18000A25DE0C0E0EE24101298C9D0E0129FC793
:10A19000C0E0EE24121298C9D0E0F0EE242512A2FD
:10A1A000247417120A6D7808120A2EEE241312ACCA
:10A1B0001812A27312A238240D12A21E12A26660F7
:10A1C00024EE242512A5D3242CF8EF3400F98A823A
:10A1D0008B8312A27A1207EB129CF78A828B83126E
:10A1E000A24212081DEE241812B5B2540360229048
:10A1F0000417E07002A3E0600FEEFAEFFB90041783
:10A20000129FBB121A8A8013EEFAEFFB12118B8099
:10A210000AEEFAEFFB90040012A2B302AEF512A907
:10A22000A6029D1E12A9A6E4F0A3F022FAEF12A244
:10A2300032223400FB029D81A3A312B0BEEE221293
:10A24000994212A24E029D81A3A3A3A3A3A3E0FA65
:10A25000A3E0FB2212A2582212A25DA322F0850ED7
:10A2600082850F83A322F0E50C2410F582E50D1200
:10A27000A9842212A2A5A3A3A322129FDBE50C248A
:10A280000EF582E50D12A9A912A28C22E0F508A311
:10A29000E0029D9612A28D2212A29DE022F0850C72
:10A2A00082850D832212A2C3A3A3A3227B0012AB3B
:10A2B000C6EE22E0F91211912212A2BD2212A2983A
:10A2C00002A01E12B652A3227B001211858A0A8BAD
:10A2D0000BAE0AAF0BEE2212A2DB2212A2EA12A2EE
:10A2E000E222E002A01E12A2EA22F08E828F8322D6
:10A2F000C082C083E9901442F09004137441F0A32B
:10A300007419F0900415740DF0A3741AF0900417EA
:10A3100074CBF0A37419F0029DA874F7120356EAE7
:10A32000FEEBFF8908EE7001EF70031214FD90043C
:10A3300023E07002A3E0900423601812A366A3E058
:10A340007002A3E088828983A3A3A3A3A3A3A3A3EA
:10A35000A370E8EEF0A3EF12A36CE4F0A312A7A49D
:10A36000E508F00299E412A0AC02985E12A37022F4
:10A3700012A7ACA3A3A32274F7120356E9FD90041D
:10A3800023800D88828983A3A3A3A3A3A3A3A3A34C
:10A3900012B0AF7001E9603488828983A3A3A3A3BC
:10A3A000A3A3A3E06D70DC88828983A3A3A3A3E0A9
:10A3B0006A7003A3E06B70CB88828983A3A3A3A3F5
:10A3C000A3A3E06C70BDE8FAE9FB80047A007B008F
:10A3D0000299E474F712035690042312B59F900477
:10A3E00023129023687002EB69701A129FBEA3A318
:10A3F000A312B0B490042312A03690042312B59F88
:10A40000803012B592EE7001EF60278E828F83A3A9
:10A41000A3A3A3A312901F687002EB6970E48A8261
:10A420008B83A3A3A3A3A3A3A3A3A312A43CA312BC
:10A43000A0301211F7EEFAEFFB0299E412ABEEA393
:10A44000A32274F212035674FE1208AF8A0C8B0D0D
:10A450008A828B83129FD06005790202A5CE12B248
:10A46000B6E50D12B5B5243012A5EC1211F18A082B
:10A470008B09AE08AF09EE7001EF700302A5CC7C2A
:10A48000307D00790012116D7901EEFAEFFB12199F
:10A4900053850C08850D09750A0078081207EB7CB6
:10A4A0001C7D00EE240B12A22C12081DEE242E128D
:10A4B000A5D324300808EF3400F98A828B8312A0D8
:10A4C00036E50C2411F8E50D3400F9E8FCE9FD8CC3
:10A4D000828D8312A23A242C1298C912A036E50C60
:10A4E00012B2ABE50D1298CC12B6481207EB8C8273
:10A4F0008D8312A0148A828B8312A24212081D85BA
:10A500000C82850D8312ABEA12A03290040112A5D1
:10A51000E2A3A3A3F0900401E00412A9B7EE242A59
:10A5200012A9551209888A828B83E508F0EE242946
:10A5300012A5D8E4851082851183F0E50C2415F569
:10A5400082E50D12B5B5A2E074015007120A6D74D0
:10A55000018004120A6DE4F0EE24271298A0851001
:10A5600082851183AA82AB83121131E924FE85080A
:10A5700082850983F0F508EE242CF582EF34001271
:10A5800098FFF8EDF9AA087B0012020DE88E828F81
:10A5900083A3A3A3A3A3A3A3A3F0ECF8EDF9AA08B4
:10A5A0007B0012020DEA7001EB600F8E828F83A395
:10A5B000A3A3A3A3A3A3A3E004F0EE242012B5B2A7
:10A5C0004408F0A3E012A9C979008002791074024E
:10A5D00002987812A965EE22F582EF12A9A9E50882
:10A5E000F02212A5E8029862E002A2EBFAA3E0349E
:10A5F00000FB2274F3120356EAFEEBFF12A9BD1210
:10A60000A99EE0C0E09014ADE0FAD0E0C39A400308
:10A6100002A77512AEFF7015EE242B12B5B204120C
:10A62000A7BBC0E0EE24291298C9D0E0F07A0080E0
:10A63000010A9014B2E0FBEAC39B50307508017523
:10A640000900EA780812098812AEFF550860E2EEA8
:10A65000242812A785F50C750801750900EA780809
:10A66000120988EE242912B5B24508F0EE2427120B
:10A67000A78DEE242C1298C9850C08EA8508F0A451
:10A68000F8ABF0E42BF9E098F8A3E099F98A08C355
:10A69000E89508E99400EE4043242712B5B2F81279
:10A6A000AEFF60409014B3E0FAA3E0FB8E828F838C
:10A6B000A3A312A06CE50C704AEE242012B5B2449C
:10A6C00020F0A3E0129D48C0E0EE24261298C9D0E5
:10A6D000E0F0EE242E12A78DA3E0804F24291298DB
:10A6E000C974FFF0900451E0F5089014B0E08508BB
:10A6F000F0A4ABF075F064A4FAACF075F064EBA4D0
:10A700002C80A8EE242012B5B254DFF0A3E012A7EB
:10A71000B3E50CF0F508EE2427F582EF12ABD2FA80
:10A72000ABF0EE242EF582EF12A79BFBEE241E1257
:10A7300098C9EAF0A3EB12A7A4A3E0C0E0EE242599
:10A740001298C9D0E0F0EE241C1298C9E812A02398
:10A75000900425E07002A3E0600EA90C900425127D
:10A760009FBB121A8AE97018EE240BFAEF3400FB33
:10A77000121A19800B7BE9EE2422F582EF12A98AC6
:10A780007F05020563F582EF12A9842A22F582EF84
:10A7900012A794223400F583E0FA2212A9842AFA3F
:10A7A000A3E03B2212A7A82212A7AC2212B0E4A376
:10A7B000A3A322F0EE242612A9A622F0EE242A1248
:10A7C000A9812274F412035690042312B59F121229
:10A7D000A58A0A8B0B7CFF7DFF8020E0C398FAA33B
:10A7E000E099FBC3EA9CEB9D500E8E828F83A3A35E
:10A7F000E0C398FCA3E099FD12B592EE7001EF6002
:10A80000528E828F8312B0BAE50AC398F8E50B998D
:10A81000F912A86AC3E89AE99B8E828F83A3A340AA
:10A82000BAA3A3A3A3E06402701DEE240B12AF022F
:10A83000600CEE240F1298C912A87012118BEEFA58
:10A84000EFFB1219478007EEFAEFFB12193B12A932
:10A85000CE801474FF6C700374FF6D600A7A017B04
:10A86000009014421298720289868E828F83A3A36D
:10A8700012A24E2274F21203568A088B09ECFAEDEA
:10A88000FB890A7C01E50812B2B8E50912B5B5F9F1
:10A8900012194D8A0C8B0DAE0CAF0DEE7001EF70DE
:10A8A0000302A949E50A600302A94912A96F12A986
:10A8B000786A600302A94912B2A9E50912AF498E6C
:10A8C000828F83A3A3A3A3A3A3A3A3E0FAE89AE997
:10A8D0009400C365D033401412A94C12AF05700C1C
:10A8E0007B0012B5A3E50912A98A805D12A94C125A
:10A8F000AF057023EE242912A9551209888A828B8C
:10A9000083E508F0EE242A12A5D89014B212A97893
:10A910002A12A99EE48022E5082414F8E5093400EF
:10A92000F9E0C0E0EE242A1298C9D0E012A9AEC026
:10A93000E0EE24291298C9D0E012A9B79014B312FE
:10A94000A43CE8F0A3E912A9C902987BE508241405
:10A95000F582E5092212A9657508FF7509009014B2
:10A96000B2E0780822F8EF3400F9E8FAE9FB2212A5
:10A97000B2A9E50912A9A922E0FAEE242812A981B8
:10A9800022F582EF3400F583E02212A794EE24141E
:10A9900012A9A612A0D9EEFAEFFB12194722F0EE87
:10A9A000242B12A9A622F582EF3400F5832212A9E6
:10A9B000B3E022F002A0AFF012A9BDF0221212A55E
:10A9C0008E828F83EAF0A3EB22F012A9CE227A01C5
:10A9D0007B00901442E0F91211B52274F012035674
:10A9E00074FD1208AF7401120A6D12AC2A8A0E8B24
:10A9F0000F8A828B83A3A3E0F91211258A088B09A1
:10AA0000AE08AF09EE7001EF70077A007B0002AB71
:10AA1000C37A117B001211F18A0C8B0DEA7001EBE5
:10AA2000700302ABBF7C117D00790012116D7902B9
:10AA3000AA0CAB0D1219537401120A6D129FBB12AE
:10AA4000ABF412A032E50E12B2B8E50F1298CC1298
:10AA5000ABDFA3A3A3A3F07508FF7509009014B2A0
:10AA6000E07808120988E50C12B5D0E50D1298CCF3
:10AA700012AC11129FBCE0C0E0E50C240BF582E59E
:10AA80000D1298CCD0E0F0E50E12B5D6E50F12B558
:10AA9000B5F508E50C12B2B1E50D12A5DBE50E1215
:10AAA000B2ABE50F12ABD2F8A9F0742328FAE4395F
:10AAB000FB12ABC6E50C1298F1E50D1298CC12B260
:10AAC000E8EE7001EF700302ABB2741A8E828F83CE
:10AAD000F0E412ABFAA3F0A312AC3812ABEA12A066
:10AAE000327401120A6D12ABDA1298DF121143852B
:10AAF0000E82850F83A3A3A3E0C0E0EE240F12987B
:10AB0000C9D0E012AC38A3A312A238241212AC04AC
:10AB1000A3A3E0C0E0EE24141298C9D0E0F0E50E43
:10AB200012B5D0E50F12B5B5C0E0EE24151298C9E4
:10AB3000D0E0F07413120A6D129D9EC0E0EE241650
:10AB40001298C9D0E0F07413120A6D12993EC0E059
:10AB5000EE24171298C9D0E0F07413120A6D129CFB
:10AB600079C0E0EE24181298C9D0E0129FC7C0E067
:10AB7000EE24191298C9D0E0F07415120A6D780805
:10AB8000120A2EEE241A12AC18F0EE2423F8EF3439
:10AB900000F9EE24211298C912A036E50E12B5A5CF
:10ABA000E50F12B5B5C0E0EE241E1298C9D0E0F052
:10ABB000800DAA0CAB0D121947750C00750D00AA7B
:10ABC0000CAB0D02AEF51211858A088B09AE08AFE9
:10ABD000092212A9848508F0A42212A018EE22E00E
:10ABE000850C82850D83A3A3A32212ABEE2212A2B1
:10ABF000E202A2EB12B0BE02A29EA312ABFF22128F
:10AC0000A2EAA32212A9A6129FDB850E82850F83DA
:10AC100022E50812ABFFE02212A9A6E508F0A3E5A1
:10AC200009F0A3E50AF0A3E50B22ECF0A3EDF0E9AF
:10AC3000851082851183F02212A25802986274F066
:10AC400012035674FB1208AF85108285118312A07F
:10AC50006C7403120A6D12B5F889097417120A6D23
:10AC6000780C120A2E7402120A6DE4129FC7241384
:10AC7000129D0CF508900425E07002A3E06011A974
:10AC800008900425129FBB121A8AE9600302AEF1F4
:10AC90007C027403120A6D12AF368510828511830F
:10ACA000E0241112B58D12194D8A0A8B0BAE0AAF32
:10ACB0000BEE7001EF705112AF23400302AEF1783A
:10ACC0000C1207E77419120A6D120653A9097409C8
:10ACD000120A6D12A0147406120A6D12A8701219CD
:10ACE000E9740612081D8A0A8B0BAE0AAF0BEE70D0
:10ACF00001EF700302AEF18E828F83A3A3A3A3A3FF
:10AD0000A3A3A3E50812A9C985080A8E828F83A38D
:10AD1000A3A3A3A3A3A3A3E0F874FF281874FF348C
:10AD200000F9E8650A7001E970087402120A6D748E
:10AD300001F0EE240B12AF02700302AE9512AF23A6
:10AD4000500375080085080A12AF43E50A98E49994
:10AD5000C365D033401EE0FAEE240E12A785F075CD
:10AD60000AFF750B009014B2E0780A120988129855
:10AD7000C6E50AF0851082851183E0240E129D112C
:10AD8000750E00780C1207EB7403120A6D12AF3CBB
:10AD9000FC7D0085080AEE240D12B5B2850AF0A4E8
:10ADA000F8A9F0EE240F12B5B22421129B7028FAF4
:10ADB000A3E039FB129D8112081D750A0112AF0B29
:10ADC000780A12098812B5AF450AF07402120A6DAA
:10ADD000E0606FEE240C12A965750AFF12AF0B0438
:10ADE000780A1209888A828B83E0450A12AF588557
:10ADF000080A850AF0A4F8A9F0851082851183E07D
:10AE0000241012AF1A28FCE439FDEE240F12B5B25B
:10AE1000241F12992B12B0C264FF7026EE240BF58A
:10AE20000AEF3400F50BEE240F1298C912A87085B2
:10AE30000A82850B8312A2B374FF850A82850B8375
:10AE400080521212A58E828F8312A06C900451E062
:10AE5000F50A9014B0E0850AF0A4FAABF0F8EBF92B
:10AE60009014ADE0F50AE8850AF0A4F8ACF0850A84
:10AE7000F0E9A42CF9E82AF8E93BF9E875F064A4B4
:10AE8000F8AAF075F064E9A42AF98E828F83A3A34F
:10AE9000E8F0A3E9F012AF4374FF281874FF39F902
:10AEA000E865087001E96010EE240C12AF0260083A
:10AEB0007402120A6DE06039EE240E12B5B2C0E0E1
:10AEC00085108285118312AF2FD0E0F012B5AFC08C
:10AED000E0851082851183E0241412992BD0E012B2
:10AEE0009FC7FCA3E0FD7403120A6D12AF36120A6D
:10AEF0007774058002740312081D7F08020563EE53
:10AF00002429F582EF12A98464FF22750B009014A6
:10AF1000B2E0F5F0E50884E5F02212AF1E22129BA4
:10AF2000A3E022851082851183129D72A2E022E0A7
:10AF3000241312994522129DA202A24FE02410125E
:10AF4000995D22EE240EF582EF12A984F89014B2D6
:10AF5000E028F8E43400F922F0EE240D12A9812251
:10AF6000C082C08390144212A2B3029DA874F4124E
:10AF70000356EAFEEBFF74805FF9E47001E9705656
:10AF8000EEA2E050631211D374016EFAEFFB805C05
:10AF90008A828B83E06401703612AFEF12064F1283
:10AFA00088711207EF12B0031219D1740612081D2E
:10AFB000E5082425F582E50912B5B57002A3E06025
:10AFC0000EE5082425F582E5091298CC129CAEAA5C
:10AFD00008AB0912118B90144212AFF87001EB709C
:10AFE000AFEEFA74806F80A57A007B00028986EA52
:10AFF00012B2ABEB12A9A922E0F91211978A088BC1
:10B0000009EA22EA2412F582EB12A984F9EA240261
:10B01000FCEB3400FDEA2417FAEB3400FB2274F752
:10B0200012035690042780048C828D83129901703C
:10B0300001ED60298C828D83A3A3E069600574FF14
:10B040006970E58C828D83A3A3A3E06A7003A3E0FB
:10B050006B70D5EC2403FAED3400FB80047A007B9E
:10B06000000299E474F712035674FE6970047E01BD
:10B0700080027E00900427800AE06970027E018CC5
:10B08000828D831299017001ED601D8C828D83A3E6
:10B09000A3A3E06A7003A3E06B70E4EE8C828D835F
:10B0A000A3A360D5E0F9800279FE0299E4A3A3127C
:10B0B000B0BEE822A3A3A3A3A3A312B0BE2212A2F0
:10B0C000E222ECF0A3EDF08A828B83E022851082ED
:10B0D000851183E02401F0A3E034002212B0E022C5
:10B0E00012B0E422F08E828F83A3A3A32274F41201
:10B0F0000356E48C828D83A3A312B2DF12B2FDC08B
:10B10000E0EC12B5D6ED1298CCD0E0F0EA241DF5B3
:10B1100082EB1298CC12B0BAEC12B2B1ED1298CC0C
:10B12000E412B2DAF0A3F012B2B0EB1298CC12B281
:10B13000BDA3A3A3A3A3A3EEF0A3EF12A9AEFE8C1D
:10B14000828D8312B30874035EF50860097402658A
:10B1500008600302B1EE8C828D83E0540CF5086028
:10B160000F74086508600974046508600302B24F33
:10B1700088828983E08C828D83A312B31174086561
:10B1800008600302B24FEC12B5D0ED1298EA8A8241
:10B190008B83A3A3A312B42770128C828D83E04407
:10B1A0000C12B2EEA3A312B2BD12B2E8740265088B
:10B1B00070098C828D83E0A2E4403312B2C912B3CD
:10B1C0001812B2C9A3A312B318E508601274086577
:10B1D00008600C740C6508600674046508700F88BC
:10B1E000828983E08C828D83A3A3A312B308888213
:10B1F0008983E0C0E0EC12B2B8ED1298CCD0E01236
:10B20000B3088C828D83E0A2E7505C88828983E05A
:10B21000FE8C828D8312B31174035E604DE0C0E03A
:10B22000EC12B2ABED1298CCD0E012B3128C828D3E
:10B2300083E054036402703288828983E0C0E0ECCA
:10B240002414F582ED1298CCD0E012B312801BECDE
:10B25000240C1298F6740C6508600302B18E12B2C9
:10B26000C912B31A02B1BBE4A3F0EC12B5AAED12F5
:10B2700098CC12A036EC2410FEED3400FFEA241D19
:10B28000F582EB12B5B5F5088E828F83E0C3982561
:10B2900008F50812B2FDC39508C0E0EC12B2B1ED9A
:10B2A0001298CCD0E0F0028986E5082413F58222BA
:10B2B000EA240DF58222E50C2411F58222E0FEA39A
:10B2C000E0FF8C828D8302986288828983E0F50A90
:10B2D000A3E0FFE50A8C828D832212B2DFA322F065
:10B2E0008C828D83A3A3A322EEF0A3EFF02212B2EF
:10B2F000F4029862F08A828B83A3A3A322F0EA244B
:10B3000017F582EB12A9842212A9B3A3A882A983FC
:10B3100022A312A9B3029BACA3A3A3A3A3A3F0A34C
:10B32000EFF0E824020808E93400F92274F412036B
:10B330005674F31208AF8A0A8B0BECFEEDFF8E8277
:10B340008F83E0540CF508E0A2E75006E508D2E749
:10B35000F508E508D2E1F50812B4297006E508D22F
:10B36000E4F508E0A2E55006E508D2E5F5087C081A
:10B370007D007900851082851183AA82AB8312112A
:10B380006D7402120A6D12AC11C0E07403120A6DE2
:10B39000D0E012B45AE50AF0A3E50BF07405120AE6
:10B3A0006D129D28120A6DE070787408120A6DE023
:10B3B000241212992B740112B44CC0E07408120AC2
:10B3C0006D12B436D0E0129F2CC0E07408120A6DE2
:10B3D00012967DD0E0F07408120A6D12ABEA12B436
:10B3E0003D129D4812A05FEE241112B5B2C0E0E8F4
:10B3F000242EF582E91298CCD0E0F0EE241412B598
:10B40000B2C0E07408120A6DE0243112992BD0E02A
:10B4100012B452C0E07408120A6D12B42FD0E012B8
:10B42000B462740D028983A3A3E05403640122E093
:10B43000243012994522E024221299452212A24872
:10B44000E82426F582E912A9A902A9C412ABFFA338
:10B45000E022F0EE241312A9812212B45E22F0023F
:10B460009FE6129D6A12197D2274F71203567E0020
:10B470008A828B83A3A3A3A3A3A3A3A3A3E06402B1
:10B48000607312919D12B5B5706B12B5CFEB12B50A
:10B49000B57002A3E0605E12A09FE054037056A353
:10B4A000A3A3A3A312B4FAE06A7003A3E06B7045F0
:10B4B0008882898312B4FAA3A3E0FFA3E0F5838F07
:10B4C00082A3A3A3A3A3A3E06A7003A3E06B7025E8
:10B4D00088828983A3A3E0FA8C828D83A3A3129C24
:10B4E000796A60108C828D83A3A3129FBDE0540CF7
:10B4F000640470010EEEF90299E4A3A3A3A312A2BF
:10B500004E02B2D574F612035674FC1208AFEAFE6E
:10B51000EBFFECFAEDFB8A828B83A3E05403601B04
:10B52000900415E07002A3E0605E7900EEFCEFFD90
:10B53000900415129FBB121A8A804D8510828511C6
:10B540008312B2E87402120A6DEAF0A3EB12B45A45
:10B55000AC82AD837A7D7B0A120CF98A088B09A82C
:10B5600008A909E87001E9601F740688828983A32D
:10B57000A3A3A3A3A3A3A3A3F07A0088828983E053
:10B58000240C12B58D120C63740402984412995D58
:10B59000F9228E828F83A3A3A3A3A3A3A3A3A3E0D3
:10B5A0000298D0E5082412F58222240EF58222EEBC
:10B5B000240CF582EF12A98422F012B5BFE022EE2E
:10B5C0001298F1EF02A9A9F0EE240E12A98122EA45
:10B5D000240CF58222EA2410F5822212A018EEFA39
:10B5E000EFFB2212B0BE029FE6E0FC8A828B83E072
:10B5F0002C129D8F8A828B83ECF0A3EDF022F8A3AE
:10B60000E0029D23C082C083900429E07002A3E081
:10B61000600B900429129FBB121A8A8002790102E2
:10B620009DA8C082C08390042BE07002A3E0600B51
:10B6300090042B129FBB121A8A80027900029DA8E7
:10B6400012081D7F07020563E0F508A3E0F50978FD
:10B65000082212A29DA322F582EB12D2A4A2E2221A
:10B66000E0F508750900750A00750B0022740912CF
:10B67000081D7F0402056312D2A4A2E52212DD5048
:10B68000E822EE2412FAEF3400FB120FF9E92279D6
:10B6900005121005740222E0FAA3E0F9EA2274020E
:10B6A00012081D7F060205631210EF90056212DD7D
:10B6B000507A147B0022340002C953E024FFF8A31F
:10B6C000E034FFF922888289832212BF7612081D96
:10B6D00002B6FF12C0A3E4F022E08E828F8312B67E
:10B6E000E222F012B6E722EE24FF1EEF34FFFF2223
:10B6F000A3A3E0FCA3E0FD22EEFAEFFB1210DD7F36
:10B70000080205637AEB7B041211A9740222A2AF2E
:10B71000E492E0FAC2AF9004F2E004F0EAA2E09210
:10B72000AF22AA82AB831218C98E828F83A3A31281
:10B73000BD26E02212081D02C1D5EE240EF582EFCF
:10B7400012C0A322EE240DF582EF12D2A4640122CE
:10B75000E0FEA3E0FFEE227F07020563FAEF34006C
:10B76000FB79E11210832212B76B2212C2D6A3A377
:10B77000A3A3A322EE2412FCEF3400FD22C082C05A
:10B7800083800A7AEB7B041211A312118B9004EBD5
:10B79000E07002A3E070EC9004EDE07002A3E060C2
:10B7A0000C7AED7B041211A312118B80EA9004EB4A
:10B7B000E4F0A3F09004F1F09004F2F09004F38030
:10B7C00003F0A3E0F002BE4D74F41203568908E9B9
:10B7D00024EFF582E4341DF583E493FEFA7B001236
:10B7E0001185EA7001EB600F12D08EE48A828B83A0
:10B7F000A3A3A3A3F080297A027B00121185EA702B
:10B8000001EB6018E50824CEF582E4341DF583E4ED
:10B81000938A828B83F0741AA312BB4B7A007B004D
:10B8200002B672C008740629FBEAA2E0501EEB754E
:10B83000F00A84AAF0EA6014740A2BC39AFBEAC3E4
:10B8400094054004740A2BFB740B2BFBE9C394137F
:10B850004004781480027806E82BFB8B08740925D5
:10B8600008F8E43400F97A0A7B00120205E8F9D0FE
:10B87000080207CFC082C08390050FE05402600A1F
:10B8800012191DE9600479018002790002BE4DC0E1
:10B8900082C08390050FE0540260199004F1E070BB
:10B8A0000F9004F4E07002A3E0600912B8B95004EC
:10B8B00079018002790002BE4D9004F4E024101258
:10B8C000BD3EA2E722C082C0839004F3E0C0E090B6
:10B8D000874EE0FCD0E0C39C500512118580047AAD
:10B8E000007B0002BE4DC082C08312118B02BE4D90
:10B8F00074F6120356EAFEEBFF8E828F83A3A3A396
:10B90000A3A3E01205E80003E5B912B964B9E5B9EB
:10B9100075B9900542E0640F6013120FC3E9700D12
:10B92000EEFAEFFB90146B12BD22121A8A90056A90
:10B93000E08E828F83A3A3A3A3A3A3F074148E82AB
:10B940008F83F0EEFCEFFD7AED7B0412119DA2AF28
:10B95000E492E0FAC2AF9004F312B7197920120F03
:10B96000B102C4B3120FBDE96007740D12B9FA80B9
:10B97000F0741580C98E828F83A3A3A3A3E06065B2
:10B980008E828F83A3A3A3A314F0EE2402EF3400CE
:10B990000A0AFB8A828B8312B67DFCE9FD8C828DBC
:10B9A00083E0F508EE2405F8EF12B9EFE50812D6AA
:10B9B0005BA882A9838A828B8312D09EE5086025CA
:10B9C0008E828F83A3A3A3A3A3E0C3940A5016EE91
:10B9D000240512B9F3240A8E828F83F0888289832A
:10B9E000E00402B942EEFAEFFB12118B02B96112C8
:10B9F000CF1622F8EF12CF16E0228E828F8312BD6F
:10BA0000BA12191722C082C0839004F6E07002A314
:10BA1000E0600B9004F612BD22121A8A80027900AF
:10BA200002BE4D74F7120356EAFEEBFFEE240D1230
:10BA3000B73D7401F0EE242F12BA8CC0E012B73A71
:10BA4000D0E0F0EE243012BA8CC0E0EE241212B72F
:10BA50003DD0E012CF39C0E0EE241312B73DD0E064
:10BA6000F0EE242B12B73D120653EE2422FCEF34E5
:10BA700000FDEE242D12BA8CF912C07412081DE9D3
:10BA80007007EEFAEFFB120EF702C1D5F582EF1246
:10BA9000D2A422C082C083120FC3E960047920803F
:10BAA00002790102BE4DC082C083EA12CBC8E0D247
:10BAB000E002B7C4C082C08312CBC112B74A701172
:10BAC00012BB40400C8A828B83A3E0F9120FB7802F
:10BAD0006CEA12CBB0EB12BA8FA2E650128A828BBC
:10BAE00083A3E0F990146D12BD22121A8A804E12BF
:10BAF000CBC112B74A700912BB4050047430803673
:10BB00008A828B83A3E0641B7004742280288A825B
:10BB10008B83A3E0700F12CBC112BA8F24E4F5829D
:10BB2000E4341D800D12CBC112BA8F24CEF582E40D
:10BB3000341DF583E4938A828B8312BB4B02BE4D86
:10BB4000EA12CBB0EB12D2A4A2E322F090050CE0F3
:10BB5000F912119122C082C0839004F4E07002A314
:10BB6000E06043E9700612BC18E4801A741B697027
:10BB7000389004F4E0240DFAA3E012B6B6E06405B0
:10BB800070E412BC18E912BC21120EE59004F4E036
:10BB9000240E12B8BF500312D34E9004F4E4F0A365
:10BBA000F07910120FB102BE4D74E969704990042A
:10BBB000F412CF04E09004F46036E0240E18181854
:10BBC00012BC14A2E29004F4E0400F24110808080B
:10BBD00012BC1414F012187580CC240F0812BC1477
:10BBE000C2E712BC2190146912BD22121A8A809CED
:10BBF00012BC1B74E9808F741C6970869004F41267
:10BC0000C17C90147312BD22121A8A9004F4E4F0DD
:10BC1000A3F0809212BD3F229004F4E012BD27A34E
:10BC200022F09004F412C1802274F4120356750AB3
:10BC300000750B00A2AFE492E0FEC2AF9004F4E006
:10BC40007002A3E06008EEA2E092AF02BD02901481
:10BC50007112BD22121A8AE94410FA9004EB801284
:10BC600085080A85090BE50824FBF582E50934FF00
:10BC7000F58312BD15E5087002E50960C912BD0A19
:10BC80005A6A70DC780A1207EFAC08AD0912B704E3
:10BC900012081D9004F4E508F0A3E509F012B8B904
:10BCA00040639004F2E014F0EEA2E092AF9004F44E
:10BCB000E0240E1818A3E03400F9E8FEE9FF8E82B4
:10BCC0008F83E0FA12BD2FF9120EA9E99004EFF06C
:10BCD000A3E412CBDDE0A2E750189004F4E02412B4
:10BCE00012BD1D1217799004F4E0241312BD1D1229
:10BCF000176D9004F412BD37A2E1B3E492E0F9129B
:10BD0000185D02B6729004F1809BE50812CC90E5B4
:10BD10000912D2A422E0F508A3E0F5092212BD3EE3
:10BD2000F92212BD2622E0F8A3E0F5838882229052
:10BD300004F412C402E022E0240F12BD3E22F812E5
:10BD4000CF10E02274F7120356EAFEEBFF120FE762
:10BD5000EE12CBB0EF12BB45400A12B7447005900B
:10BD6000874C800390874DE0F9EEFCEFFD7AEB7B8A
:10BD7000041211AFE9602FEEFAEFFB90146F12BDC1
:10BD800022121A8AEE240EF582EF12B65A400812D9
:10BD9000B70E120EF18014EEFAEFFB90146712BD8D
:10BDA00022121A8A800574F112BDAE02C1D58E82AC
:10BDB0008F83A312BDBA120EE522F0EEFAEFFB223A
:10BDC000C082C083120EF102BE4D74F7120356EA10
:10BDD000FEEBFF75080090050FE05402700EEE2494
:10BDE0002FF582EF12B65A50037508E890050FE060
:10BDF0005460700DEE242F12BA8CA2E15003750826
:10BE0000E88E828F83A3A3A3A3E0C3947540037538
:10BE100008E8EE242D12BA8C701AEE242A12BA8C7D
:10BE200070127508F5120FE7A908EEFAEFFB120F72
:10BE3000B702C1D5E50870ED120ED380F4C082C000
:10BE400083740D8A828B83F01219178000D083D0FF
:10BE5000820207CFC082C083E48A828B83F0A3F082
:10BE6000EA242F12B65740189004F2E0C0E0908701
:10BE70004CE0FCD0E0C39C401879F1120FB780CDA4
:10BE80009004F1E0C0E090874CE0FCD0E0C39C500F
:10BE9000E812BB4C80E874F4120356E9FFEA240E62
:10BEA000F582E4341EF583E493244AFE8F0A250AC2
:10BEB000FAE43400FB121185EA7001EB600FEF8A9F
:10BEC000828B83A3A3A3A3F012D08E80047A007B7D
:10BED0000002B672C082C083E490050AF090050BA0
:10BEE000F09004FE12BEFB7402900500F09005076E
:10BEF00012BEFB740190050902B7C474B1F0A374BB
:10BF00000FF022C082C08374F11208AF7402851052
:10BF100082851183F07401120A6DE9F060047AFFE2
:10BF20007BFF7402120A6DEAF0A3EB12DB34740F8C
:10BF30008002741112081D02BE4DC082C08374FEBF
:10BF40001208AF740A851082851183F07401120AF9
:10BF50006D12DB33740280DC74F012035612D8BF0A
:10BF6000120A2E7808790C12026678081207E77A0E
:10BF7000017B0502B6CA1210E374042274F41203A2
:10BF80005674CE1208AF900542E0640F6007742E1D
:10BF900012C8DD80237AF87B0412B6A812020D883D
:10BFA000088909750A00750B0078081207E77AF806
:10BFB0007B0412BF7612081D743202B66F74F7123A
:10BFC0000356EAFEEBFF7A0012C08F6007E06403BD
:10BFD00060027AE8EE241712BA8CC3940B4028E072
:10BFE000C3941D5022EA7021EE241712B75CEE2490
:10BFF0002212C07A12C08F7026EE241912DD4690EC
:10C00000055112D09E802B7AE8EA8E828F83A3F0AE
:10C0100074178E828F83F0EEFA120FC902C1D59089
:10C02000055174FEF0A374FFF0EE241912C08512BE
:10C0300018C990050AE04401C0E012B73AD0E012F6
:10C04000C098740212CCF1242412CCDD242212B741
:10C050003D120653EE2419FCEF3400FD79831A1AC1
:10C0600012C07212081DE970B3EEFAEFFB120EF760
:10C0700080AAEFFB120FFF740222FAEF3400FB7963
:10C080005012108322FCEF3400FD7A487B0522EE2B
:10C09000242112D2A1640222F0EE240D12C0A022AB
:10C0A000F582EF3400F58322C082C08374F7120852
:10C0B000AF90050BE070327401F0F912182785106B
:10C0C00082851183AA82AB83120FED900557120669
:10C0D0005390050AE04401FB7402120A6DAC82AD74
:10C0E000837A0312B68F12081D740902BF3474F7E5
:10C0F00012035612C2BA700474EBA3F090050BE061
:10C10000A2E25003C2E2F0E0A2E1500512C2CB80ED
:10C1100005742A12D83502C1D574F712035674FE7D
:10C120001208AF12C1DA12C3EA8510828511831298
:10C13000C40CE0F5087017851082851183AA82ABC4
:10C14000837953121083EE2412FAEF12DA958510D8
:10C150008285118312C17CA908120F2190050BE082
:10C16000A2E1500A8E828F83A3E0F9120F27E49098
:10C17000050AF090050BF0740202B73412C1802258
:10C18000E0FAA3E0FB2274F7120356EAFEEBFF7419
:10C19000EB8E828F83A3F090050BE0A2E15005792E
:10C1A000EB120F27EEFAEFFB120F57802874F712ED
:10C1B000035612C1DAE490050AF090050BF07AFFFD
:10C1C0007BFF8E828F83A3E0F9120F218007EEFAA6
:10C1D000EFFB12104D7F01020563EAFEEBFF7901D0
:10C1E00012182D7AF87B041210EF7A017B051210D9
:10C1F000EF2274F7120356EAFEEBFF120F5180CEC6
:10C2000074F7120356EAFEEBFF790112182D8E82A5
:10C210008F83A3A3A3A3E060047A0080027AEB12C9
:10C22000C24B5003C2E2F0E0A2E1500512C2CB8043
:10C2300011A2E0500D742A8E828F83F074EBA3124A
:10C24000D839EEFAEFFB120F09808AEA8E828F83CB
:10C25000A3F090050BE0A2E22274F7120356EAFE67
:10C26000EBFF90050BE0D2E1F07901121827EE24E4
:10C270000B12B73D120653EE2402EF3400FF0E0EF0
:10C280007401C0E0120FF3E9FAD0E0FBEEFCEFFD21
:10C2900012B68F02B73474F712035612C2BA700482
:10C2A00074EBA3F090050BE0A2E25003C2E2F0E0D1
:10C2B000A2E1500312C2CB02C1D5EAFEEBFF790125
:10C2C00012182D8E828F83E0642022C2E112C2D622
:10C2D000E0F9120F2722F08E828F83A32274F712C7
:10C2E0000356EAFEEBFF790112182D7AF87B04124F
:10C2F000DC93E060047A0080027AEB12C24B5003B8
:10C30000C2E2F0E0A2E1500312C2CB02C24274F7D3
:10C31000120356EAFEEBFF790112182D74EB12C2DC
:10C320004C5003C2E2F0E0A2E1500312C2CB02C1C2
:10C33000D574F712035612C34702C1CE74F7120325
:10C340005612C34702C1D5EAFEEBFF7AF87B04120E
:10C3500010EFEEFAEFFB120F7B2274F71203567404
:10C36000EF1208AFEAFEEBFFEE241212C08512189E
:10C37000B7E9605C7409851082851183F07401123D
:10C380000A6D74EFF012C3EAF87402120A6DE81233
:10C39000C40CA3A3E0C0E07404120A6DD0E012CB79
:10C3A000DDA3A3A3A3E0640870158E828F83A3A3EB
:10C3B00012C3FBE0C0E07405120A6DD0E080067481
:10C3C00005120A6DE412CF417406120A6D12C3D52C
:10C3D000741102B734AA82AB8312101785108285BC
:10C3E0001183AA82AB831219172212CCFA12DD50E4
:10C3F00088828983E0FCA3E0F9EC2212C402A3A3A3
:10C40000A32212C4062212DC1DA3A322F0A3E91268
:10C41000CBBD12DC1922C082C08312105902BE4D5E
:10C42000C082C08390052C7413F0A3741DF0900596
:10C430002E74FAF0A3741DF09014777414F0A374A2
:10C440001BF09014797476F0A3741BF090051874A7
:10C450001BF0A3740FF090050FE0440102B7C1C0B8
:10C4600082C083EAFCEBFDEA241612D2C7790212DD
:10C470000FD502BE4DC082C083790602D36574F623
:10C4800012035690050DE07002A3E0600312C4B8D9
:10C4900090050DE4F0A3F0900511F0800312118BCC
:10C4A00090050CE0F9121197EA7001EB70EF800330
:10C4B00012081D7F0202056390050D12C180121142
:10C4C0008B2274F7120356E9FA7B0090050CE0F911
:10C4D0001211B502C1D574F412035674F11208AFEB
:10C4E0008A828B83E024D9F582E4341DF583E493BA
:10C4F000851082851183F0640B700DE98A828B832D
:10C50000A3F012103B02C5BCE0700302C5BC640C72
:10C51000600302C5B47403120A6D12C8D7EA242E50
:10C52000F582EB12BA8FC0E07402120A6DD0E012ED
:10C53000CF2BA3A3A3A37808120A2E7405120A6DA9
:10C5400012CF488A828B83A3A3A3A3A3A3A312B66B
:10C55000F07409120A6DECF0A3ED12CC0750047CC4
:10C56000008011EA2411F582EB12BA8FFC90056469
:10C57000E0C39CFC740B120A6DECF0EA2414F58203
:10C58000EB12BA8FC0E0740C120A6DD0E0F0EA240E
:10C5900015F582EB12BA8FC0E0740D120A6DD0E06F
:10C5A000F0EA2416F582EB12BA8FC0E0740E120A7C
:10C5B0006DD0E0F07401120A6D12DB33740F02B615
:10C5C0006FC082C083900511E07004790180027908
:10C5D0000002BE4DC082C083900511E06403700468
:10C5E00079018002790002BE4D74F612035690055F
:10C5F0001112C6802475F582E93414F58312C94EF0
:10C60000E0C2E7F0C333FCE82CF582E912B740A39F
:10C61000E493FEC333FCE433FDEC2475F582ED3482
:10C6200014F583E07002A3E06005EE900511F08A36
:10C63000828B83E0C333FCE433FDE82CF582E93DD3
:10C64000F583E493F508C4540FC3332426F582E43C
:10C650003405F58312B67D7001E97005121029804A
:10C660001C740F5508C333FCE82CF582E912C68C04
:10C6700093C0E0740193F583D082121A8A02C4B386
:10C68000E0C333F8E433F9E822F582EB12C0A3E407
:10C690002274F212035674FE1208AF890C8A088BBA
:10C6A0000912C748FA12C7677001EF60238E828FA4
:10C6B00083E50CF0E4A3F0F50A78081207EB12C743
:10C6C0005524020A0A12C77612081D12C6D6800324
:10C6D00012C78002B69EEEFAEFFB02BB4C74F0125A
:10C6E000035674FE1208AF890C8C088D0912C748D6
:10C6F000F50EEA60067405250EF50EAA0E12C76740
:10C700007001EF603B8E828F83E50CF0E4A3F0EEC6
:10C71000250EF8EF3400F98E828F8312D09CE48EC0
:10C72000828F83A3A3A3A3F0F50A78081207EB1264
:10C73000C7552417FA12C77612081D12C6D68003F1
:10C7400012C780740202B6CDE924B8F582E4341D24
:10C75000F583E49322E50C24C3F582E4341DF583CC
:10C76000E493FC7D00EE227B001211858A0A8B0B7C
:10C77000AE0AAF0BEE22EF3400FB121161740322FC
:10C78000851082851183E50CF0791AAA82AB831299
:10C790000FB722C082C083E990050C02B7C474F4BD
:10C7A00012035674FE1208AFEAFEEBFFEE5420703F
:10C7B000318040A2AFE492E0FAC2AF9004F3E014FB
:10C7C00012B71B8508828B8312C8C8AA08120FC92A
:10C7D000851082851183E064156007AA08AB0912F1
:10C7E000118B7AED7B041211A38A088B09EA700180
:10C7F000EB70C074805FF9E47001E9701D802DE476
:10C80000900517F090051512C8D7120FC99005179B
:10C81000E07007AA08AB0912118B90050CE0F91221
:10C8200011978A088B09EA7001EB70D3EE541060FF
:10C8300005742D12C8DDEEA2E05005742412C8DD87
:10C84000EE54026005742512C8DDEE5404600574D0
:10C850002612C8DDEE54086005742812C8DDEE54B7
:10C8600040600C7401120A6DE4F0742C12C8DDEE05
:10C870005480600C7401120A6DE4F0742F12C8DD4C
:10C8800090050DE07002A3E06035A2AFE492E0FAFB
:10C89000C2AF90050D12BD1590050DE4F0A312B7BF
:10C8A0001B900512E508F0A3E509F0E490051412C9
:10C8B000DA9E900514E07007AA08AB0912118B7A72
:10C8C000007B00740202B66FE0851082851183F050
:10C8D00022A3A3A3A3A3A3EAF0A3EBF022851082D3
:10C8E000851183F0AA82AB83120FC922C082C08354
:10C8F00090051512DE897002EB69700774019005CE
:10C9000017801190051212DE897002EB69700674AF
:10C9100001900514F002BE4DC082C083900551E025
:10C9200064FE7004A3E064FF70097C487D05121862
:10C93000BD801574028A828B83A3A3A3A3A3A3A3A0
:10C94000A3F012C94B12D09E02BE4D90055112DDCC
:10C95000508001FB8A828B8322C082C08390055B5A
:10C96000C3E094FEA3E094FF4004790380027902BF
:10C9700002BE4DC082C0838A828B83A3A3A3A3A3DC
:10C98000A3A3A3E06402701412C94BE0687003A370
:10C99000E06970047901800F7900800BEAFCEBFDFF
:10C9A0007A487B051218B702BE4D74F01203567414
:10C9B000FD1208AF7401120A6DECF0A3EDF08A0AC3
:10C9C0008B0B7508007401120A6D12CBD085108292
:10C9D000851183F0E9A2E75008750EFF750FFF80FF
:10C9E0000A900557E0F50EA3E0F50FE9C2E7F9EA72
:10C9F000240EF582EB12B677EA500B12CBB0EB1295
:10CA0000B74074088005240F12C68912CBEDA2E24C
:10CA1000EA500712CBC87480800512CBC87410127C
:10CA2000CC075008EA241112C6898011900564E0F1
:10CA3000C0E0EA2411F582EB12B740D0E012CBED52
:10CA4000A2E050037508208A828B83A3A3E024FF11
:10CA5000FEA3E034FFFF12CBC112BA8FC39402E0F1
:10CA600040061412B6DA74034508F508890C750DF2
:10CA700000740E780C120988E50DF50974026970CE
:10CA80001490055C12B6D990055BE08E828F83F01E
:10CA900012B6E7801D7403697015EE24F9FEEF34B9
:10CAA000FFFF7C6B7D05EEFAEFFB1218C980E1E910
:10CAB000602F851082851183E060187413120A6D4F
:10CAC000E0650E7004A3E0650F700874404508F53A
:10CAD00008800E8E828F83E50F12CC02E50E12B60F
:10CAE000DE851082851183E0F50C750D00740A78DF
:10CAF0000C120988E50D4509F509E06402701C7403
:10CB000001120A6D12BC1BE012CBE3120A6D12B7C0
:10CB10002F8E828F83F012B6E78021E064037019B4
:10CB2000EE24F9FEEF34FFFF7401120A6D12B6F223
:10CB3000EEFAEFFB1218C980DDE060117413120ADF
:10CB40006DA312B6D97413120A6D12B6D9EEF8EFAE
:10CB5000F9E824FF1EE934FFFFE50A240DF582E51C
:10CB60000B12BA8F70059005478003900553E0FAC9
:10CB700004F0EA8882898312CBDDE50912CC02E554
:10CB800008F0E50A2404F8E50B3400F9E50A24026C
:10CB9000FAE50B3400FBEEFC12CBB5FDE02DC39C97
:10CBA00012CBBDEEF0A3EFF07900740302B6CDE82E
:10CBB000240FF582228A828B83E002B6C5F002C977
:10CBC00054EA240DF582EB2212CC90EB12C0A32282
:10CBD00012CBD42212C406A3A3A3A3E022F08E8218
:10CBE0008F83228E828F8312B6E274012212CBF1E0
:10CBF00022F0EA240EF582EB12CBFC223400F583FE
:10CC0000E02212B6E280D712CBF1A2E42274F01235
:10CC1000035689088A098C0E8D0F8B0C7410120A2A
:10CC20006D12DA08AA0C120EA38A0A8B0BA80AA9A5
:10CC30000BE87001E9604AE8240EF582E912B7407A
:10CC4000E50CF0E8240DF582E912B740E508F08E16
:10CC50000C8F0D780C1207EFAC0EAD0FA90912C0A6
:10CC60007412081DE9701AE5081205E807017ACC6C
:10CC700074CC74CC12CC84D2E5F0AA0AAB0B120EA1
:10CC8000F702B6FFE50A12CC90E50B12D2A422E817
:10CC90002410F5822274F7120356EAFEEBFF7A01A4
:10CCA000EE242312BA8C60027A0512B73AEA12C057
:10CCB00098740412CCF1242212CCDD242012B73D4A
:10CCC00012065312D08879031A1A12C07212081D64
:10CCD000E97007EEFAEFFB120EF702C1D512C0A001
:10CCE00012CBB9F074018E828F83A3A3A3A3F0EEBD
:10CCF00022F012CCFA12CD08EE22EE2402F8EF3424
:10CD000000F9E8FAE902C95312B6BB8A828B83E8BC
:10CD1000F0A3E9F02274F01203568A0C8B0DECFE9E
:10CD2000EDFF74058A828B8312CF398A828B83A3AD
:10CD3000A3F0EA2403F50EEB3400F50FEE242412E1
:10CD4000B73D7808120A2E850E82850F8312CF0414
:10CD500012CF4812B774850E82850F8312C17C12E0
:10CD600018BD850E82850F8312D297FAA3E0FB8847
:10CD7000828983A3A3A312C8D1EE242E12BA8CC039
:10CD8000E012CC8FE912B740D0E012CF1C2415126C
:10CD9000CEFF12CF1C240E12CEFF12CF41850E8281
:10CDA000850F83E02416FAA3E03400FB1210178EDF
:10CDB000828F83A3A3A3A3A3A3E0C0E0850E8285F3
:10CDC0000F83E0240DF8A3E012B9EFD0E012CF25D5
:10CDD000FAA3E0FB850E82850F8312B67D240BFC3F
:10CDE000E93400FD8A828B83E08C828D83F0A3E49A
:10CDF00012CF30E0F5098C828D83E0F0A3E0450985
:10CE000012CF2BE0FCA30A0AAB83A2E7E492E0C0B6
:10CE1000E012CBAFE912B740D0E0F074075C6004D9
:10CE200078018002780075F00374075CA428F8EAA2
:10CE300028FAEB3400FBE50C2405F8E50D3400F985
:10CE400012CBB512CF30850C82850D8312C8D188E4
:10CE5000828983E0F50AF50874075508C333FC742A
:10CE600070550AC430E30244F0F5083395E0F50943
:10CE700074037808120988E5082CF8E5093400F9EC
:10CE8000EA28F8EB39F9850C82850D83A3A3A3A3C7
:10CE9000A3A3A312D09C8E828F8312CEF2E02AFA33
:10CEA000A3E03400FBC3EA98EB9940278E828F837E
:10CEB000A3A3E0F8850C82850D83A3A3A3A3A312EB
:10CEC000CEF2A3A3E0C39A28850C82850D83A3A389
:10CED000A38016E4850C82850D83A3A3A3A3A3A33B
:10CEE000A3A3F0850C82850D83A3A3A3A3A3F002C3
:10CEF000B6FFA3A3A3A3E0FA8E828F83A3A322127B
:10CF0000CF0BE422E0241112CF0B22F812CF102213
:10CF1000A3E012CF16223400F902B6C5F0850E82C6
:10CF2000850F83E02212C2D6A3E02212CBBDA3223A
:10CF300012CBBDA3AA82AB8322F0EE243112D2A180
:10CF400022F0EE240702B777E508F0A3E509F0A385
:10CF5000E50AF0A3E50BF022C082C0837C0B7D00C4
:10CF6000790012116D02BE4D0207CFC082C08379D5
:10CF700018120FB702BE4DC082C0838A828B83E035
:10CF8000C3940B500312102302BE4D74F7120356C4
:10CF9000EAFEEBFF8E828F83E07003120FE77919B0
:10CFA000EEFAEFFB120FB702C1D574F7120356EA7F
:10CFB000FEEBFF90050DE07002A3E0601590050DFB
:10CFC00012C17C12102F12C4B890050D12C17C1230
:10CFD0000FE790050DEEF0A3EFF002C1D574F71244
:10CFE000035674DE1208AFEAFEEBFF8E828F83E0F9
:10CFF0001206D8011E1F44D0030304D00544D018E4
:10D0000004D04DD07416120A6DE412D083740B1242
:10D010000A6DAA82AB831218C97413120A6D7403C5
:10D02000F090055B12DD4C7402120A6D12D09E74F2
:10D030000A120A6D740212D07B7414120A6DE8F0A1
:10D04000A3E980107416120A6D740180BD74161263
:10D050000A6D7402F0740B85108285118312CBDD8A
:10D06000A3E0C0E07401120A6DD0E012CF41741742
:10D07000120A6D12C3D5742202B734F0900557120C
:10D08000DD5022F012D08822EE241702B7778E08E6
:10D09000EA2508F8EB3400F98A828B83A3A3E8021F
:10D0A000CD1074F7120356EAFEEBFF750800EE246C
:10D0B0002012D0FD7003A3E06960037508E8EE2438
:10D0C0001712B6856016EE2423F582EF12B6D3E56B
:10D0D00008701AEEFAEFFB12100B801EEE242312DA
:10D0E000BA8C60EB900538E070E57508E88E828FA9
:10D0F00083A3E508F0741912D83502C1D512C0A077
:10D1000012DD50900557E06822C082C08374F1128E
:10D1100008AF7402120A6D740412CF2BE0C0E074E1
:10D1200003120A6DD0E0F0EA2420F582EB12DD490B
:10D13000740D120A6D12D09EEA2417FCEB3400FD28
:10D140007404120A6DAA82AB831218BD7404120A09
:10D150006DAA82AB83120FF9E9600312D1CE74027B
:10D16000120A6DAA82AB8312191702BF2E74F6122F
:10D17000035674E81208AFEAFEEBFF7402120A6D60
:10D180007403F0EE2412F508EF3400F509AC08FD45
:10D190007404120A6D12B722C0E0740C120A6DD02A
:10D1A000E012CF41740D120A6DAA82AB83121017E0
:10D1B000AA08AB09120FF9E9600312D1CE7402126A
:10D1C0000A6DAA82AB83121917741802C4B08510B5
:10D1D0008285118374FFF0A312D1E9795312108371
:10D1E00090055174FFF0A3F02212D1EF02CF34F07A
:10D1F0008510828511832274F712035674D41208A5
:10D20000AFEAFEEBFF8E828F83A3A312BC1BE0A2CA
:10D21000E6501790055712D297687003A3E0697023
:10D2200009900539E0604D121059740B120A6DA86F
:10D2300082A9837403120A6D12D09EEEFCEFFD8565
:10D240001082851183AA82AB83121011742B12C82D
:10D25000DD90053CE060087408120A6DE06010740F
:10D2600005851082851183F0AA82AB831219177489
:10D270002C02B734900560E060B012B68270AB90BB
:10D2800005571206537B017C487D057A0379061207
:10D29000B69112081D80D812DD50EE242A12D2A1B8
:10D2A00022F582EF12CBFC22C082C08374EF1208F9
:10D2B000AF7409851082851183F07401120A6D74B0
:10D2C000EE12DB3402BF32F582EB12D2A4FA2274E2
:10D2D000F7120356A2AFE492E0FFC2AFE960031277
:10D2E00010711216E312D34E900539E0F91217555A
:10D2F00012D5F112D5E77A6B7B051217677E00EE27
:10D30000C333F8E433F912D343E07002A3E06009B9
:10D3100012D34312BD22121A8A0EEEC3940740DFC5
:10D32000120FABE4900575F0120E9DE4900539F0F4
:10D330007A5A7B057952121083EFA2E092AF7900FE
:10D3400002C1D5E82418F582E93405F58322900559
:10D350006AE0F9121779900569E0F912176D22C099
:10D3600082C0837909120FCF02BE4DC082C0839064
:10D370000526749EF0A3741DF09005287404F0A394
:10D38000741EF090052A74ACF0A3741DF090050F84
:10D39000E4F0A3F01216DD02BE4DC082C083901CE3
:10D3A0009C7C3A7D05743B12072912174FE99005C2
:10D3B00053F012174FE990054702B7C4E9C39440F0
:10D3C000400CE9C3945E500674C029F98012E9C389
:10D3D00094E0400AE9C394E45004743E80EC79225E
:10D3E0000207CF74F4120356EAFEEBFF121077E93E
:10D3F000FA8A0874226A700479F48049A2AFE49230
:10D40000E0F50BC2AF75090074027808120988E5CF
:10D4100008248CFAE509341AFB8A828B83E493246E
:10D420003AF508E43405F509750A0078081207EBA7
:10D430008A828B83A3E49312D9FC12081DE50BA208
:10D44000E092AF790002B67274F11203568908EACD
:10D45000FEEBFF74456508700B90053FEEF0A3EFFF
:10D46000F002D5C8121077E9FA8A0A74226A7005A8
:10D4700079F402D5CA890C750D007402780C120972
:10D480008812D5DA7014890C750D007402780C12AC
:10D49000098812D5CD700302D52B890C750D007447
:10D4A00002780C120988E50C248CFAE50D341AFB7D
:10D4B0008A828B83A3A3E493FC8A828B83A3A3A396
:10D4C000E4936C700579FB02D5CA74586508702125
:10D4D0008E828F83C3E0948FA3E09400400E8E82EF
:10D4E0008F83C3E094B1A3E09464400579E802D54A
:10D4F000CA8E828F83E0C0E0890C750D00740278BB
:10D500000C12098812D5DAFAD0E0C39A40DE890CF1
:10D51000750D007402780C12098812D5CDC0E08E0A
:10D52000828F83E0FAD0E0C39A40C1A2AFE492E0D8
:10D53000F509C2AF750B007402780A120988E50A72
:10D54000248CFAE50B341AFB8E0C8F0D750E0078C7
:10D550000C1207EB8A828B83A3E493FC7D008A8202
:10D560008B83E493243AFAE4340512DA0212081D9C
:10D57000E509A2E092AFE5081206D800065091D561
:10D58000529BD55396D5E0C0D5E1ADD5E2B7D5C80D
:10D59000D512D5F1803212D5E7802D90055AE07969
:10D5A000026005121821802012182D801B90056A38
:10D5B000E0F912177980117A6B7B051217678008E2
:10D5C000900569E0F912176D790002B757E50C2450
:10D5D0008FF582E50D341A02C750E50C248EF582D2
:10D5E000E50D341A02C75090055B12C18012176115
:10D5F0002290055712C18012175B220207CF74F2E6
:10D6000012035674078A828B8312D662E08A828B59
:10D6100083A3A312D662A3A3E08A828B83A3A3A3CE
:10D6200012D65BA37808120A2E8A828B83A3A3A347
:10D63000A312CF48E48A828B83A3A3A3A3A3A3A3AB
:10D64000A3F0EC2415F582ED12B74012C94EA3A346
:10D65000A3A3A3A3A312D09C02B6A3F08C828D83B4
:10D66000A32212D65B02B76E74F4120356EAFEEBE5
:10D67000FFE490057712B767E0C39404400674E8AE
:10D68000900577F08E828F83A3A3A3A3A3A3A3E027
:10D69000C3940F40158E828F83A3A3A3A3A3A3E0FB
:10D6A0006403601574E8900577F08E828F83A3A3DE
:10D6B000A3A3A3A3E06403700E90050FE0A2E040D3
:10D6C0000674E8900577F0EEFCEFFD7A767B0512A4
:10D6D000108F8E828F83A3A37808120A2E740A7883
:10D6E0000812085190058A7808120A1F8E828F83CB
:10D6F000A3A3A3A3A3A3A3E090058E12D7559005DF
:10D700008FF0740A900590F090056AE0900591F012
:10D7100090058712BEFB7404900589F0900577E0B0
:10D720007022900578E0600674EA900577F0900525
:10D7300078E0F912178574268E828F83F0790412AF
:10D740001821800774298E828F83F0EEFAEFFB1286
:10D750000FC902B67212B76B02CBD874F41203561B
:10D7600074F71208AFEAFEEBFF900578E070319095
:10D770000590E0640A6029121797E9C0E0900590CF
:10D78000E0F890057FE028F8A3E03400F974F5286C
:10D79000F58274FF39F583D0E0F090057EE004F067
:10D7A00090058A7808120A2E7401780812085190A0
:10D7B000058A7808120A1F900590E004F0E508A297
:10D7C000E04006E0C3941D40D7E0641D60557A90A8
:10D7D0007B0579E1121083900578E06004640270A3
:10D7E00009EEFAEFFB1210A1803E7408120A6D12C6
:10D7F000D82BF0900578E06401700679087A808073
:10D800000479077A837508FF7509FF78081207EF16
:10D810007B007402120A6DAC82AD8312B6911208BD
:10D820001D8005742912D83502B66D740212D1EF2D
:10D8300074FFF0A3228E828F8312BDBA120FC92209
:10D8400074F0120356750801750900750A00750B0E
:10D8500000900590E0780812078B78081209D090A4
:10D86000057A780812093C900578E06403700F127D
:10D87000D8BF120A2E7808790C1202668035750816
:10D8800001750900750A00750B0090058EE0780897
:10D8900012078B9087797808120903908765780CB6
:10D8A000120A2E7808790C120266900578E070034F
:10D8B00012179178081207E77A817B0502B6CA90A1
:10D8C000056512B660908765780C2274F2120356D3
:10D8D00074D41208AF8A0C8B0D900578E064026056
:10D8E00008E06401600302D9F7E4900577F0740B57
:10D8F000120A6DA882A9837403120A6D12D09EAC1D
:10D900000CAD0D851082851183AA82AB8312101194
:10D9100090058FE0700302D9B490057EE0C0E090DE
:10D92000058FE0FAD0E0C39A400302D9B490057F96
:10D9300012DA0890057EE0F508803B8E828F83A383
:10D94000A3A3A3A3A3A3A3A312DD4C7414120A6D73
:10D95000E0687003A3E0696013740B120A6DAC8277
:10D96000AD83EEFAEFFB1218B7E960141508EE2448
:10D9700021FEEF3400FFE50870C190057EE07034B1
:10D98000740B120A6DA982AA8389088A09750A0094
:10D9900078081207EB7C217D0090057EE08CF0A4D6
:10D9A000F8A9F0EE28FAEF3912DA0212081D9005F4
:10D9B0007EE004F090053CE0600E7408120A6DE011
:10D9C000700690058FE0700D851082851183AA8204
:10D9D000AB8312191790058FE0601C90057EE0FA6A
:10D9E00090058FE06A70107429850C82850D83F094
:10D9F000AA0CAB0D120FC9742C02B6A0FC7D00EE70
:10DA0000FAEFFB02C77AA3A3E0FEA3E0FF2274F6BD
:10DA100012035674FE1208AF8A088B09EA241AF51D
:10DA200082EB12BA8F64037067EA2423F582EB124B
:10DA3000BA8F6403705AEA2412FAEB12DA95850859
:10DA40008285098312DA0612DAA77950121083123E
:10DA5000DAA7794B121083EEFAEFFB79E11210830B
:10DA60008E828F83A312B69785108285118312CD83
:10DA700010851082851183AA82AB8379531210839B
:10DA8000E4900577F0742985088285098312DA9E6F
:10DA9000740202C4B03400FB794A12108322F0AA47
:10DAA00008AB09120FC9228E828F83E0FAA3E0F936
:10DAB000EA851082851183F0A3E9F012DAC7851098
:10DAC0008285118302CF34EE24020E0EEF3400FF64
:10DAD00022C082C083900577E064E860267A817B6B
:10DAE000051210EF12178B790412182D900578E0AB
:10DAF00064037006900577E060097A917B0579E10F
:10DB00001210837A767B0502BE48C082C08374F50A
:10DB10001208AFEAFCEBFD851082851183AA82AB67
:10DB20008312108F7401120A6D74FC12DB34740BB3
:10DB300002BF34E912D1E912191722C082C08379D9
:10DB40000702D36574F4120356900596E4F0A3F02F
:10DB5000900592E07002A3E0603D90059212DC1502
:10DB6000C082C08390147F7808120A2ED083D0829E
:10DB700078081208C5502012DC9D90059212DCB284
:10DB80001208C5500990059212DCB2120A1F9005C6
:10DB90009212DC0E12D09E900594E07002A3E090E9
:10DBA0000596602DE07002A3E0601B90059412DCE6
:10DBB00015C082C08312DCAF120A2ED083D08278C7
:10DBC000081208C5501290059412DC0E12D09E80E7
:10DBD00007E07002A3E0603090059612DC15C08269
:10DBE000C08390147F7808120A2ED083D0827808E0
:10DBF0001208C5501312DCAF120A2EAA08AB09ACEA
:10DC00000AAD0B121683800312168902B67212DD5A
:10DC1000509005962212DC192212DC1D22E0F8A396
:10DC2000E0F5838882A3A32274F012035690059630
:10DC3000E07002A3E0605912DCAF120A2E75831463
:10DC400075827F78081208C5500D1214FD90059654
:10DC5000E07002A3E0603912DC9D90059612DCA909
:10DC6000120A2E780C79081209E0402490059612C9
:10DC7000B750FAEFFB12DC93A3A3A3A3E0F98E82C3
:10DC80008F83A3A3A3A3A3A312BD22121A8A80BDCC
:10DC900002B6FF1210EF8E828F8302B76F121677D3
:10DCA0008A088B098C0A8D0B2212DC19780C2290C1
:10DCB000059612DC1978082274F01203568A0C8B30
:10DCC0000D8C0E8D0F7410120A6D80248E828F833E
:10DCD000A3A3C082C08390876D7808120A2ED083D8
:10DCE000D08278081208C550031214FD8E828F83EB
:10DCF00012B7507001EF604B8E828F83A3A3780C14
:10DD000012096290059612DD4CEE687002EF6970A0
:10DD1000BB8E828F83A3A3C082C08390876D780857
:10DD2000120A2ED083D08278081208C5509E9087A0
:10DD30006D7808120A2E8E828F83A3A37808120AA8
:10DD40001F80A902B6FFF582EF12C0A312DD502298
:10DD5000E0F8A3E0F92274F3120356A2AFE492E0D4
:10DD6000F50CC2AF90059412DA0890059212065392
:10DD700090147F7808120A2E78081209AEAA08AB10
:10DD800009AC0AAD0B1210D1740212081D80378E37
:10DD9000828F83A3A3C082C08390147F7808120A65
:10DDA0002ED083D08278081208C5401390147F7853
:10DDB00008120A2E8E828F83A3A378081208EF8E92
:10DDC000828F8312DA08EE7001EF70C390147FC067
:10DDD000829014837808120A2E758314D0827808F2
:10DDE0001208DA60239014837808120A2E90147FA8
:10DDF0007808120A1F90147F7808120A2EAA08AB1E
:10DE000009AC0AAD0B1216711210C5E50CA2E09216
:10DE1000AF7F0502056374F1120356A2AFE492E0EE
:10DE2000F50EC2AF8C0C8D0D8C828D8380088E0C0C
:10DE30008F0D8E828F8312B7507001EF60208A821F
:10DE40008B83A3A3C082C0838E828F83A3A3780811
:10DE5000120A2ED083D08278081208C550D0850CC3
:10DE600082850D8312C8D78A828B83EEF0A3EFF0F0
:10DE70008C828D8312DE897002EB6970031210C5EB
:10DE8000E50EA2E092AF02B75712DD50EA682274A5
:10DE9000F0120356EAFEEBFF7410120A6D780C12B2
:10DEA0000A2E12DC9D780C79081209168E828F8357
:10DEB000A3A3780C120A1F7C927D0502B6F874F7B2
:10DEC000120356EAFEEBFF8C828D83A882A983128F
:10DED000C17C8A828B83E5827002E5836018EE65DF
:10DEE000827003EF658370E312C17C88828983129C
:10DEF000C8D779018002790002C1D574F7120356A0
:10DF0000EAFEEBFFA2AFE492E0F508C2AF7C927D9F
:10DF1000051210E9E9700B7C947D05EEFAEFFB1217
:10DF200010E990059612DD4CEE687002EF697003FF
:10DF30001210C5E508A2E092AF02C1D574F4120335
:10DF40005674F81208AF7F008F088F09900DD3E444
:10DF5000F07E79750A08750B00780A1207EF7402D3
:10DF6000120A6DAC82AD837A007B00EE12EFF112E3
:10DF7000081D851082851183E0F47003A3E0F4701E
:10DF800013900DD3E07004EEF0802B7A01EEF912BD
:10DF9000120380227402120A6DE0F47003A3E0F40D
:10DFA00070048E0880107404120A6DE0F47003A3EC
:10DFB000E0F46002EEFFAC097A007B00EEF9121289
:10DFC000098B0BEA450B60057509017E780EEEC3DF
:10DFD000947F500302DF53E508601D900DD3E0608D
:10DFE0000C7A01A908121203EF7008800BEF600E83
:10DFF000E508F0EFF9121215900DD3E070117E795B
:10E00000EEF912120F0EEEC3947F40F41211FD7957
:10E0100001740812081D7F0402056374F712035689
:10E0200074F81208AFEAFF851082851183E4F0A32B
:10E03000F0EF60087402120A6DE480077402120A9D
:10E040006D74FF12E3DF7A007B0012123374081242
:10E05000081D7F0102056374F012035674F612085E
:10E06000AF851082851183EAF0A3EBF0890E8C0F47
:10E07000750A08750B007E007F00801CE5082408E7
:10E08000F8E5093400F9EE28FEEF39FFE50A250826
:10E09000F50AE50B3509F50B7508087509007808D0
:10E0A0001207EF7404120A6DAC82AD83AA0AAB0B9F
:10E0B000A90E12EFF212081D7402120A6DE0F4703C
:10E0C00003A3E0F46041E50A2408F50AE50B3400F7
:10E0D000F50B7404120A6D12E84112E39FF508E98A
:10E0E000F509E50A2508F8E50B350912E388403300
:10E0F000EE2408F8EF3408F9E8C3950AFEE9950B19
:10E10000FF750A00750B08E50E12E22EE50AF0A372
:10E11000E50B12E232EEF0A3EFF07A007B00740A16
:10E1200002EFA27402120A6D12EC38700302E07C56
:10E1300085108285118312EC38605285108285111A
:10E1400083A3E0547FF97402120A6DE0687003A3A0
:10E15000E069600302E08C7408120A6D12ECB2856B
:10E160001082851183A3E05480700F74FF6A7003DE
:10E1700074FF6B600302E08C800D74FF6A7003749F
:10E18000FF6B700302E08CAA0AAB0B8091AA0AAB6A
:10E190000BA90E12E391120A6DE0687003A3E06907
:10E1A00070507408120A6D12EC32E50F603074FF83
:10E1B00068700374FF69600302E08C7402120A6DD8
:10E1C000E0FAA3E04480FB12121BEA4B700302E06A
:10E1D0008C7C01900DD4E0F9121A0702E08C74FFD8
:10E1E00068700374FF69700302E08C7AFF7BFF02A2
:10E1F000E11E7C01AA0AAB0BA90E121A0702E07CF1
:10E2000074F7120356E9FE79041214F7E9700790C7
:10E210000DD574018014EEF9121539EE12E22E7448
:10E2200008F0A3E412E232E4F0A3F002E05212E3B9
:10E23000C722F012E2372274D528F582740C39F522
:10E24000832274F212035674F61208AFE9FE12E349
:10E25000BFE0F508A3E0F50912E3D87A04FBEEF974
:10E260001212398510828511837408F0A3E402E349
:10E270000812E39FF50AE9F50B7402120A6D12EC1D
:10E2800038607785108285118312E3ABF912E39130
:10E29000120A6DE0687003A3E06970597C0012E314
:10E2A000B07402120A6D85820C85830D780C1207FA
:10E2B000EF7C087D00AA08AB09900DD3E0F912129B
:10E2C0003F740212081D12EC0B780A1207EF78084F
:10E2D0001207EF900DD3E0FC7404120A6D12E3AB49
:10E2E000F9121245740412081DE508250AF508E51F
:10E2F00009350BF5097C0112E3B085108285118385
:10E30000E0250AF0A3E0350BF0750A08750B0078DC
:10E310000A1207EF7404120A6DAC82AD8374021204
:10E320000A6D12E3AB12EFF112081D7402120A6DAE
:10E33000E0F47003A3E0F4602B851082851183E084
:10E340002408F0A3E03400F07404120A6D12E841CE
:10E35000851082851183E02CF8A3E03D12E38850FC
:10E360000302E27112E3BFE508F0A3E509F0EEF95C
:10E3700012120F7A01900DD3E0F9121203EE900DF4
:10E38000D3F0740A02E6653BF9C3E89401E9940806
:10E390002212122D8A0C8B0DA80CA90D740622ECEA
:10E3A0002403F8ED3400F9E854FC2212ECB6EE2216
:10E3B00085108285118312ECB6EEF9121A072290AD
:10E3C0000DD3E012E3C722C333F8E433F974C9284C
:10E3D000F582740C39F58322851082851183E4F06F
:10E3E000A3F0851082851183AC82AD832274F41270
:10E3F0000356EAFEEB800374804FFF7508797C00BA
:10E40000EEFAEFFBA9081212098B0BA90BEA49607F
:10E4100008E508900DD4F080150508E508C3947F41
:10E4200040DCEF548060D0900DD4E4F0FAFB02E0C1
:10E430001674F012035689088A0E8B0F12E39F247C
:10E4400008FAE93400FB750900750C06900DD3E05D
:10E4500004FFEFC3947F40027F79900DD3E06F609B
:10E460003674872FFEC333F8E433F974BB28F58282
:10E47000740D39F58312ECAA74C728F582740D392E
:10E48000F58312EC32E50AC398F8E50B99F9E82A0E
:10E49000F8E912E38740090F150CE50C70B48054BD
:10E4A000E50C6050E50A2AF8E50B12E38740059079
:10E4B0000DD3E0FFE508F50978091207F37411128E
:10E4C0000A6D120653AA0EAB0FEFF912124B74032A
:10E4D00012081DE9F509900DD3E06F701774792EBD
:10E4E000F9E5086005121215800A7410120A6D12FF
:10E4F000EFDDE9F0A90902EFA574F212035674F8F2
:10E500001208AF890A8C0BEA24F8F508EB34FFF502
:10E5100009750C08750D00780C1207EF7402120AC9
:10E520006DAC82AD83AA08AB0912EFF212081DE5AB
:10E530000B70237406120A6DE4F0A3F07404120A3F
:10E540006DAC82AD83E5082404FAE5093400FBA92B
:10E550000A121233802B7402120A6D12EC18FEE9B3
:10E560003400FF12E3D8AA08AB09A90A121233E556
:10E570000AC333F8E433F912E237E02EF0A3E03FA8
:10E58000F0740802E66574F112035674FC1208AFC9
:10E59000890E8A088B09ECFEEDFF750A00750B00E9
:10E5A000EE2403F50CEF3400F50D7402780C120A1A
:10E5B00010AE0CAF0D12E9BA604F750C04750D006A
:10E5C000780C1207EF7402120A6DAC82AD83AA08B0
:10E5D000AB09A90E12EFF212081D12E9EB780088C0
:10E5E0000C851082851183E582250CF582E5833444
:10E5F00000F583E0FAE50A2AF50AE50B3400F50B8D
:10E6000008E8C3940450AE80D6AA0AAB0B74041277
:10E61000081D7F0702056374F2120356890A8A08EF
:10E620008B09ECFEEDFF79041214F7E9602F750CED
:10E6300001750D00780C1207EFEEFCEFFD74027807
:10E6400008120A10850A0C7409780C120988E5086A
:10E650002400FAE50912E82512081D8006900DD560
:10E660007401F0800312081D7F0602056374F7121F
:10E67000035674FC1208AF8C828D83E0851082856E
:10E680001183F08C828D83A3E0C0E07401120A6DC7
:10E69000D0E0F07402120A6D74FFF07403120A6D78
:10E6A00074FF12E3E1121233740402E04F74F012AB
:10E6B000035674FC1208AF890F8A088B09ECFEED33
:10E6C000FFEA5403F50E606B74FC5508F508750AF3
:10E6D00004750B00780A1207EF7402120A6DAC82FF
:10E6E000AD83AA0812EFF212081DEE4F60327414C7
:10E6F000120A6D12EC27C0E0850E0A12E82ED0E057
:10E70000F07414120A6D12E847120A6D12EC4005FB
:10E710000EEE24FF1EEF34FFFFE50EC3940440CA43
:10E72000851082851183AC82AD83AA08AB09A90F3D
:10E7300012E9E4EE5403F50E8E0A8F0B7402780A88
:10E74000120A10AE0AAF0BEE4F607079041214F784
:10E75000E96035780A1207EF7416120A6D12E84163
:10E7600085080A85090B7402780A120A10850F0CB5
:10E77000F50D7409780C120988E50A2400FAE50BF6
:10E7800012E82512081D8006900DD57401F08E0A3E
:10E790008F0B7402780A120988A80AA90BE50828C9
:10E7A000F508E50939F5097414120A6DE028F8A393
:10E7B000E039F97414120A6D12EC40E50E60617EC6
:10E7C00000750A048E0B780A1207EF7402120A6DA4
:10E7D000AC82AD83AA08AB09A90F12EFF212081D93
:10E7E00080217414120A6D12EC27C0E08E0A12E820
:10E7F0002ED0E0F07414120A6D12E847120A6D125E
:10E80000EC400EAF0E74FF2FF50E0470D58510820C
:10E81000851183AC82AD83AA08AB09A90F1212330C
:10E82000740402EFA2350DFB121533740222851019
:10E8300082851183E582250AF582E5833400F5831C
:10E8400022E0FCA3E0FD22E02401F8A3E03400F97B
:10E8500074142274F012035674FB1208AFE9851089
:10E8600082851183F08A0E8B0F8C0B7415120A6D42
:10E87000E0F508A3E0F5097417120A6DE0FEA3E0C5
:10E88000FFE5085403F50A606BF50CC3E508950C29
:10E89000F508E5099400F509750C04750D00780C70
:10E8A0001207EF7403120A6DAC82AD83AA08AB099C
:10E8B000A90B12EFF212081DEE4F6030750C0178B3
:10E8C0000C1207EF850A0C7403120A6D12E9C912C3
:10E8D0000A6D12EFF012081D12E9AD050AEE24FFD1
:10E8E0001EEF34FFFFE50AC3940440CC7401120A02
:10E8F0006D12E9DAEE5403F50A8E0C8F0D7402786E
:10E900000C120A10AE0CAF0D8037750C04750D009B
:10E91000780C1207EF7403120A6DAC82AD83AA0E55
:10E92000AB0F7402120A6D12EFF012081DE50E24EF
:10E9300004F50EE50F3400F50F7401120A6D12E9AB
:10E94000DA12E9BA70C4E50A605E7E00750C048EC6
:10E950000D780C1207EF7403120A6DAC82AD83AA16
:10E9600008AB09A90B12EFF212081D801F750C01EC
:10E97000780C1207EF8E0C7403120A6D12E9C9129B
:10E980000A6D12EFF012081D12E9AD0EAF0A74FF06
:10E990002FF50A0470D77401120A6DAC82AD83AAF8
:10E9A00008AB09A90B121233740502EFA2E50E247D
:10E9B00001F50EE50F3400F50F22EEF8EFF9E8242B
:10E9C000FF1EE934FFFFE84922E582250CFCE583C0
:10E9D0003400FDAA0EAB0F740222AC82AD83AA08EC
:10E9E000AB09A90B12123312E9EB22E5082404F556
:10E9F00008E5093400F5092274F112035674F41283
:10EA000008AF851082851183EAF0A3EBF0E9FE8C54
:10EA10000A8D0B741D120A6DE0F50EEEC333F8E497
:10EA200033F974C928F8740C39F97402120A6D129A
:10EA3000EC407402120A6D12EC27F508A3E0F50908
:10EA40007F00900DD3E06E70077A00EEF91212038A
:10EA500012EC2C7404120A6D12EC407406120A6D4A
:10EA6000E50AF0A3E50BF07404120A6DAC82AD83E5
:10EA7000AA08AB09EEF9121233750C088F0D780C49
:10EA80001207EF7406120A6DAC82AD83AA08AB09B7
:10EA9000EE12EFF112081D7404120A6D12EC3285A9
:10EAA0001082851183E0687003A3E069600302EBC4
:10EAB000E37406120A6DE0650A7004A3E0650B605A
:10EAC0000302EBE3E50E700302EBE1741B120A6D27
:10EAD00012EC3288828983A80AA90BE85403F50C4A
:10EAE000E58245837015E875F0FFA4F8AAF075F08B
:10EAF000FFE9A42AF9E8FAE9FB80207A007B00808C
:10EB00000AE0FCEA2CFAEB3400FBA3E8FCE9FDEC9C
:10EB100024FF18ED34FFF9EC4D70E6E50C601E742F
:10EB200004C3950CF895E0F9E875F0FFA4F8ACF093
:10EB300075F0FFE9A42CF9EA28FAEB39FB8510827D
:10EB4000851183EAF0A3EBF012EC0B741B120A6D33
:10EB500012EC38601A741B120A6D120653AC0AAD1F
:10EB60000BAA08AB09EEF912123F740212081DAC91
:10EB70000AAD0BAA08AB09EEF912122D8A0A8B0B0B
:10EB8000A80AA90B851082851183E0687003A3E0B1
:10EB9000697050851082851183AC82AD83E50824AD
:10EBA000FCFAE50934FFFBEEF9121239750A088FF9
:10EBB0000B780A1207EF7406120A6DAC82AD83E57A
:10EBC0000824F8FAE50934FFFBEE12EFF112081DF4
:10EBD00012EC2C7408120A6DE0687003A3E06970EF
:10EBE00002EEFF7406120A6D12EC18F8E93400F90F
:10EBF0007402120A6DE0FAA3E0F5838A82E028F03D
:10EC0000A3E039F0EFF9740C02E60FE5082408F5EB
:10EC100008E5093400F50922E02403F8A3E03400F4
:10EC2000F9E854FC24082212EFE1E02285108285E5
:10EC30001183E0F8A3E0F922E0F8A3E0F9E8492223
:10EC4000E8F0A3E9F022C082C0831211FDD083D086
:10EC5000820207CF74F2120356EAFEEBFF8C088D96
:10EC600009740E120A6D12ECAA900DD5E4F012127E
:10EC70001B8B0DEA450D60047900802B780A120782
:10EC8000EFAC08AD09EEFAEFFB7901121221740224
:10EC900012081DE9600F900DD5E060051211FD808E
:10ECA0000479098002790A02E668E0F50AA3E0F532
:10ECB0000B2212ECB622E0FAA3E0FB2274F012035E
:10ECC0005674F11208AF7403120A6DEAF0A3EBF068
:10ECD0008C0A8D0B750900900DD5E4F0741F120A93
:10ECE0006D12EC38700302EF9E7403120A6D12EC81
:10ECF000B212121B8A0C8B0DA80CA90DE8FEE9FFBD
:10ED00007405120A6D12EC40EE4F7005790902EF9E
:10ED1000A0750C08750D00780C1207EF7409120A23
:10ED20006DAC82AD83EE24F8FAEF12EFEA12081D03
:10ED30007409120A6DC082C083741F120A6D12EF2B
:10ED4000BED083D082C3E098A3E0995005790A022F
:10ED5000EFA012EFAA120A6DE0F50EA3E0F50F7412
:10ED60001F120A6D12EC327401120A6D12EC40751A
:10ED70000C01780C1207EF7402120A6DAC82AD839D
:10ED8000EEFAEF12EFEC12081DEE24010EEF340044
:10ED9000FFA80EA90F88828983A385820E85830F21
:10EDA000851082851183E0FA88828983E06A701772
:10EDB0007401120A6DE024FFF0F8A3E034FFF0F9CB
:10EDC000E84970AB02EF9285108285118385820C31
:10EDD00085830D780C1207EF740B120A6D12E8414F
:10EDE0007405120A6D12ECB279001212217402122B
:10EDF000081DE9F508700302EF8F7409120A6DE02F
:10EE00002403F8A3E012E3A4F87401120A6D12ECD3
:10EE100040E508C333F8E433F974C928F8740C39B1
:10EE2000F97403120A6D12EC407403120A6D12EFAA
:10EE3000DDC082C0837401120A6D12EC32D083D01F
:10EE40008212EFB5900DD4E0F50E7C007405120A25
:10EE50006D12EFC8780A1207EF8E0C8F0D780C1226
:10EE600007EFAC087409120A6D12ECB2A90E121267
:10EE700045740412081D12EFAA120A6D120653748B
:10EE800021120A6D12EFD112123F740212081D7482
:10EE900009120A6DE0C3950AFAA3E0950BFB741FF3
:10EEA000120A6D12EC32EAC398F50CEB99F50D7865
:10EEB0000C1207EF7421120A6DE02EF50CA3E03F4F
:10EEC000F50D780C1207EFAC087409120A6D12EFF9
:10EED000BE7423120A6DE028FAA3E039FBA90E12D2
:10EEE0001245740412081D7403120A6D12EFDDC07E
:10EEF00082C0837401120A6D12EC32D083D0821268
:10EF0000EFB57409120A6D12EFD112122D740112AD
:10EF10000A6DEAF0A3EBF0EE24F8FEEF34FFFF7485
:10EF200001120A6DAC82AD83EE2404FAEF3400FBCB
:10EF3000A908121239750A08750B00780A1207EF32
:10EF40007409120A6DAC82AD83EEFAEFFBA90812C8
:10EF5000EFF212081D7401120A6D12EC32740B12DA
:10EF60000A6DE0687003A3E069700C7C01740512FF
:10EF70000A6D12EFC8800375090A900DD3E0650889
:10EF80007010851082851183E0F9121215800375C7
:10EF9000090A900DD5E060061211FD75090AA9094C
:10EFA000740F12081D7F08020563EE250AFEEF3577
:10EFB0000BFF742122E0C398FEA3E099FF22E02515
:10EFC0000AF8A3E0350BF92212ECB6A90E121A07C3
:10EFD00022E0FCA3E0FDEEFAEFFBA9082212EFE12C
:10EFE00022E0F8A3E0F58388822234FFFB900DD461
:10EFF000E0F912152D74022274F21203568C088D5A
:10F0000009740E120A6D12ECAA7410120A6DE0FE59
:10F01000A3E0FF12121BEA4B7004790A8018780AE9
:10F020001207EFEEFCEFFDEA2508FAEB350912EFC7
:10F03000EC12081D790002E668C082C083900ED2EF
:10F04000E4F0A3F07C027D047A5B7B0E1218C99079
:10F0500014B8E07004790080027901121A73120B5F
:10F060009D02FB1E74F712035674F51208AFE9FEF9
:10F07000EAFF74016E600574026E705CEF600574E7
:10F08000036F706C90148F740212F147120A4A12C7
:10F090000BAFE9F8900E6AE0A2E34019E870169011
:10F0A0000ED4E004F06404700C908761120A4A9058
:10F0B00014A2120A5674036F701B900ED5E0F974F7
:10F0C0000129F0E9C39405400C908761120A4A9027
:10F0D00014A2120A56E860107CE87D037A017B00D6
:10F0E000900E63E0F912128D740B12081D02FCE100
:10F0F00074016F704574016E90148F702E740AF055
:10F100007401120A6DE4F07402120A6D7403F09037
:10F11000876D120A4A7404120A6D120A5674081294
:10F120000A6DE412FA57120C8D80BD740A12F14771
:10F13000120A4A120BC1E9F8809B7C5D7D867A1F1A
:10F140007B8612156F8091F09014A6E0F99014A2BE
:10F150002274F4120356890890059812FA18120DB9
:10F1600047900E5112FA9C120D4180308E828F838F
:10F1700012FA11601B7A027B00121185EA4B6010B3
:10F180008A828B8374D1F0A3E50812FBA012F803E6
:10F190008E828F83A3A3A3A3A312FA18EE4F70CC81
:10F1A0007F0402056374F4120356E9FEECFF740C4D
:10F1B000120A6D12FA86750B008002050BE50BC36F
:10F1C0009E5033750A008002050AE50AC39F50EB82
:10F1D000E50BC333FCE433FDEA2CF582EB3D12F181
:10F1E000FBE50AC312FDE5E065087004A3E06509CC
:10F1F00070D679018002790002F1A0F58312FB3DFF
:10F200002274F612035612F28F7003A3E06D70178A
:10F2100075086875090E78081207EFEEFA12147F68
:10F22000740212081D801A75080275098078081288
:10F2300007EF8C088D0978081207EF12F2AA12085E
:10F240001D8005740212081D7F0202056374F61208
:10F25000035612F28F7003A3E06D70177508757571
:10F26000090E78081207EFEEFA12148574021208DC
:10F270001D801A75080375098078081207EF8C083D
:10F280008D0978081207EF12F2AA12081D80B9EA58
:10F29000FEEBFF12F2A4EF12FABEFCE439FD900E71
:10F2A00051E06C22EE2413F58222EE240E12FB456F
:10F2B000FD7C8012FA0012FB45F9121497740422A7
:10F2C00074F612035674FE1208AFEAFEEBFF8510C7
:10F2D00082851183E4F0A3F012F2A4EF12FAE7FAA8
:10F2E00088828983A3A3E0F9750800750900600589
:10F2F000C394F140057509828029900E51E06A702F
:10F3000003A3E06B701A851082851183AA82AB83F8
:10F3100012112BE9F50812FB25700875098380038B
:10F3200075098085108285118312FA7DA909EEFA8C
:10F33000EFFB12148BE508600812FB25600312FA3C
:10F340003602F24374F21203568A0C8B0D750800D4
:10F3500075090012FAB3120D47EA6E7002EB6F7076
:10F3600012121137E914F50879017A9E7B0E1211F9
:10F370003D8003750980E50C240E12FAABF50A787E
:10F380000A1207F3750A9E750B0E780A1207EF78BA
:10F39000081207F38E0A8F0B780A1207EFE509F5BA
:10F3A0000878081207F312FAD1F582E50D12FA0C6B
:10F3B0007A057B8012149102FE6F74F6120356E9EF
:10F3C000FE7F00802F8A828B8312F9C1F9E5082421
:10F3D00000E439F509EF33F8E433F9EC28F582ED70
:10F3E00039F583E508F0A3E509F0EA24020A0AEBFF
:10F3F0003400FB0FEFC39E40CC02F24874F01203BE
:10F400005674F51208AF7403120A6D12FA9C740256
:10F41000120A6DE4F07409120A6DE4F0A3F07407A7
:10F42000120A6DE4F0A3F07403120A6DE0241312C3
:10F43000FB0B12F7FB850A82F58312FB7D2400F596
:10F4400008E439F509850A82850B83A3A3E0FA85D0
:10F450000A82850B83A3A3A3E0F9EAFEE439FFE562
:10F460000A2404F50AE50B3400F50BAA08AB0912CF
:10F470000DA7E96401703C7403120A6D12F80E12B4
:10F4800007F3E4F508F50978081207EF7808120782
:10F49000F3900E5112065375088078081207F37422
:10F4A0000A120A6D12F7EF120A6D12F81912081DEE
:10F4B00002F7D0AA08AB09120DA7E9700E900E5101
:10F4C000E065087004A3E0650970AC12F7D5880FF9
:10F4D000602EC333FAE433FB1211F17409120A6D82
:10F4E00012FA9C7409120A6D12FB2B601374091234
:10F4F0000A6D12F7E5A90F12142B8A0A8B0B8003F1
:10F50000750F0012F7D5880E602AC333FAE433FB77
:10F510001211F17407120A6D12FA9C7407120A6D27
:10F5200012FB2B600F7407120A6D12F7E5A90E1279
:10F53000142B8003750E00900598804DE4F0A3F025
:10F54000AA0CAB0D7405120A6D12FA11F8A312F889
:10F550000385108285118312FA11C0E07402120A29
:10F560006DE0F8749E28F582740E12FB79D0E0F0FD
:10F570007402120A6DE004F0E50BA2E0500312FAE7
:10F58000367405120A6D12FE3112FA867405120ADB
:10F590006D12FA517405120A6D12FB2B700302F7FB
:10F5A000507405120A6D12FA22E8FAE9FB8A828B7E
:10F5B00083E060CD7405120A6D12FE25A3E0A2E07F
:10F5C00050BF7405120A6D12FA1E12FA83E8FCE9A4
:10F5D000FDEC4D8A828B836019E0FA79018C828D73
:10F5E00083121A8A85108285118312FA9C750B0189
:10F5F000800F12FA8385108285118312FA51750BE0
:10F600000012FB25700302F57885108285118312A4
:10F61000FA1EA3E06E7003A3E06F600302F578E5C5
:10F620000F7004E50E605B85108285118312FE3336
:10F63000A3A31206537402120A6D12FE3BE0FC747F
:10F640000B120A6D12FB01A90F12140D740212089D
:10F650001DE9702E85108285118312FA311206532E
:10F660007402120A6D12FE52E0FC7409120A6D1245
:10F67000FB01A90E12140D740212081DE970030299
:10F68000F578E50E250FC333240AFA7B00121185A5
:10F690008A0C8B0DEA450D700302F5518A828B832B
:10F6A00074D2F07403120A6D12FB548A828B831297
:10F6B000FA4F8A828B83A3A3A3A3E50F12FD6EA347
:10F6C000A3A3A3E50EF0EA2405FAEB3400FBE50F53
:10F6D0006033E50C240AF8E50D3400F98A828B8347
:10F6E00012FA517409120A6D12FE611207EBE50F4E
:10F6F000C333FCE433FD8A828B8312FB0112FB3798
:10F7000012081D80088A828B83E4F0A3F0E50C24A4
:10F7100008F582E50D12FB79E50E700302F53CE574
:10F720000FC333F8E433F9E50C28F8E50D39F9E8AF
:10F73000240AFAE93400FB12FA9C7407120A6D12CB
:10F74000FE611207EBE50E12FB3112081D02F540B7
:10F750007402120A6DE060497403120A6D12F80E09
:10F760001207F375089E75090E78081207EF7405E5
:10F77000120A6D12FA961207F3900E511206537583
:10F78000080078081207F3740A120A6D12F7EF12D4
:10F790000A6D12F81912081DE970117CF87D868037
:10F7A000047C8F7D867A3F7B8612156F7409120A5E
:10F7B0006D12FB2B60087409120A6D12FA3C740773
:10F7C000120A6D12FB2B60087407120A6D12FA3CC4
:10F7D000740B02FA5F850A82850B83E0F8A38582A9
:10F7E0000A85830B22E0FCA3E0FDAA0AAB0B22E012
:10F7F0002402FCA3E03400FD740A22E0F50AA3E031
:10F80000F50B2212FE2C12FA72F912119122E02449
:10F810000E12FB5BF50878082212FA697A067B80E3
:10F8200012149174072274F012035674F41208AF84
:10F830008A0A8B0BECFEEDFF740B120A6D7403F059
:10F84000120A6DAA82AB831218C9120D41EAFCEBB1
:10F85000FD7403120A6DAA82AB831218C3E9600E0D
:10F8600012F9B9F87403686010740168600B8510B0
:10F8700082851183748402F9688E828F83A3A3A387
:10F88000A3A3A3A3A3E0F96021C394F1501CEE2429
:10F8900014F508EF12FD337403687019850882852A
:10F8A0000983E06005C394F1400B851082851183C4
:10F8B000748202F968EE240BF50EEF3400F50FE5C3
:10F8C0000A240CF582E50B12FAAF64217002A3E062
:10F8D00070738510828511837487F0120B25901E3A
:10F8E00022E493F8740193F9C3EA98EB99507A12E1
:10F8F000FA901207F312FAF08E828F83A3A3A3A3C8
:10F90000A3A3A3A3E0F9121A01740112081DE97060
:10F9100058851082851183E4F01213A712F9B96497
:10F920000370467401120A6DAC82AD83AA0EAB0F50
:10F930001219F5E970337D007C007900AA0EAB0F37
:10F94000121467802412FA901207F312FAF01219B7
:10F95000FB740112081DE98510828511837007E48C
:10F96000F01213A780037488F012FCA4E50B12FBBD
:10F970007912FA961207F37401120A6D85820885CE
:10F98000830978081207EFE50A240CF582E50B12CB
:10F99000F9BE4480F50978081207EF7901E50A24D9
:10F9A00002FCE50B3400FDE50A240FFAE50B12FA20
:10F9B000E012081D740C02FA5F12FAA2E02212FA99
:10F9C00043E0F508A3E022C082C08374F31208AFBD
:10F9D000851082851183E4F004120A6D12FA9C747A
:10F9E00003120A6DAA82AB83120AB98510828511AF
:10F9F00083AA82AB83120AE9740D12081D02FB1E52
:10FA0000EE2402FAEF3400FBEE240F2212FB48F939
:10FA10002212FA722212FD47E0FEA3E0FF2212FA40
:10FA20002A2212FA2A12FA8A22F8A3E0F58388829F
:10FA30002212FE56A32285108285118312FB051225
:10FA400011F7223400F58322EE240412FB9522A341
:10FA5000A3E8F0A3E9F02212FAC9AA82AB8322122A
:10FA6000081D8014F812FB5C22E0240FF812FB60E2
:10FA7000F922E012FA29E0227F08020563E0FCA3E4
:10FA8000E0FD22A3A3A312FA8A22E0F8A3E0F92260
:10FA9000850882850983E0F508780822EAF0A3EB5F
:10FAA000F02212F2A4EF3400F58322F582E50D1264
:10FAB000FB482212FCC812FABEFEE439FF2212FCF7
:10FAC000D2FAA3E0F9EA240022F08510828511839E
:10FAD00022E50C2402FCE50D3400FDE50C240F2288
:10FAE0003400FB12FB4E2212FCCEFCA3E0FBEC2206
:10FAF000AC0EAD0F8E828F83A3A3A3A3A3A3A3A356
:10FB0000A312FB0522E0FAA3E0FB2212FB0F22F86E
:10FB1000A3E012FB16223400F98882898322D08365
:10FB2000D0820207CF85108285118312FA8AE849B4
:10FB300022C333FCE433FD121161740322E0F508A3
:10FB4000A3E0F50922F582EF3400F583E0221214D8
:10FB50006174052212FE4312FA8A22F812FB602217
:10FB6000A3E03400F988828983E022F08A828B83C3
:10FB700022E508240CF582E50912FA4322E0FAA3F3
:10FB8000E0F9EA223400FB12FB8B221218C9EE24A2
:10FB90000812FB9522FEEF3400FF8E828F83E02255
:10FBA00012FD38E0F8A32274F61203568C088D0972
:10FBB00012FA1512FD7F7014EEFCEFFD12FE0DC05F
:10FBC000E0E508241412FB75D0E0800312FD60F01C
:10FBD00002F24874F2120356EA2413FEEB3400FFDB
:10FBE000EA2410F582EB12FAAFC3940C400E8E8219
:10FBF0008F83E0240B12FA64F50A8003750A00E58E
:10FC00000AC333F8E433F9E8240DFAE912FE1E8A38
:10FC1000088B09EA450960758E828F8312FD438A3D
:10FC2000828B8312FD1A7065EEFCEFFDEA24030A55
:10FC30000A0AEB12FB8412FEF112FC9E240BF8E57B
:10FC4000093400F9E8FAE9FB8A828B83E4F0E50ADB
:10FC5000603BE508240D0808E5093400F9AC0A8E7C
:10FC6000828F8312FC9812FD3EC0E012FB71D0E03F
:10FC700012FD738E828F83E0F50AA3E0FBE50A880C
:10FC800082898312FCAB12FC941CEC70E6AA08ABD0
:10FC90000902FE7412FDDB22E08A828B832212FDB0
:10FCA000CFE50822E50A240EF58222F0A3EBF0123C
:10FCB000FCB322E824020808E93400F92212FCC24D
:10FCC000E022F08882898322EA12F2A5EB2212FC5C
:10FCD000D2223400F583E0F8A3E0F988828983E03A
:10FCE000227F0102056374F7120356EA2413F8EB2E
:10FCF00012FB16E0FAA3E0F5838A8212FDFD12FCE6
:10FD0000BDF8A3E0F988828983A3E0FA8882898319
:10FD1000A312FDF312FA5202FCE112FD1E2212FDA3
:10FD20002222F08E828F83A3AE82AF832212FB6BDE
:10FD3000A3A3223400F50922F08E828F832212FDC4
:10FD400077E02212FD552212FD4B22EA12F2A5EBBA
:10FD50003400F58322E0FEA3E0FF8E828F83E02251
:10FD6000E0FCA3E0F9EC8A828B83F0A3E92212FD88
:10FD70002DA32212FD772212FD38A30EAF8322EEAF
:10FD8000FCEFFDAA08AB0912FB8B8508828509836D
:10FD9000A3A3A3A3A3A3A3A312FE0385088285099B
:10FDA00083A3A3A3A3A3A3A3A3A312FDCF8E828F98
:10FDB00083E0F8E50812F2A5E50912FA43E812FD1E
:10FDC00077E508240BFAE5093400FB74036822F098
:10FDD000A3E912FDD622F012FDDB22EE24020E0E64
:10FDE000EF3400FF2233FCE433FDE82CF582E93DDB
:10FDF000F58322A3E0F9EA8C828D83A322E08C8232
:10FE00008D832212FD22E0FAA3E0F9EA221218C93A
:10FE10008E828F83A3A3A3A3A3A3A3A3E022340072
:10FE2000FB1211F122E012FE2A22F8A312FA2BA3F0
:10FE300022E0F812FE2BA3A3A3A32212FE43A3A346
:10FE4000A3A32212FE4722E0F8A3E0F5838882A351
:10FE5000A32212FE562212FE47A3A3A3A3A3A3A389
:10FE60002212FB3D750A0078082212FD4BE0227435
:10FE70000712081D7F0602056374F61203568C08EC
:10FE80008D0912FED1850882850983120A5612FA5D
:10FE900048FAE5082404F8E5093400F9EA8882897B
:10FEA0008312FD1AC39406500512FEFE801F74FED5
:10FEB0006A600574FF6A701612FEFEA312FD738855
:10FEC000828983E0F4700712FEE2F0A3E9F002F207
:10FED0004812FE6AFEA3E0FF7904EEFAEFFB12116E
:10FEE00073228E828F83E012FEF1A3A3A3A3A3A3A8
:10FEF00022FAA3E0F9EA850882850983A322E08536
:10FF00000882850983A3A3A3A3A322D083D082025E
:10FF100007CFC082C0838019198C828D83E08A82CA
:10FF20008B83F0A3AA82AB838C828D83A3AC82AD3A
:10FF300083E970E480D5C082C083801D198A828BDA
:10FF400083E08C828D83F08A828B83A3AA82AB8329
:10FF50008C828D83A3AC82AD83E970E080AD74F7B1
:10FF6000120356EAFEEBFF8908E970031214FD8EB6
:10FF7000828F83E0F5D9A3AE82AF831508E50870C0
:10FF8000EE7F0102056374F7120356EAFEEBFF8968
:10FF900008E970031214FDE5D98E828F83F0A3AEB9
:10FFA00082AF831508E50870EE80D6C082C08374E6
:10FFB00070900F67F074B1900F68F0900F69E05483
:10FFC0001FF0741D900F6BF07442900F6CF0747002
:10FFD000900F6DF074B2900F6EF0900F71E0541F9F
:10FFE000F0741E900F73F07412900F74F08000D0B4
:10FFF00083D0820207CFC082C083120E9102FFEF2E
:020000040001F9
:1000000074F212035674F41208AF8A0C8B0D8C0A2A
:100010008D0B8908741A120A6D1289857C0C7D007B
:100020007900851082851183AA82AB8312116D74C9
:1000300009120A6DE4128138A3A3A3A3A3A3A3E02A
:10004000C0E07408120A6DD0E0F0850A82850B8347
:100050001281CAF0901496E024FFF50AA3E034FF61
:10006000F50B850C82850D8312896775091E780949
:100070001207F3780C1207EF780A1207EF85080AC7
:10008000E50A2401F50AE43400F50B780A1207EFBB
:100090008E0A8F0B780A1207EF900F27E0F97C90F9
:1000A0007D147409120A6DAA82AB831211197409A6
:1000B00012081D740C028BA174F212035689087485
:1000C0000E120A6D128E7B7410120A6D1282B0121B
:1000D0000A6DE0F5099014961287B2AE0880238568
:1000E0000A82850B83E0850C82850D831281388519
:1000F000820A85830B850C82850D83A385820C85FE
:10010000830DEEFF74FF2F1E0470D4E509600575A2
:100110000A408003750A00E50A441E900F27F08804
:100120000A890B780A1207EFA9081289A612081D7E
:10013000900F27E4F0028BA4F0850A82850B83A33D
:100140002274F412035674F71208AF8A088B0989D7
:100150000B8C0A901496128985AC08AD097AD37B72
:10016000041218C3E970127408120A6D740F128118
:10017000EF74FDF0A374FF800E7408120A6D740210
:10018000F0900E511281CAF0AC08AD09EEFAEFFB07
:100190001218C98A088B09AE08AF098E828F83E5D1
:1001A0000BF0A3E50AF0E4F508F50978081207EF6B
:1001B000790A7402120A6DAC82AD837AD67B0E1274
:1001C00089A612081D740902899A128E7F851082F1
:1001D000851183E8F0A3E9227402120A6DAC82ADA6
:1001E000837AD67B0E1289A612081D7409800BF043
:1001F000851082851183221289A612081D7F0202B2
:10020000056374F01203568A0E8B0F8C088D09E972
:10021000FE7410120A6D1282B0120A6D1287B27447
:1002200014120A6DE0FB7415120A6D12897F128E8A
:1002300078EE2BC3332406FAC3944F400479108020
:100240006C88828983E508F0A3E5091282DFE50B5B
:10025000F0A3EE1284E560197F00EFC333F508E4E4
:1002600033F509E50C2508F50AE50D1282B69E4026
:10027000E9EB888289831284E560177F00EFC3333E
:10028000F508E433F509EC2508F50AED1282B69B72
:1002900040EB75080675090078081207EFEAF9AC1B
:1002A0000EAD0F7AD67B0E1289A612081D0289ECBC
:1002B0001289567412223509F50B850A82F58312CC
:1002C0008A25A882A983850A82850B831282D30F8F
:1002D000EFC322A31282D822128A2508A98322F012
:1002E000A3E50AF0A32274F612035674F71208AFBE
:1002F000E9FE7408120A6D1283251289BBEA128383
:1003000036EBF0901496E02402FAA3E03400128950
:10031000ACA3A3EEF075081375090078081207EF77
:10032000790B0281D8740FF085108285118374FDDA
:10033000F0A374FFF022F012833B229014961289EE
:10034000C6A32274F01203568A0C8B0D7508007533
:100350000900EA240CF50EEB3400F50F850E82F54A
:1003600083128C61EA4B70047C0880027C02E50CED
:100370002413F582E50D128E63128E7BE82CF58234
:10038000E9128A01F50AEA4B701D88088909AC0850
:10039000AD097AD37B041218C3E9700302844E902E
:1003A0000E51128985802288828983E0FAA3E0F9C0
:1003B000EA2400FEE439FF900E51E06E7003A3E0E2
:1003C0006F70067508D375090474FE6E700374FFB0
:1003D0006F607BE50845096075128C5EE50A601761
:1003E0007401650A60117402650A700E850E8285BB
:1003F0000F83128C587003E4800274808A828B838E
:10040000128A52AC08AD091218C9EE8A828B83F0A9
:10041000A3EFF0900F277410F0850E82850F83E014
:10042000F508A3E04480F50978081207EF790BE599
:100430000C2402FCE50D3400FDE50C240FFAE50D5B
:100440003400FB1289A612081D900F27E4F00289E0
:10045000EC74F6120356740A120A6D128985128E14
:1004600078888289831284DD1284E58E828F83E00E
:10047000541F88828983F0A308128A31A31284EC66
:100480001284EDA31284FC1284FC128A37128A3F74
:100490002408FCEF3400FD8C828D83128A2D8C821F
:1004A0008D831284EC128A3F240B128E60128A46CE
:1004B000240CF582EF128A0188828983F075080284
:1004C00075098078081207EF7910EA2402FCEB34F2
:1004D00000FDEA240FFAEB3400FB0281F7E4F0A3FD
:1004E000ECF0A3ED22F0A3A882A98322A31284F149
:1004F000221282D88E828F83A3A3A3221284F1A317
:10050000A32274F6120356EAFEEBFF740A120A6D78
:100510001287BA128C61128A4B128BB78882898338
:100520001289DF540FF9740C7808120A10E508C418
:10053000498A828B83F07508037509807808120751
:10054000EF7905EE2402FCEF3400FDEE240FFAEF04
:10055000808574F012035674FD1208AF7401120AFC
:100560006D128A13E9851082851183F0128C5EEC7E
:100570002409F50CED3400F50DEC2406F50AED34F4
:1005800000F50B851082851183E0702BEC4D602700
:10059000850C82850D83C082C083850A82850B838A
:1005A000E0D083D082F8E028C333240CF9C3944F01
:1005B000400779100286ED79048510828511831237
:1005C0008A6A900E51128BBB900E52128A59E9C35F
:1005D000940550030286BE74FC29F0A30A0AAB837B
:1005E0008C828D83128BBB8C828D83A3AE82AF8372
:1005F0001286FAEC2403FEED3400FF8E828F831204
:1006000086FA8C828D83A3A3A3A3A3E0C454F08AAB
:10061000828B83F0A30AAB83850A82850B83128BBE
:10062000BB850A82850B83E060427800EC2407F5E5
:100630000EED3400F50F8027E8C333FEE433FF8569
:100640000E82850F83E02EF508A3E03F128A6585B0
:100650000E82850F83E02EF508A3E03F1286F08519
:100660000A82850B83E0FEE8C39E40CC850C828520
:100670000D83128A6A850C82850D83E060427800C2
:10068000EC240AFCED3400FDECFEEDFF850C8285C8
:100690000D83E0FCE8C39C5027E8C333FCE433FD42
:1006A0008E828F83E02CF508A3E03D128A658E824E
:1006B0008F83E02CF508A3E03D1286F080CEE4F0B5
:1006C00075080475098078081207EF7403120A6D23
:1006D000E02402FCA3E03400FD7403120A6DE02460
:1006E0000FFAA3E03400FB1289A612081D0289E765
:1006F000850882F58312870508221287068E828F6D
:100700008312870522A3E08A828B83F0A30AAB833E
:100710002274F012035674FF1208AFE98510828527
:100720001183F0EAFEEBFF8C0E8D0F7411120A6D2F
:10073000E0F87412120A6D12897F7414120A6DE0C7
:10074000F97415120A6DE0F508A31289CF750C042F
:1007500074066E700374806F7005750B10800375DE
:100760000B00E88A828B831284DEF0A3E9128A529E
:100770006017740429F50C750A0078081207EB89D4
:1007800008AC08128BC512081DE50B900F27F08EE0
:10079000088F0978081207EFA90CAC0EAD0F740290
:1007A000120A6D1289A212081D900F27E4F00402AC
:1007B00089E9E0F50CA3E0F50D22128E7F901496E6
:1007C0002274F612035674FF1208AFE98510828571
:1007D0001183F0ECFE740B120A6D128E7B740D12F5
:1007E0000A6D1289DF128815EEF0128815A3E8F061
:1007F000128821128337A3A3E4F078081207EF7957
:1008000004EAFCEBFD7402120A6D1289A212081DA3
:1008100074010281FA901496E0FCA3E0F5838C82C7
:100820002212833BA3E9F02274F012035674FC12E7
:1008300008AF7402120A6D128A137401120A6DE96C
:10084000F0ECFEEDFF7414120A6D1289DF741612BB
:100850000A6DE0F50E7419120A6DE0F50F9014960A
:10086000128956E50E250FC333240F85108285119A
:1008700083F0C3944F40057910028951120D47EA65
:100880006E7002EB6F60057902028951EE850A8273
:10089000850B83F0A3EF12895E120D41EAFCEBFD9C
:1008A000AA0AAB0B1218C97401120A6D128A59E513
:1008B00008F0A3E509F0A3E50E12895E7C0080290B
:1008C000ECC333FAE433FB7417120A6DE02AFAA37F
:1008D000E03BFB8A828B831289678A828B83A31217
:1008E0008A2185820A85830B0C850A82850B83A366
:1008F000A882A983ECC3950E40C6850A82850B8326
:10090000E50FF0880A890B7C008023ECC333F8E400
:1009100033F9741A120A6DE028F8A3E039F98882D5
:10092000898312897488828983A31289740CECC329
:10093000950F40D775082075090078081207EF74E5
:1009400002120A6DE0F97404120A6D12898B120802
:100950001D74040289E9E0F50AA3E0F50B22F0A377
:1009600085820A85830B2212896B22E0850A8285A3
:100970000B83F02212896BA385820A85830B22E008
:10098000FCA3E0FD22E0FEA3E0FF22E0FCA3E0FDEB
:100990007AD67B0E12145B74022212081D7F0402A9
:1009A0000563AA82AB8312145B740222FB1218C97E
:1009B00012833BA3A3A3A3A3A3A3229014961289FB
:1009C000C2221289C622E0F8A3E0F583888222E0E1
:1009D000F509901496E0FAA3E0FB223400F583E0D9
:1009E000F508A3E0F50922740312081D7F0802052B
:1009F000633400F98882898322E50E2410F582E5AC
:100A00000F3400F583E022F02401FAE43400FB12F5
:100A100011F122EAF0A3EBF022EAF0A3EBF074026A
:100A200022128A2522E088828983F0A3221282D4AE
:100A300022A9838E828F831282D38E828F8322A3F8
:100A4000A3A3A3A3A3A31282D4EE228A828B831230
:100A500084DDF0A3AA82AB8322128A5D22E08A821F
:100A60008B83F0A322850882F583128A5DAA82AB6C
:100A7000832274F212035674F61208AF7405120A38
:100A80006DE9F07408120A6D128A137404120A6D6B
:100A9000ECF0ED851082851183F07418120A6D78E0
:100AA00008120A2E741C120A6D1287B2741E120AE2
:100AB0006D128985851082851183E0240AC0E07457
:100AC00001120A6DD0E0128A077402120A6D128AAE
:100AD00019120A6D128C5870057910028B9F7402DE
:100AE000120A6DE0240108A3E03400F97406120A2A
:100AF0006D128E727406120A6D128C617404120AE1
:100B00006D128A6A78081207E7121A7F74041208B5
:100B10001D8A828B83E50CF0A3E50DF0A3EEF0A314
:100B2000EF128A52851082851183128BBB85108249
:100B3000851183E0601B7420120A6D1289DF750A2B
:100B40000078081207EB7403120A6D128BBF1208AB
:100B50001D7406120A6D1287BA128E727422120A5E
:100B60006DE0900F27F07508387509807808120736
:100B7000EF7403120A6DE0F9740A120A6D12897F8C
:100B80007407120A6D1289A212081DE9FE7402127E
:100B90000A6D128C61128BA9900F27E4F0EEF974A4
:100BA0000A12081D7F060205631211F7901496744D
:100BB000D8F0A3740EF0228882898312870622E07F
:100BC000FC128BC5227D0012116174032274F21293
:100BD0000356890AEAFEEBFF900F288008880889EF
:100BE0000988828983128C58601F88828983A3A315
:100BF000E0650A70E888828983A3A3A3E06E70038E
:100C0000A3E06F70D87900804C7A057B001211F157
:100C10008A0C8B0DA80CA90DE8496037888289835E
:100C2000A3A3E50AF088828983A3A3A3EEF0A3EF30
:100C3000F088828983E4F0A3F0900F28128C61EA97
:100C40004B600B850882850983128E7280B7900FE6
:100C50002880F67910028BA4128E7FE84922901426
:100C600096E0FAA3E0FB2274F01203568A0E8B0F73
:100C7000750800900F28028D1E850C82850D83A3B8
:100C8000A3A3128E7BE50E240C1289FD687003A3CA
:100C9000E0696003028D181289F92415FAE4340022
:100CA000FB1211858A0A8B0BAE0AAF0BEE4F606800
:100CB000850E08850F09750A0078081207EB7C1568
:100CC000128BC512081D1289F96032EE2415FAEF55
:100CD0003400FBEE2413128E60128A13E50E2413E7
:100CE000F582E50F1289DB78081207EBE50E241078
:100CF000F582E50F128E63128BBF12081D8E828F54
:100D00008374D3F0EEFAEFFB850C82850D83A3A3E9
:100D1000E0F9121191750801850C82850D83128707
:100D2000B2E50C450D6003028C79A9080289EC74C8
:100D3000F612035674EB1208AF7E00740A120A6DA5
:100D40007402128E68A3A3128E7B7402120A6D12B3
:100D50008E72EA2415F582EB128A01C0E0740B1240
:100D60000A6DD0E0128E68128E7B740C120A6D121E
:100D70008E72EA2419F582EB128A01C0E0740E1219
:100D80000A6DD0E0F0EA241FF582EB128A0114C04C
:100D9000E07410120A6DD0E0F0EA2421F8EB128919
:100DA000F1E02401FCA3E03400FD7413120A6DECA1
:100DB000F0A3EDF0888289831289BEE0C0E0740F51
:100DC000120A6DD0E0F0EA2412F582EB128E631263
:100DD0008E7B7411120A6DE8F0A3E91281EFAA82EA
:100DE000AB831214AFE9FC80010E8E087509007404
:100DF00002780812098874F72508F8741C3509F977
:100E000088828983E493C0E0740193F583D082AA39
:100E100082AB8374FF6A700374FF6B602E740C12D4
:100E20000A6DE06A7003A3E06B70BE8510828511C5
:100E300083AA82AB8388828983A3A3E493C0E074EE
:100E40000193F583D082121A8A8010EC700D851000
:100E500082851183AA82AB8312138974150281FAE9
:100E6000F582EF3400F58322F08A828B83A3A3A35B
:100E7000A322E8F0A3E9F022901496128E7F22E0DC
:100E8000F8A3E0F92274F7120356E9900E63F0908C
:100E90000E597402F0900E5174FEF0A304F0120D7E
:100EA0004112131D1213FB7A907B1412110190143E
:100EB0008FE060097A007B00121311800D7CF47DB5
:100EC000017B327A0079081215C312132F0295772D
:100ED00074F6120356EAFEEBFF5480703AEEA2E07D
:100EE000504E90148F7401F07C0F7B0F900E66E0D3
:100EF000FA900E68E05407F9121401D2F0A2903073
:100F0000F001B39290EE6401FAEFFB805D121323BF
:100F1000AA08AB0912118B900E63E0F91211978A9F
:100F2000088B09A909EA4970E4EEFAEF648080DAD7
:100F30005410600D90148FE0F9121407EE641080C5
:100F4000C7EE54086006EE6408FA801EEF54026093
:100F500005EF640280B4EE5404600BC2AF75C9ABF8
:100F600075C95B0080FD7A007B0080057402120861
:100F70001D7F0202056374F612035674FE1208AF59
:100F8000851082851183EAF0A3EBF090148FE07056
:100F90000579001214CD1213AD900E6AE090045B37
:100FA000F090148F7401F012134185108285118323
:100FB000AC82AD837A8F7B1412134D90148FE07046
:100FC000047902803412131712117F851082851163
:100FD00083EA547FF8E028F8A3E03400F9E82464B9
:100FE000FEE93400FF1214BBEEFAEFFB12138F90F0
:100FF0000E6AE0F9120DA17901028F6CC082C083E4
:101000009014B8E0700E900E667402F0900E68E0D6
:1010100054F8802E6401700A900E68E054F8440180
:10102000800DE064027009900E68E054F84402F00C
:101030007A027B04120E8BE9900E667003E4800244
:101040007403F0029490E0F8A3E0F9E822C082C0B3
:1010500083121551E96401700590148FE4F0029435
:101060009074F012035674FF1208AFEAFEEBFF8E85
:10107000828F83E014603E1470030291F5147003B4
:1010800002920724E9600B2447600D24D6600F020A
:1010900092311214B5029231121329029231900E3C
:1010A00096129046497003029231E0F583888212CD
:1010B0001A8A02923190148FE06402600302923126
:1010C0009014B8E064016008E064026003029231A9
:1010D0008E828F83A3E060030291DC90148DE0C3C5
:1010E000940350030291DCEE2403F50EEF3400F577
:1010F0000FEE2402F50AEF3400F50BEE2404F50898
:10110000EF3400F509900E66E0704490148F74037C
:10111000F012139B900E6AE0F50C780C1207F38521
:101120000882850983E0F9850A82850B83E0FC85C6
:101130000E82850F83E0FBEC2400E43BFDEE2406E9
:10114000FAEF3400FB120BCD740112081D807A6493
:1011500003707C90148F7404F0900461E064FE705E
:1011600003A3E0F4701412117F900461EAF0A3EB82
:10117000F07A617B0479531218E190046EE064FE0A
:101180007003A3E0F47021850A82850B83E0FA8561
:101190000E82850F83E0F9EA90046EF0A3E9F07AFD
:1011A0006E7B0479501218E18510828511837401D9
:1011B000F0AA82AB8379521218E1850882850983EF
:1011C000E0F97A5B7B0E120BC7E96003129444903E
:1011D0000E6AE0A2E3505A12942E805590148EE0CD
:1011E000604F90148DE004F012117FEA2464FAE459
:1011F0003400FB80399014B8E064016005E06402BB
:10120000702F121335802A9014B8E064016005E055
:101210006402701D900E67E4F0900E6604F0900E6C
:101220005A12923B9014A67402F07A007B001213BB
:101230008F740112081D7F08020563F07C827D0413
:101240007A5B7B0E1218C92274F612035674EB12E5
:1012500008AF1298B7F508A3E0F50978081204D191
:10126000020021002200A292008001807292000000
:10127000C0921214498A088B09AE08AF09EE4F607C
:101280003F8E828F83E07011EE2403FCEF3400FD6B
:10129000A3E0FAA3E0FB12143DEEFAEFFB1211F704
:1012A000801E851082851183AC82AD831214438524
:1012B0001082851183AC82AD83EEFAEFFB121437F6
:1012C0007415028F6EC082C0837A011292E47A0094
:1012D0001292E47A217B001292E67A227B0012922B
:1012E000E60294907B80900E63E0F91214A92274B8
:1012F000F612035674FE1208AF90148FE064036078
:1013000015E0640A60030293BA900E68E054076423
:101310000160030293BF900E64E070171298E99089
:10132000148FE0640370031213A190148F7406F0FD
:1013300002942B900E66E064017031900E67E00419
:10134000F0C394034026129453700374FF69600A3B
:1013500074FE68700374FF697006900E66E4800B7B
:10136000900E667403F0900E5A7401F0120D478AC5
:10137000088B0974FE6508700474FF6509700D9090
:101380000461E064FE7003A3E0F4602385108285AD
:10139000118374FEF0A304F090046114F0A304F030
:1013A000851082851183AA82AB8379531218E1904C
:1013B000148D7401F01294448071E06404705E90A6
:1013C0000E64E0701312945F900E6AE0A2E3500383
:1013D00012942E1213A18053900E66E0640170D512
:1013E000900E67E004F0C3940450281294537003E5
:1013F00074FF69600A74FE68700374FF6970079077
:101400000E66E4F080AF900E667403F0900E5A748E
:101410000180F090040AE0640160E480989004ADDB
:10142000E0640270061213A11298E9028F6C7A0030
:101430007B00120D657A007B00120D6B7A007B0039
:10144000120D712212117FEA547F2464FA7B00127C
:10145000138F2290046EE0F8A3E0F974FF682290E5
:10146000148F7406F07A107B00900E63E0F912116D
:10147000B5227B0012125D740422C082C083EAFC94
:10148000EBFD7A047B00900E63E0F912128D800070
:10149000D083D0820207CF74F612035612955812E9
:1014A00007EF7C017D007A857B00121257740212CF
:1014B000081DE9702078081207EF7508017509000A
:1014C00078081207EF7C007D007A857B001212639A
:1014D000740412081D028F7174F6120356E9FE900F
:1014E0000E657401F06E70037403F075086575097C
:1014F0000E78081207EF75080175090078081207C1
:10150000EF7C007D007A85129472028F6E74F61261
:1015100003568C828D83E4F0A3F0900E65E0A2E088
:101520005033A2E1500C8C828D837488F0A3741325
:1015300080058A828B83E4F01295581207EF7508B4
:101540000175090078081207EF7C007D007A85128A
:10155000947212081D028F71900E65E4F075086593
:1015600075090E78082274F71203561213477A8809
:101570007B1312133B80007F0102056312976C807E
:10158000F674F012035674FE1208AF7401120A6D5D
:10159000E9F0EA851082851183F08C0E8D0F8B8225
:1015A000AE82EEFA7B001211858A0C8B0DEA450D96
:1015B000603FEE6020E50E450F601A850E08850F2E
:1015C00009750A0078081207EBEEFC7D0012116124
:1015D000740312081D851082851183E0850C8285B5
:1015E0000D83F0AA0CAB0D7401120A6DE0F9121113
:1015F00091740202923374F012035674F01208AF21
:10160000851082851183EAF0A3EBF0890B750A003F
:10161000750800851082851183E0FEA3E0FF75093F
:10162000008020E0640270087401687003750A018C
:10163000E50860030296FD0509EE24161298BEFE29
:10164000A3E0FFEE2407F50EEF3400F50FEE240DB6
:10165000F50CEF3400F50DE509C3950B507F9014A0
:10166000B6E0F47003A3E0F460158E828F83E0F897
:10167000A3E0F99014B6E0687003A3E06970B87A4B
:101680005B7B0E120E8BE96401700EAC0CAD0D7A13
:101690005B7B0E1218C3E9609E8E828F83A3A3A387
:1016A000A3A3A3E06091850E82850F83E0F89004E8
:1016B0005EE06870828E828F83A3A3A3A3A3A3A3FB
:1016C000A3E0F89014A7E0686033E06401600302CF
:1016D0009623740268600302963002962DE50A6034
:1016E0000C0508E508C394025003029613E50B6548
:1016F00009700A7403120A6D7401F08058740312A1
:101700000A6DE4F08E828F83E0C0E07404120A6DEB
:10171000D0E0F08E828F83A3E0C0E07405120A6DE2
:10172000D0E0F08E828F83A3A3E0C0E07406120A9B
:101730006DD0E0F0850E82850F83E0C0E074071263
:101740000A6DD0E0F0AC0CAD0D7408120A6DAA82DF
:10175000AB831218C97402120A6DAC82AD837B0E82
:101760007A0112976C79007410029233900E63E044
:10177000F9121359227A0179041215BD7A007908F9
:101780001215BD90148FE02274F7120356E9900EE3
:1017900064F0700A129775700C7403F080077A0475
:1017A00079041215BD7C007D007B027A0202957CD3
:1017B00074F7120356EAFEEBFF120D41EAFCEBFD53
:1017C000EE2402FAEF3400FB1218C3E9640170063C
:1017D000EE240B12982C02957774F6120356EAFE4B
:1017E000EBFF8E828F83A3A3A3A3A3A3A3A3A3A38F
:1017F000E064017008EE240C12982C802C120D4D20
:101800008A088B09A808A9098E828F83E068700373
:10181000A3E0697014EE240B1298BE640160D690A8
:101820000E68E05407640260CC028F71F582EF34D9
:1018300000F583E0F91213532274F7120356E9FE00
:1018400074016E700E120E197C007D007B027A030B
:1018500012976C0295770207CF0207CF74F6120336
:10186000561298B7F8A3E0F954807048EE240B1292
:1018700098BE70407413687001E96038E8F508E9B3
:101880004480F50978081207EFE4F508F5097808AF
:101890001207EFEE240E1298BEFD7C84EE24020A9D
:1018A0000AEF3400FBEE240F1298BEF9121497745D
:1018B0000412081D028F71EAFEEBFFEE240CF58284
:1018C000EF3400F583E022C082C083EA4B6012EA65
:1018D000FCEBFD7A017B00900E63E0F912128D8023
:1018E000057A011298EB0294907A107B00900E63B7
:1018F000E0F91211B522C082C0837A007B02900EFB
:1019000063E0F912129902949074F6120356900E45
:101910006AE0A2E150568A828B83A3A3A3A3E0F9D5
:101920008A828B83A3A3E0FE8A828B83A3A3A3E096
:10193000FDEEFCEA2406FAEB3400FB120C998A82D5
:101940008B83E58245836024A3A3A3A3A3A3A3A3BE
:10195000E0F89014A7E0686013900E68E054F84433
:1019600002F0900E6A740CF0F9120DA1028F7174DE
:10197000F61203567A007B00121A31120D418A08C2
:101980008B09AE08120D4775080078081207F3900E
:101990000E6AE0F9EEFCAD09121473740112081D11
:1019A0007A007B00121A31028F710207CFC082C009
:1019B00083900598E4F0A3F002A26B74F41203562E
:1019C0008A088B09ECFEEDFF7A077B001211F1EA21
:1019D0004B60508A828B83E508F0A3E509F08A8288
:1019E0008B83A3A37401129A28EEF0A3EF129A2816
:1019F000A3A3E4F0A3F090059812A126700590052A
:101A000098801BE0F9E82405F8E93400F9E8FCE9DE
:101A1000FD8C828D8312A12670EB8C828D83EAF07F
:101A2000A3EBF07F04020563F08A828B83A3A3A358
:101A30002274F6120356EAFEEBFF8E828F83E0F9E2
:101A400012111F8B09EA45096004790280187C0095
:101A50007D00EEFAEFFB1210FB8B09EA45097004DA
:101A600079108002790002A22D74F2120356E9FE69
:101A7000EAFF8B08129C6CEA450D60307A047B000B
:101A8000121185EA4B60258A828B8374FDF0A3E5F1
:101A900008F0EE8A828B83A3A3F0EF8A828B83A364
:101AA000A3A3F0850C82850D83129E857F06020517
:101AB0006374F012035674F41208AF7401120A6DC5
:101AC000EAF0A3EBF0740A120A6DECF0A3EDF074E7
:101AD00005120A6DE9F07420120A6D7808120A2EB8
:101AE0007403120A6D74FFF0A3F07401120A6DE022
:101AF0002402F8A3E03400F97408120A6D12A1421E
:101B00007401120A6DE02404F8A3E03400F97406AD
:101B1000120A6D12A1427401120A6D129C9B701C74
:101B200079FE7406120A6D129CA37003029C621265
:101B30009C747003029C62129C7E80377408120AA7
:101B40006D12A11DF974FF69700D900598129C9398
:101B50007003029C628011129C6CA80CA90DE8FE17
:101B6000E9FFE849600D80CF850E82850F83E0FE96
:101B7000A3E0FFEE4F7003029C62802085108285F7
:101B80001183E0F97406120A6D129CA37003029C83
:101B900062129C747003029C62129C7E850E828588
:101BA0000F8312A2EAE8FCE9FDEC4D8E828F836080
:101BB0001912A114121A8AEA4B601D8A828B8312B1
:101BC0009C8D120A6D12A148800E12A12C60091280
:101BD0009C8C120A6D12A1427401120A6D129E753C
:101BE000A3A3A3A3A3129C8C120A6DE0687003A3A5
:101BF000E069600B8E828F83E0703CE84970387832
:101C0000081207E77422120A6D1206537422120A90
:101C10006D1206537412120A6D120653740F120AD3
:101C20006DE0F9EEFCEFFD740B120A6D12A19F122C
:101C30001113740A12081D7401120A6D129C9B7014
:101C400003029B7C7408120A6D12A11DF4701385A7
